:020000040800F2
:10000000F0FF001059CE05082D58050845E00108FD
:10001000F9CE0508F9CE0508F9CE05080000000064
:10002000000000000000000000000000315805083A
:10003000355805080000000039580508F5A60108E4
:10004000F9CE0508F9CE0508F9CE0508F9CE050860
:10005000F9CE0508F9CE0508C9AF0008D1AF0008F0
:10006000D9AF0008E1AF0008E9AF0008B5AC00085F
:10007000C9AC0008DDAC0008F1AC000805AD000813
:1000800019AD00082DAD0008F9CE0508F9CE050818
:10009000F9CE0508F9CE0508F9CE0508F1AF00083C
:1000A00045C60008A5C5000855C6000895C5000846
:1000B000CDC50008DDC50008EDC50008B1A30008E6
:1000C0005DBB0008B9A3000861BB0008F9CE0508B4
:1000D000F9CE050829A001082DA1010831A20108C7
:1000E000F9AF0008F9CE0508BD8D050865C6000802
:1000F0001DC6000875C600080DC6000841AD000801
:10010000F9CE0508F9CE0508FDC50008F9CE0508A9
:1001100035A3010839A40108D9DA000811DB000869
:1001200055AD000869AD00087DAD000891AD00082F
:10013000A5AD0008F9CE0508F9CE0508F9CE0508E9
:10014000F9CE0508F9CE0508F9CE05083D58050891
:10015000B9AD0008CDAD0008E1AD00083DA501082E
:10016000C1A3000865BB0008F9CE0508F9CE050853
:10017000F9CE0508F9CE0508F9CE0508F9CE05082F
:08018000F9CE0508F9CE0508CF
:10800000074BD0F8E4105B68D0F8F0205B1A9A4276
:10801000B8BFC0F8F030012380F81C310020704751
:10802000001000E0B74B00EB800270B503EBC20418
:1080300053F832205268B2F814C01CF0010F4FEA16
:1080400080016AD15FFA8CFE1EF0020F3DD0BFF3B3
:108050005F8F257F012D5FFA85FC00F0CC80148BAB
:10806000BFF35F8F0C1803EBC404257F022D00F0D3
:10807000E3800C1803EBC404257F032D06D1A47FF5
:1080800024B193F87940002C40F0E5809488A4B2A4
:1080900044F48064948093F978C001EB000E03EB04
:1080A000CE0E9EF81CE00EF1010EE6450CD1002428
:1080B00083F8794093F87A40002C40F0B680084469
:1080C00003EBC00300225A7670BD1EF0040F5BD193
:1080D0001EF0400E00F0C880158A93F978C0666AD9
:1080E000EDB206F80C505FFA8CFE267F0EF101040B
:1080F00064B2E51CAE4283F87840A44600F02A81C1
:108100000D1803EBC5052D7FAC42C6D10EF1020C54
:108110004FFA8CFC83F878C0BFE7B2F800C02CF4AB
:10812000006C4FEA0C4C4FEA1C4CA2F800C0B2F8AD
:1081300000C01FFA8CFC4CF4806CA2F800C0A57F34
:108140004FF0000C83F878C0002D46D093F879509A
:10815000002D3FD0012483F879400C1803EBC404B0
:10816000247F022C04D11488A4B244F40064148047
:108170000C1803EBC404A47E44F0010414820844E8
:1081800003EBC0031B7F70BDA57F4FF0010C83F88C
:108190007AC0002D6FD093F87950002D70D10C1853
:1081A00003EBC404647F002C00F0AE80148893F8C5
:1081B00078C0A4B244F400740CF1010C14804FFA9E
:1081C0008CF483F87840B2F800C01CF4807FFAD1B8
:1081D000A44662E7E47EFF2CBCD00C1803EBC40479
:1081E000A57E05F0FE051582E27EFF2AC7D0FF229C
:1081F00083F87820C3E7A47F002C3FF430AF93F8D6
:108200007940002C3FF42BAF148824F480642404BC
:10821000240C1480BFF35F8F148B148883F87AC00A
:10822000A4B244F40074148030E7948824F44074B9
:108230002404240C948042E7A47F002C3FF419AF5F
:1082400093F87940002C3FF414AF148824F4806430
:108250002404240C1480948824F480642404240CC2
:10826000948093F978C018E71FFA8CF52D0631D465
:1082700093F978C011E793F87940002C8FD095E7F7
:10828000257F022D15884AD925F480652D042D0CF3
:108290001580158A666A93F978C0EDB206F80C501D
:1082A000666A1488A4B244F4007414805FFA8CFCEB
:1082B000158A0CF1010464B2EDB2355595880CF1C4
:1082C000020CADB24FFA8CF445F4806583F8784027
:1082D000958078E793F978506E1C42D0266A765DD7
:1082E0001682247F05F1010C4FFA8CFC644583F85B
:1082F00078C07FF4D2AE948824F480642404240CE3
:108300009480CAE6E81800201488A4B244F480746B
:108310001480012483F8794093F9784053E7ADB293
:1083200045F400751580158A666A93F978C0EDB238
:1083300006F80C505FFA8CFC666A158A0CF1010491
:1083400064B2EDB20CF1030C35554FFA8CF483F89E
:10835000784038E7958825F480652D042D0C9580AC
:10836000CEE6E57E1582A57F83F878E01DB9247FEF
:10837000002C7FF404AF948824F480642404240C3B
:108380009480FCE61B4B01681B4A03F5727C03E0FA
:1083900063452CD053F82C2F9142F9D170B593F846
:1083A00004E0427996450AD0634505D053F82C2F56
:1083B0009142F4D06345F9D14FF0FF3070BD9E4635
:1083C0008468DEF80C50A5424FF0000208D001325C
:1083D000032A0EF10C0EE7D0DEF80C50A542F6D1C0
:1083E000DEF81050C668B542F1D150B270BD4FF002
:1083F000FF30704708E705080000014030B5EAB1DA
:108400008E464FEA014C034600F1C005002419686E
:108410009A6841EA0C0142EA0E029A60C3E900142C
:108420000C33AB42F3D1D0F8C030C0F8C44043EABB
:108430000E03C0F8C030C0F8C84030BD4FEA014E4E
:108440008C46E0E783691969B3F80CC00A6830B458
:108450009C6822F0010224680A60A28992B222EA92
:108460000C02A281027D04681F2A06D96568203AA1
:1084700008209040284245D0FEE72568082090401B
:108480002842F9D1202000FA02F2A260264A12788E
:10849000002A35D01A7E012A39D0D3F8F4200132CF
:1084A000C3F8F420EFF31181502282F31288586848
:1084B0005C6C026822EA04029C6C2243C9B202602E
:1084C00081F31188D3E90C401A6999681D6C096819
:1084D00014605061D3E90E40546090600024B3F8FA
:1084E000A800D5604C62C862106801242043106067
:1084F0001C7683F8F1408A899B8913439BB28B8158
:1085000030BC7047202000FA02F2E260BEE7002291
:1085100083F8F120D3F8F8000A68013022F0010254
:10852000C3F8F8000A60EBE70400001010B40C4C2C
:108530006368002B11DD002004F1080C0146DCF813
:10854000A03003F1C00259600C339342FBD1636841
:10855000013083420CF5807CF1DC5DF8044B704700
:1085600004000010F0B5494C04EB401C9CF8242496
:1085700002B9F0BD464B4FF08C0E0EFB003E93F857
:10858000DC6493F8DD249EF87E708CF80A749642C1
:108590004FF0000C4FEA40158EF87EC00ED002EB73
:1085A000420C03EBCC0C57009CF8E0C40CF1FF3EEE
:1085B000BEF1010F5CD9BCF1030F53D06019A0F8D4
:1085C0000814EFF31182902383F3128890F80A3491
:1085D000B0F8081443EA41030021D2B29BB280F8FC
:1085E0000A1482F311881A09217882EA13225A4068
:1085F000D9B1D0F82044D0F80C14D4F8A040D2431C
:108600001B019BB202F00F0201208840134304F1CA
:10861000C0015A0013F4004F93B202D162680243C2
:1086200062600C348C42F4D1F0BDD0F82014D0F844
:108630000C04D1F8A0401B0100F110019BB202F024
:108640000F0201208840134304F1C0015A0013F4C3
:10865000004F93B202D16268024362600C34A142BF
:10866000F4D1F0BD02F1010C0CF0030CB445A5D01F
:108670003A4403EBC202131893F8ED1400299DD07D
:108680006319012283F80A2498E700BF0400001050
:10869000E8180020704700BF024B03EB401090F831
:1086A00025047047040000104368B0F8502010B44F
:1086B0001A83EFF31182502383F312884168446CCC
:1086C0000B6823EA0403C46C2343D2B20B6082F329
:1086D0001188D0E907418268036912681C605961FA
:1086E000D0E909415C60C46A9960B0F86010DC6050
:1086F0000023D1625DF8044B0376704710B4037D0C
:1087000001681F2B09D94C68203B202202FA03F391
:108710001C4215D15DF8044B70470C68202202FA08
:1087200003F31C42F6D00D4A4068002482F840450D
:1087300002685DF8044B22F0010202608B60704712
:10874000064A4068002482F8404502685DF8044B00
:1087500022F001020260CB60704700BFE8180020E1
:10876000704700BF0B4890F83C1589B101EB4101FF
:10877000002310B4490000F244501C4650F8232056
:10878000063302B114608B42F8D15DF8044B704798
:10879000704700BF040000100B4890F83C1589B1E9
:1087A00001EB4101002310B4490000F244501C4683
:1087B00050F82320063302B114609942F8D15DF8D5
:1087C000044B7047704700BF040000100120704741
:1087D000034B00EB400003EBC00090F855057047D9
:1087E000040000101F4890F83C35002B39D00022BF
:1087F0002DE9F04300F244531B4E1C4D4FF0500E38
:108800004FF02C0C144607E053F8181B0C6090F83E
:108810003C150132914222DD197C0029F4D05F68B9
:10882000B90AA1F5801105EB010952294FF0FE08A4
:1088300098BF99F8F483EFF311898EF31288796A5F
:108840000CFB08680131C8F86C15B98A89B241F08F
:1088500001015FFA89F8B98288F31188D4E7BDE88D
:10886000F083704704000010E818002008E70508AE
:1088700007EE900AB8EE670A704700BFBCEEC00A68
:1088800010EE103A98B270470D4B0E49DB68DB438F
:10889000C3F30223C3F104030122DBB202FA03F3A0
:1088A00001EB000C1B0103F0F0038CF800334309CB
:1088B00000F01F0002FA00F041F82300704700BFEB
:1088C00000ED00E000E100E0122301480B8070475A
:1088D00088010020042301480B8070479C01002080
:1088E0002048D0F8E837D0F8EC2730B59B184FF087
:1088F0001A040C8001D11C4830BD1B4AD0F8EA177D
:108900004FF0000E10467546B3F1204F4FEA137C2E
:108910000CF130040EF1020E2ABF0CF1370C8470FA
:1089200080F802C0BEF1100FC5704FEA031300F1CA
:108930000200E9D100200446B1F1204F4FEA117343
:1089400003F1300C00F102002ABF373382F812C065
:1089500093740828D4744FEA011102F10202EBD19A
:10896000014830BD00F0FF1FA0010020B42282802A
:108970002E224FF4A57C4FF4EB7102814FF48772E5
:108980000023A0F802C0C1804FF4E17C96218281CF
:1089900044220370A0F80AC0C1810282438270475A
:1089A00082B01F4B002201920193019B1D4A0433A8
:1089B0000193019B1968936803F00C03042B07D003
:1089C000082B0AD0184B194AC3F8AC2702B07047DD
:1089D000154BC3F8AC1702B070475368506813F4D6
:1089E000800F00F03F00536813D1C3F388130F4981
:1089F000B1FBF0F101FB03F30A4A0B495268C2F3E1
:108A0000014201325200B3FBF2F3C1F8AC3702B0BD
:108A10007047C3F38813B1FBF0F101FB03F3EBE7FD
:108A20005028004000380240E81800200024F400DC
:108A300038B5074BD3F8B0371B6A14460D46984734
:108A40004FF4007302682A600020236038BD00BF25
:108A5000E818002008B5074BD3F8B03733B15B698D
:108A6000984780F00100404240B208BD4FF0FF300F
:108A700008BD00BFE8180020002070472DE9F04134
:108A800023B3164D164688469F18D5F8B0470023E5
:108A9000A4681A4641463046A0470028F5D0D5F8CC
:108AA000B03733B15B69984720B9D5F8B037002BA0
:108AB000F8D1FEE70136B74208F50078E5D1D5F8E0
:108AC000B437C5F8B8370020BDE8F081034DD5F8BC
:108AD000B437C5F8B8370020BDE8F081E8180020A9
:108AE0002DE9F0415BB31A4C16460F4603EB020822
:108AF00004E0D4F8B01719B14B699847D4F8B0170F
:108B00000D6900231A4639463046A8470028F0D19F
:108B1000D4F8B03733B15B69984720B9D4F8B0378F
:108B2000002BF8D1FEE70136B04507F50077E5D117
:108B3000D4F8B437C4F8B8370020BDE8F081044C4D
:108B4000D4F8B437C4F8B8370020BDE8F08100BFCE
:108B5000E818002000207047034B93F8E007003826
:108B600018BF0120704700BFE8180020826D136A0B
:108B70005B681B78FF2B08D090F8F030013BDBB22C
:108B800080F8F0301BB10120704700207047126A56
:108B90005268022013707047836D1B6A5B681B78F4
:108BA000FF2B0AD190F8F030002B03F1FF3280F850
:108BB000F02014BF0120022070470020704700BF42
:108BC00010B5124C12498CB0002384460DF10700F9
:108BD0000122CDE90230069104F6140002A90492A4
:108BE0008DF82820CDE907338DF8143009930B93C5
:108BF00084F8ACC810F0A4FAD4F81428136A002B37
:108C0000FCD19DF807000CB010BD00BFE818002093
:108C1000998B000870B5054690B008200C46FFF708
:108C2000CFFFFF2826D0FE2802D0022010B070BD52
:108C3000124E039400230220CDE90730012201A93E
:108C400006F61400CDE90135CDE90533CDE90A3347
:108C5000CDE90C338DF810308DF824300F938DF85A
:108C6000382010F06DFAD6F81438186A0028FCD1B4
:108C700010B070BD012010B070BD00BFE81800201A
:108C800030B51E4D91B00023FD200DF103010122EE
:108C9000CDE905318DF8030001A905F61400CDE9F1
:108CA0000133CDE90732CDE90A33CDE90C33C5F8FC
:108CB000DC378DF810308DF824300F9303928DF847
:108CC000382010F03DFAD5F814381C6A002CFCD17D
:108CD0000120FFF775FFFF2809D0D5F8B437C5F894
:108CE000D0370922204685F8E02711B030BD042393
:108CF000022085F8E03711B030BD00BFE818002031
:108D0000034B93F8E007032894BF0020012070472D
:108D1000E818002000487047CC20002030B4194BE0
:108D200000209C7B14B11D688D4206D001300B28B9
:108D300003F11003F5D130BC70479AB1124B03EB2D
:108D400040218A4219D0114B93F8E4278AB1104B85
:108D500001225A7000F5B17003EB001001238371FA
:108D600030BC70470A4B00F5B17003EB0010827104
:108D7000E1E7012283F8E427E9E7022CE3D1183B7D
:108D8000E8E700BF804600208030002068400020D7
:108D90006830002030B41D4C002384F8D03604F530
:108DA000C36004E001330B2B00F1100015D00568FF
:108DB0008D42F7D190F80EC0BCF1030FF2D1C2B1D1
:108DC000134901EB4320824209D1A1F1180203F5B6
:108DD000B17302EB031301229A7130BC704794F80F
:108DE000E42712B9012284F8E4270A4A01215170CC
:108DF000EDE70849D4F8CC2603F5B17301EB031372
:108E0000013204219971C4F8CC26E6E768400020BD
:108E10008030002068300020A8B183681BB10E4B61
:108E200007229A7070470C4A1178D36003294FF0DB
:108E300004000CBF80214FF48071C2E9011113615D
:108E4000137590707047044A02F5805101235370E6
:108E500081F8E437704700BF6830002010B5164C29
:108E6000D4F810386BB11A689B88116994F80D28F2
:108E70000B4022B12BB1002384F8E03710BD002B4A
:108E8000F9D094F8E037032B0FD894F8D437013396
:108E9000DBB2072B84F8D437EDD8D4F8B427C4F864
:108EA000D027012384F8E03710BD044810F0BAFA47
:108EB000A4F81808E9E700BFE8180020801A0600A7
:108EC00070B5224B93F8DC2493F8DD349A4237D105
:108ED0001F4D95F80436E3B195F808461D4B002068
:108EE00040F20D3CB4B19A689989516016681968CE
:108EF00046F001061660A1F848C08A8992B242F491
:108F000080728A8195F804260130824203F11803A9
:108F1000E8DC70BD1A68118821F080010904090C91
:108F200011809988D162118889B241F08001118045
:108F30005462998A9689314389B291819C82E1E792
:108F400051F076F90028C3D170BD00BFE8180020A9
:108F500004000010982100202DE9F0411E4B93F8E9
:108F6000DC2493F8DD349A422FD11C4F7D68002D0C
:108F700012DD3846002410F8086BA046013416B103
:108F8000037E012B1CD002691368AC4243F001033D
:108F900000F580701360F1D111F0F6FBD7F80C46A4
:108FA000002C0BDD0E4A02EBC404116893888889FB
:108FB000083203439BB294428B81F6D1BDE8F08125
:108FC00080F8F080FFF770FBDDE751F031F9002801
:108FD000CBD1BDE8F08100BFE818002004000010EC
:108FE000140600102DE9F04F037D02681F2B83B09B
:108FF000044609D95068A3F120052021A940014267
:1090000007D103B0BDE8F08F1068202199400142DC
:10901000F7D05149514D4968C5F8301695F80816F2
:10902000A7694F4E19BB8C2101FB0761D1F8840061
:10903000D1F8FCE0D0F800C0DEF80000B1F888807C
:1090400020F00100CEF80000BCF80C1089B221EA33
:109050000801ACF80C10297801BB1F2B6FD9A3F1C4
:10906000200120238B40D36003B0BDE8F08F8C211A
:1090700001FB0761D1F88410D1F810C00868DCF852
:10908000001021F00101CCF80010818921F48071D9
:109090000904090C818129780029DED04FF08C0861
:1090A00008FB07F806EB08032E49D3F8FCA0D3F819
:1090B00084200193504608F11809D2F800B0894481
:1090C0004CF09AF8019BD5F838262649012083F800
:1090D000D000002A3AD0BBF800309BB243F08003A6
:1090E000ABF8003008F174084FF0FF334144CBF87F
:1090F0002C3058464CF006FA8C2303FB07660023FD
:109100004946C6F8A03050464CF00CF9D6F8FC3071
:1091100016225A601A6842F001021A60D6F88420BA
:10912000B6F88830126891890B439BB293810A4943
:10913000237D49682268C5F834161F2B8FD820215B
:1091400001FA03F3936003B0BDE8F08F11F01CFB4C
:109150000449C5F83806BEE7001000E0040000101E
:10916000E8180020641900202DE9F04111F00CFBF3
:109170001F4F204E05464FF000087C68002C2ADD6A
:1091800000231A4607EB0321013391F8F9109C42A2
:1091900042EA0102F6D142EA0804E4B2904673685A
:1091A000C3F30803A3B9EFF311838BB913F07EFB6C
:1091B000431BB3F5FA6F02DCB8F1000FDDD124B127
:1091C0000D4B93F87029542A09D02046BDE8F08150
:1091D00011F0AEFAECE744464FF00008DFE7B3F8D1
:1091E00078290132A3F878292046BDE8F08100BF34
:1091F0000400001000ED00E0E8180020BA4B1B78D6
:109200000BB9012070472DE9F04FB84DB849D5F89A
:10921000B427B84BA1FB02125209A3FB023A4FEA52
:10922000DA0A0AEB8A0AA2EB4A0A85B0AE4A5FFA6A
:109230008AF3039302F61C1302F23C6701930023A6
:1092400007EB8A0A02F581699846A74BD3F8243ABE
:10925000434540F31481D9F81830D9F80460D3E9B4
:109260003A34029311F090FA029B95F870C902907B
:109270004FEA860E95F884090EF1085E04F18061CC
:109280000EEB431E3939BCF1540F0EEB81110EEB7E
:10929000801301D1A5F87A09994240F266811A68D3
:1092A000002A00F05A811A6C002A00F06C81D3F871
:1092B0008020002A00F06981D3F8C02003F5807374
:1092C000002AE9D1A3EB0E0E99424FEAAE1E40F2FE
:1092D0004C81A4EB0E0145294FF0000428BF452125
:1092E00003EB81119B46204626460DE01A6C002AAE
:1092F00040F0CD80D3F88020002A40F0F380D3F8EE
:10930000C02003F580732AB9994206D91A68002A49
:10931000ECD04033994200F2BE80112E344640F228
:109320002881D6F1150200F124817349029E4B6B0E
:109330009E45D5F8883938BFC1F834E0F11A0029C4
:1093400017DB03F5F42303F590739E4288BF029B5D
:10935000694988BF0533C5F88839674B5B6B052BB6
:1093600086BF053BDBB2002385F884394FF0FF331D
:109370004B6342B100FA02F2C4F11404012000FA76
:1093800004F444EA02005D4BC0F3C43203EB8202F2
:10939000D2F8481400F01F0203EB8202D2F84824EE
:1093A00042EA0131C0F3441203EB8202C0F384208D
:1093B00003EB8000D2F8483441EA0311D0F8483476
:1093C00041EA032181EA112383EA131303F00F0317
:1093D0000F2B40F0B080B1F5803F80F0AC80BCF145
:1093E000540F4FEA111104D1B5F874390133A5F8BF
:1093F00074393D4AD2F82439B1F5606F03F10103A5
:10940000C2F8243900F0D380019B998197F8583035
:109410000398834210D0DAF808203B689B1A3B601F
:10942000DAF830207B689B1A7B600023CAF808308A
:10943000CAF8303087F858003B6801333B60DAF8EF
:1094400008300133CAF808304FF6FF73994207D14C
:109450007B6801337B60DAF830300133CAF8303092
:10946000019B08F101081433B8F1080F07F15C07FC
:109470000AF15C0A019309F120097FF4E6AE1A4A69
:109480000123012082F8203A05B0BDE8F08F803337
:1094900099427FF642AF5A469A1A9211541C184AC2
:1094A00082FB04B2A2EBE472012AB8BF0122904011
:1094B00001241644013A04FA02F210431C462268C1
:1094C00002B3226C002A62D0D4F88020002A60D037
:1094D000D4F8C02004F58074AAB1A142EFD89B460D
:1094E000234611E7C03315E704000010E8180020F8
:1094F0001F85EB51CDCCCCCC8801002008E70508B6
:10950000565555554034A142E9D9E31A9B115A1CCE
:109510002F4B83FB02B3A3EBE273012BB8BF0123F4
:1095200098401E440122013B02FA03F318432346EC
:109530009B462346E8E6BCF1540F2CD0254AD2F8CE
:1095400024390133C2F82439224AD2F820390133B0
:10955000C2F820394FF6FF7158E74033A3EB0E0EE7
:1095600099424FEAAE1E3FF6B4AE10B1013885F80D
:109570008409BCF1540F7FF473AFB5F87639013329
:10958000A5F876396CE780339CE6C0339AE68034E0
:10959000B9E7C034B7E7B5F874390E4A0133A5F816
:1095A0007439D2F824390133C2F82439CCE795F85C
:1095B000DD3403EB430305EBC303434493F8ED347D
:1095C0000D2B7FF421AF019A802393771EE700BF14
:1095D000565555550400001010B5044654F054FA81
:1095E00081B22046BDE81040FEF7BCBF38B50B4D38
:1095F00000EB400005F2445303EBC00393ED027A05
:10960000D3ED037AE7EE007AC4002C44B0EE670A8B
:1096100054F03AFAD4F84435186038BD040000100C
:109620000C4AF8B5136855692B4003EA00055561EB
:109630007DB1094F0126B5FA85F4C4F11F0407EB8B
:10964000840306FA04F4D3F88C0903689847A54309
:10965000F1D1F8BD003C0140E8180020038A2DE953
:10966000F047B0F80C901FFA89F919EA03092BD0DA
:1096700005460E464FF000474FF00008B9FA89F34F
:1096800027FA03F2D24391B21B3B298209EA02096D
:10969000042B16D8DFE803F0352C231A0300B36A35
:1096A000002B37D003F1FF3A1FFA8AFAC6F8288058
:1096B000746A34B123682046514698476468002C88
:1096C000F8D1B9F1000FD9D1BDE8F0877068696BA6
:1096D000036889B29847B9F1000FCFD1F4E7B068B9
:1096E000A96B036889B29847B9F1000FC6D1EBE7BF
:1096F000F068E96B036889B29847B9F1000FBDD1F2
:10970000E2E73069296C036889B29847B9F1000F24
:10971000B4D1D9E7E96A1FFA81FAC9E70A4608B560
:10972000054920B905484CF013F8034808BD044822
:109730004CF00EF8004808BDB4220020645E060814
:109740008C5E060810B5044C04480A4621464BF0CE
:10975000FFFF204610BD00BFB4220020B45E060803
:1097600010B5044C04480A4621464BF0F1FF204650
:1097700010BD00BFB4220020C85E060810B5044C1E
:1097800004480A4621464BF0E3FF204610BD00BFC7
:10979000B4220020D45E060810B5104CD4F8CC2AB0
:1097A00094F8CB3A2AB103F001039BB9136892886D
:1097B0001A8350F031F802E05B69984720B9D4F879
:1097C000B037002BF8D1FEE7D4F8B437C4F8B83777
:1097D000002010BD136892885A83EAE7E818002039
:1097E00010B592B00A0E04468DF805200A0A00232F
:1097F000080C44F0400C8DF807200122CDE9073316
:10980000CDE90D338DF804C08DF806004FF0950CAE
:1098100017488DF8081004938DF818300A928DF8C7
:109820002C300F938DF84020119301A906220DF1E1
:1098300003038DF809C00C900391059209934FF032
:10984000BBFF00B98CB90B4C082303A904F6140024
:1098500084F8AC380FF074FCD4F81428136A002B89
:10986000FCD19DF8030012B010BDFF2012B010BD56
:10987000998B0008E81800202DE9F041314C05468D
:10988000884617461E4694F8E007042839D0082871
:1098900007D1D4F8D837AB4206D0FFF7F1F9022848
:1098A000F1D00120BDE8F081FC23D4F8142884F81D
:1098B000D83A117B244BC3F8608051B1526942B150
:1098C00094F89C28002A0CBF4FF480724FF4007269
:1098D00001E04FF480729A661C491D480FF030FC7D
:1098E00001220623C4F8BC87C4F8C057C4F8C8775F
:1098F000C4F8CC6784F8C42784F8E0370020BDE8BA
:10990000F08194F8D63753B969021820FFF768FF41
:1099100038B994F8E037082BC6D0FE23C5E72946AE
:10992000F3E7D4F81428136A002BFCD151F016FA8F
:10993000D4F81C3813B11A689B881383FFF78EFA8A
:109940000320AFE7E818002088010020C0010020B4
:10995000FC20002070B5234E96F8E037042B054616
:109960000C4609D0082B21D1D6F8D837834236D0FF
:10997000FFF786F9022819D100213720FFF730FFC1
:1099800021461720FFF72CFFC0B996F8D6377BB9D0
:1099900069021920FFF724FF80B9082386F8E03711
:1099A000C6F8DC47C6F8D857022070BD012070BD4C
:1099B00029461920FFF714FF0028EED0D6F8142806
:1099C000136A002BFCD151F0C9F9D6F81C3813B139
:1099D0001A689B881383FFF741FA032070BD0220A9
:1099E00070BD00BFE81800202DE9F843214D95F81F
:1099F000E047042C8046894617461E4608D0082CAE
:109A000002D00020BDE8F883FFF73AF90228F8D128
:109A100095F8D637B3B141461120FFF7E1FEC0B942
:109A2000D5F8B437C5F8BC97052285F8E027C5F806
:109A3000C087C5F8C877C5F8CC67C5F8D03701200E
:109A4000BDE8F8834FEA48211120FFF7C9FE00283E
:109A5000E6D0D5F814381C6A002CFCD151F07EF900
:109A6000D5F81C38002BCCD01A689B88138320466D
:109A7000BDE8F883E8180020817899B10C48D0F847
:109A8000DC3A102B0FD003EB430202444FF0200CC2
:109A9000013382F8E01A012182F8E1CA82F8E21A61
:109AA000C0F8DC3A70470521002013F05DB900BF13
:109AB000E81800202DE9F041B34C94F80C6894B0FC
:109AC000002E00F0B28194F8E03704F2FC775A1EC1
:109AD000082A00F24681DFE812F03B007300BC0068
:109AE000440132015B011B00440109004FF064FE98
:109AF000002840F0FB82D4F8D037D4F8B427FA33EA
:109B0000934280F02B81FFF7A9F994F8E037DEE764
:109B10004FF052FE0028EED0D4F8DC270023012AB3
:109B200084F8D43740F20E83D4F8D817013A0131C3
:109B30000823C4F8DC27C4F8D81784F8E037A3F169
:109B40000806B6FA86F67609304614B0BDE8F0810C
:109B500000210846FFF744FED4F814280546136A8E
:109B6000002BFCD151F0FAF8D4F81C3813B11A6864
:109B70009B881383012D40F0F1804FF0000840F2E4
:109B8000AB11082084F8D587FFF72AFE052800F0DE
:109B9000B181012800F06681D4F81428136A002BE3
:109BA000FCD151F0DBF8D4F81C3813B11A689B884B
:109BB000138394F8D537002BBFD0022384F8E03705
:109BC00094F8D5370021022B0CBF4FF080450D468D
:109BD0003720FFF705FE29462920FFF701FED4F8BC
:109BE00014280546136A002BFCD151F0B7F8D4F8BD
:109BF0001C3813B11A689B881383002D40F0AE8087
:109C000094F8D537022B00F0E18184F8D657002173
:109C10000920FFF7E5FD002800F071810025D4F848
:109C20001428136A002BFCD151F098F8D4F81C3892
:109C300013B11A689B881383002D00F08F800021D8
:109C40000A20FFF7CDFD002840F08D81032384F822
:109C5000E037102105A8FEF7DDFF00287ED1BDF812
:109C600015209DF81C309DF8141084F8EA1752BA9C
:109C7000A4F8E8279DF8172084F8EB279DF8182012
:109C800084F8EC279DF8192084F8ED279DF81A2018
:109C900084F8EE279DF81B2084F8EF2703F00F01CE
:109CA0001A099DF8213084F8F4271B019DF8222021
:109CB000DDF81D0084F8F517DBB243EA121302F059
:109CC0000F0200BA03F5FA6384F8F827D4F81428D1
:109CD000C4F8F007A4F8F637136A002BFCD151F052
:109CE0003DF8D4F81C3813B11A689B88138394F894
:109CF000D637ABB94FF400711020FFF771FDD4F8DF
:109D000014280546136A002BFCD151F027F8D4F82B
:109D10001C3813B11A689B881383002D7FF4F3AEAF
:109D20001A480FF07FFB00220423A4F818083046DD
:109D3000C4F8DC2784F8E03714B0BDE8F081D4F82B
:109D4000BC074FF40071FEF765FF012800F0AB80FF
:109D5000022800F0B080002800F0158194F8E03768
:109D60005A1ED2B2022A0BD8D4F8B427D4F8D0178E
:109D7000521AC82A7FF6E3AEFFF770F894F8E0377E
:109D8000042B7FF4DCAEDFE6E818002040787D018C
:109D9000D4F81428117B136A00294CD05269002A88
:109DA00049D094F89C28002A45D0B3FA83F35B0984
:109DB000002BD3D004AA002305920222CDE906325B
:109DC0000DF10F020B92C548ADF81030012205A924
:109DD000CDE90933CDE90E33CDE910338DF82030CC
:109DE0008DF8343013930C928DF848200FF0A8F9B9
:109DF000D4F814381D6A002DFCD19DF80F3003F003
:109E00001F03052B00F08681FFF728F8D4F8C887D8
:109E1000B8F1000F6BD0D4F8CC37D4F8C0172A466D
:109E20000120C04794F8E03751E6304684F8E067F7
:109E300014B0BDE8F081D4F8BC3794F8C417A74833
:109E400003EB01214FF480724FF070FC94F8C4379B
:109E50000133DBB284F8C437A3F10203B3FA83F30E
:109E60005B09A5E704AB06939C488DF834500423A6
:109E700005A9CDE90988CDE90B88CDF814808DF8C6
:109E80002080CDF8388007930FF05AF9D4F81428C1
:109E9000136A002BFCD19DF81330AB2B04BF0223B7
:109EA00084F8D5377AE6D4F8D037D4F8B4276433B9
:109EB0009342BFF453AFD4F81428136A002BFCD19B
:109EC00050F04CFFD4F81C3813B11A689B881383E8
:109ED000FEF7C4FFD4F8C8574DB10022D4F8CC37F0
:109EE000D4F8C0171046A84794F8E037EFE594F887
:109EF000E037ECE5D4F8142884F8D5574EE6102165
:109F00003846FEF787FE00287FF488AE94F80B38B9
:109F1000DB077FF583AE94F8FC17891100F08F8082
:109F200001297FF47BAE94F80328DFF8B4C19200D6
:109F30000546D2B216210220C0F108038B4228BF89
:109F40000B46C3F1080002419D40C91A45EA0205CB
:109F50004FF000001CF8012FEED16B1C9B02C4F8DF
:109F6000E43735465BE6D4F81428136A002BFCD19D
:109F700050F0F4FED4F81C38002B3FF4C4AD1A683E
:109F80009B881383BFE5D4F81428136A002BFCD1F7
:109F900050F0E4FED4F81C3813B11A689B88138380
:109FA000D4F8C8570423002084F8E03784F8D40795
:109FB000002D3FF4C9ADD4F8CC37D4F8BC27D4F881
:109FC000C017A84794F8E0375A1ECAE629463A2037
:109FD000FFF706FC04AB0693042307938046012396
:109FE0003E488DF8343005A9CDE90955CDE90B552A
:109FF00005958DF820500E950FF0A2F8D4F814387E
:10A000001A6A002AFCD1B8F1000F11D11A6A002A8D
:10A01000FCD150F0A3FED4F81C3813B11A689B8809
:10A020001383049B1BBAC3F3807384F8D637EEE521
:10A030001A6A002A9CD01A6A002AF9D198E794F883
:10A04000013894F80508DFF89CE003F00F03800165
:10A0500001255FFA80FC9D4006200323C0F1080221
:10A060009A4228BF1A46C2F108004CFA00F091400B
:10A070009B1A41EA00011EF801CF4FF00000EDD11C
:10A0800094F802E8DFF860804FEA8E1E02315FFA32
:10A090008EFE4FF00C0C062200E00022C2F10802F6
:10A0A000624528BF6246C2F108004EFA00F09340B4
:10A0B000BCEB020C18F801EF43EA0003EDD10133C9
:10A0C0008B40E917A3FB055203FB01226D0A45EA09
:10A0D000C255C4F8E4573546A1E500BFFC20002076
:10A0E000EB200020ED200020EA200020D4F81428E6
:10A0F000136A002BFCD1019050F030FED4F81C38CC
:10A10000019813B11A689B881383042384F8E037FD
:10A11000064619E5D4F8C857D4F8B427C4F8D027B0
:10A12000072384F8E037002D3FF409ADD4F8CC378D
:10A13000D4F8BC27D4F8C0170120A84794F8E0371A
:10A140005A1E0EE615D00423D4F8142884F8E037FC
:10A15000136A002BFCD150F001FED4F81C38002B00
:10A160003FF4FCAD1A689B88138394F8E0375A1EBD
:10A17000F7E5FEF785FD02287FF4F0ADD4F814383A
:10A180001A6A002AFCD1E6E7084B10B5D3F8103B59
:10A1900018440C46807D0FF0FDFB18B182880368DF
:10A1A0000CB11A8310BD5A83FCE700BFE8180020E9
:10A1B00010B42A492A4A91F804367BB3D2F8B04841
:10A1C000A04239D0012B29D0D2F8C848844239D0D6
:10A1D000022B23D0D2F8E048A04235D0032B1DD06B
:10A1E000D2F8F848A04231D0042B17D0D2F8104949
:10A1F000A0422DD0052B11D0D2F82849A04229D059
:10A20000062B0BD0D2F84049A04225D0072B05D011
:10A21000D2F85849844208BF07230ED003F1010C3D
:10A2200081F804C603EB430102EBC1025DF8044B65
:10A23000C2F8B008184670470023DBB218465DF834
:10A24000044B70470123F8E70223F6E70323F4E702
:10A250000423F2E70523F0E70623EEE704000010ED
:10A26000E818002038B5424C8C2303FB004393F8D8
:10A270008B3003B938BD94F8DCC494F8DD349C45C8
:10A280000ED003EB430204EBC20292F8E0E40EF1BD
:10A29000FF35012D4FEA430246D9BEF1030F3ED0F0
:10A2A0008C2202FB0042A2F87C10EFF31181902374
:10A2B00083F31288B2F87C5092F87E3043EA45036B
:10A2C0000025C9B29BB282F87E5081F311882949DA
:10A2D0001A090D7882EA13225A4005B1D2431B01B4
:10A2E0009BB202F00F021A4391F808365BBB8C2335
:10A2F00003FB0044D1F8283AD4F80401012198471F
:10A30000D4F80011B4F888508A8AD4F8FC302A4373
:10A310008A8258601A6842F001021A6038BD5D1CDA
:10A3200005F003056545BBD0134404EBC3030344A8
:10A3300093F8ED140029B3D08C2303FB00430122D2
:10A3400083F87E20ACE78C2303FB0044D1F8285A25
:10A35000D4F88430D4F800115B79086903F0FC0369
:10A3600018440421A847D4F800318000988138BDF2
:10A37000E81800200400001043680B4A23F04073E3
:10A3800023F4807343F48073436083681A4042F07F
:10A3900002028260C36A0139CAB223F4700141EA41
:10A3A0000251C162704700BFFDF7FFC0704700BF98
:10A3B0000020FDF737BE00BF0120FDF733BE00BF10
:10A3C0000220FDF72FBE00BF10B1036882881A83F8
:10A3D000704700BF10B1036882885A83704700BF7E
:10A3E00010B404698269E468416814604024D46050
:10A3F000446900230C31C2E90433C2E90633C2E9DF
:10A400000833C2E90A33C2E90C33936093635160A5
:10A4100084B1C269E0689363C2E90233C2E90433DC
:10A42000C2E90633C2E90833C2E90A33C2E90C3390
:10A43000C2E900015DF8044B704700BF4368002289
:10A440001A60037D1F2B08D9203B2022016802FAE5
:10A4500003F343F01803CB6070472022016802FA2F
:10A4600003F343F018038B60704700BF0268136A60
:10A4700011B1D96901B3143330B49C681D68916976
:10A48000DDB14FF4806088618D60104640690C61D9
:10A4900080B15968D369C9B10A464FF480619A60A6
:10A4A0009961224312F0010F14BF00224FF40052B1
:10A4B0001A621C6130BC704770478D61054D4FF0CA
:10A4C000FF0C05F888CF00688D60DFE7024A9A60CC
:10A4D0009961E6E788010020FC2300200168F8B5B7
:10A4E000D1E9042304465568002B49D09861107DBA
:10A4F0005E681F2831D81768202202FA00F040F069
:10A500001800B8601A7D1F2A32D91868203A202313
:10A5100003FA02F242F01802C26000232B6033609B
:10A520003368896943F01003336028464AF0FAFE25
:10A5300023683046D9694AF0F5FE2B68226843F05B
:10A5400001032B603368526843F001033360938842
:10A550009BB243F003039380F8BD17682038202294
:10A5600002FA00F040F01800F8601A7D1F2ACCD8DB
:10A570001868202303FA02F242F018028260CCE746
:10A58000137D90611F2B1CD81068202202FA03F360
:10A5900043F01803836000232B602B68896943F024
:10A5A00010032B6028464AF0BDFE2B68226843F05A
:10A5B000010352682B6093889BB243F0020393809F
:10A5C000F8BD1068203B202202FA03F343F0180381
:10A5D000C360E0E72DE9F0417F4D804E07463C68BF
:10A5E00097F888806368B888012284F824201A8844
:10A5F00022F040021204120C1A802289824223D0D7
:10A60000198821F038010904AB424FEA114100F0EA
:10A61000BF80734A934200F0BB800246B2F5807F50
:10A62000A8BF4FF48072022AB8BF0222002A92FA11
:10A63000A2F2B2FA82F208BF4FF0FF32013A41EAC9
:10A64000C20292B21A802081397BA27A8A420CD04F
:10A650001A8822F003021204120C1A801A8892B28D
:10A66000002900F092801A80A1721A8892B242F0FA
:10A6700040021A80226A9168002900F0A3804FF0FE
:10A68000000C1432E64652F8100C8E4400EA060123
:10A6900020B1B1F1805F23D0616909B352F8140C85
:10A6A000143200EA060110B1B1F1805F18D052F8FF
:10A6B0000C1C0CF1010C0029E5D1227B82B1B8F110
:10A6C000000F0DD0BCF1010F6FD8BEF1070F6CD891
:10A6D0000CEB8C018900226A11440A7B002A64D0A9
:10A6E000226A92684FF00008002A53D0B8F1000F98
:10A6F00002D098F80C2022B1BA6812B11168928881
:10A700004A83226AD2F800E0226A5168226A92687B
:10A71000501E9AB1BEF1000F23D01EF801CB1A894A
:10A720009207FCD5A3F80CC01A89D207FCD59A89E8
:10A7300092B209B101F8012B0138EBD2236A1B7BDD
:10A74000E3B9236A1B697BB1236AD7F894001B69BC
:10A75000984701280DD0022806D100232362BDE8C6
:10A76000F0814FF0FF0CDAE7D4F82080236A14332D
:10A770002362236A9B686BB16368B7E7BB68002BF1
:10A78000DFD01A689B881383DBE742F003026AE795
:10A79000420843E7236A1B68DBB1236AD3E90072EE
:10A7A00022620022C3E9002219E700213846FFF7A0
:10A7B0005DFEBB6813B11A689B8853833846BDE8B9
:10A7C000F0418BE6227B002A8AD0B8F1000F82D1BB
:10A7D00086E72362C3E700BF003800400000FFFFA8
:10A7E000003C004038B5D0F8E0102B4B04465A68C6
:10A7F000D0F8D80071B1131A99420BDC94F8D0301C
:10A80000C4F8D820012B10D0D4F8D4300133C4F8C8
:10A81000D43038BDD4F8E430C4F8D8200344C4F8A8
:10A82000DC3094F8D030012BEED16168201D04F1AA
:10A83000E805EFF3118C102383F3128863681B6A19
:10A840000BB3D4F8F0302A461BB1D3691432002B75
:10A85000FBD10B6A6BB1996839B9934209D0196879
:10A8600029B15B6899680029F7D01433F3E7C3E98D
:10A8700000055FFA8CFC8CF31188D4F8D4300133D6
:10A88000C4F8D43038BD0D625FFA8CFC8CF31188AB
:10A89000FFF7A0FEB8E700BF001000E02DE9F0418F
:10A8A000826992F8DC30012B8AB005464CD0023B1D
:10A8B000012B54D892F84C31D2F89C202E4C63F0E6
:10A8C0007F0313708669D6F8A030D6F8108003F1A4
:10A8D000010E0FCCEC46ACE80F00D6F89C30CDE969
:10A8E000003E0FCCACE80F0094E8030006F110071F
:10A8F0008CE80300EFF31180102383F3128833698F
:10A900001B6A002B2FD0029B6A461BB1D3691432FD
:10A91000002BFBD1D8F8203073B1996839B9934234
:10A920000AD0196829B15B6899680029F7D01433F7
:10A93000F3E71F60C3F804D0C0B280F31188AA699E
:10A9400011690B6A002BFCD1D2F8A0305A8852BA98
:10A95000EA819A8852BA2A82DB885BBA6B8201202C
:10A960000AB0BDE8F081C8F820D0C0B280F31188E9
:10A970003846FFF72FFEE2E7D0EB05082DE9F0415E
:10A9800090F8DC30D0F8A050012B8AB0044672D089
:10A9900016D8D0F89C304FF0FF321A605A609A6097
:10A9A000DA60D0F8E0300522B3F57A7FC0F8F02005
:10A9B0007CD8032380F8DC3001200AB0BDE8F081A8
:10A9C000023B012BF8D890F84D31D0F89C20524E24
:10A9D00063F07F031370D0F8A030D0F8108003F13B
:10A9E000010E00F110070FCEEC46ACE80F00D4F8D2
:10A9F0009C30CDE9003E0FCEACE80F0096E8030096
:10AA00008CE80300EFF31180102383F3128823698D
:10AA10001B6A002B73D0029B6A461BB1D3691432A8
:10AA2000002BFBD1D8F8203073B1996839B9934223
:10AA30000AD0196829B15B6899680029F7D01433E6
:10AA4000F3E71F60C3F804D0C0B280F31188226915
:10AA5000136A002BFCD16B885BBAA4F8D030AB88AA
:10AA60005BBAA4F8D230EB8801205BBAA4F8D430EA
:10AA70000AB0BDE8F08190F84C2190F84D319B1A56
:10AA80005B100133DBB205EB430235F813305BBAE0
:10AA9000A0F8D03053885BBAA0F8D23093885BBA64
:10AAA000A0F8D43001200AB0BDE8F08103691A7B18
:10AAB00072B35B6963B390F898304BB390F84C3144
:10AAC000D0F89C20C4F8A40063F07F03137090F8C2
:10AAD0004C1190F84D31D0F8A0201048C4F8040172
:10AAE0005B1A07330121C4F8FC30D4F89C3084F899
:10AAF00000110A44C4E93D3284F8DC105CE7C8F870
:10AB000020D0C0B280F311883846FFF763FD9EE77E
:10AB1000022384F8DC304FE7D0EB05080180000801
:10AB200008B51D200EF036FF08B183794BB11E2009
:10AB30000EF030FF08B1837903B108BD5523C380FF
:10AB400008BD5523C380F2E7D3B2012B23D870B5DB
:10AB500002EB4202114C4FEA820E4FF0000C2246EB
:10AB60000EF10805634604E00133152B11D012F8ED
:10AB70001CCF6045F8D192F801C08C45F4D15659EC
:10AB8000002EF1D0C3EBC3030EEB83030433E018B4
:10AB900070BD002070BD0020704700BFF8EB0508B5
:10ABA00010B40C4C002304F6183C01E0152B0CD01B
:10ABB00003EB430201331CF802108142F6D1224418
:10ABC0005DF8044B92F91A0B70474FF0FF305DF8B7
:10ABD000044B7047E8180020D3B2022B21D830B5BF
:10ABE00002EB4202104D114C4FEA820C0CF10C0E9C
:10ABF0002A46002304E00133172B10D052F82C4FC3
:10AC0000A042F8D114798C42F5D152F80E40002CB4
:10AC1000F1D02C2202FB03C30833E81830BD00201A
:10AC200030BD0020704700BF08E705080000014064
:10AC3000002838D030B51C4D90F804C0002305F62C
:10AC4000183401E0152B2CD003EB43020133A15C37
:10AC50006145F7D12A44046892F91A3B90F805E05F
:10AC6000DAB2022A1DD803EB4303104810494FEA19
:10AC7000830C02460CF10C05002304E00133172B72
:10AC80000FD052F82C1F8C42F8D111797145F5D1B3
:10AC900051590029F2D02C2202FB03C30833184477
:10ACA00030BD002030BD7047E818002008E70508D7
:10ACB000000001400348D0F89C300BB18C3018479D
:10ACC000704700BF880100200348D0F8C0300BB1A6
:10ACD000B0301847704700BF880100200348D0F803
:10ACE000E4300BB1D4301847704700BF8801002012
:10ACF0000348D0F808310BB1F8301847704700BF4F
:10AD0000880100200348D0F82C3113B100F58E7073
:10AD100018477047880100200348D0F8503113B11C
:10AD200000F5A07018477047880100200348D0F84C
:10AD3000743113B100F5B2701847704788010020D4
:10AD40000348D0F8983113B100F5C4701847704724
:10AD5000880100200348D0F8BC3113B100F5D6704B
:10AD600018477047880100200348D0F8E03113B13C
:10AD700000F5E87018477047880100200348D0F8B4
:10AD8000043213B100F5FA701847704788010020AB
:10AD90000348D0F8283213B100F506701847704701
:10ADA000880100200348D0F84C3213B100F50F7031
:10ADB00018477047880100200348D0F8703213B15B
:10ADC00000F5187018477047880100200348D0F834
:10ADD000943213B100F521701847704788010020A4
:10ADE0000348D0F8B83213B100F52A7018477047FD
:10ADF00088010020094B0A4A013800EBC00003EB30
:10AE00008000116BD0F88C30064883420CBF4FF4A1
:10AE100000134FF480030B43136370478801002035
:10AE2000003802400060024070B501383C4C3D4D96
:10AE300000EBC00C04EB8C0C9646DCF88C603A4AB4
:10AE4000AE420CBF4FF400154FF48005166B35432E
:10AE50001563CCF89C10CCF8A4303449DCF8903061
:10AE60008B424FEAC0023ED001F580618B423AD05E
:10AE7000A1F57A718B4247D001F580618B4243D0B6
:10AE8000A1F57A718B4241D001F580618B423DD0B2
:10AE9000A1F57A718B4235D001F580618B4231D0BA
:10AEA000A1F57A718B4233D001F580618B422FD0AE
:10AEB000A1F57A718B422DD001F580618B4229D0AA
:10AEC000A1F57A718B4227D001F580618B4223D0A6
:10AED000A1F57A718B4221D0154D01F580618B422D
:10AEE00018BF002500E0134D104404EB8003CEF39F
:10AEF0008711C3F8AC5093F8A100BDE87040002260
:10AF00004EF0C0BE0C4DEFE70C4DEDE70C4DEBE7FE
:10AF10000C4DE9E70C4DE7E70C4DE5E7044DE3E7A1
:10AF200088010020006002400038024010600240AA
:10AF30000080002820800010008000180088001089
:10AF40000080201020800020008800200080202029
:10AF5000800AA0F58010522808D8054B184490F8B4
:10AF6000F4330D2B02D8034AD056704700207047A7
:10AF700008E70508E45E0608094910B54B6C094C62
:10AF800043F480434B644022002104F68C1053F0BC
:10AF900056FB4FF0FF33C4F8583BC4F85B3B10BD81
:10AFA00000380240E818002058B183884FF0004272
:10AFB000B3FA83F332FA03F303D002490A68134366
:10AFC0000B607047003C01400120FEF729BB00BF29
:10AFD0000220FEF725BB00BF0420FEF721BB00BF07
:10AFE0000820FEF71DBB00BF1020FEF719BB00BFF5
:10AFF0004FF47870FEF714BB4FF47C40FEF710BBA3
:10B0000030B50C4683B0054618B3036803F13F43DF
:10B0100003F57E039B0A104A134493F83C074EF055
:10B020001FFFA988009104F00303C4F381028DF887
:10B03000043028688DF80520C4F300136946C4F372
:10B0400041148DF806308DF807404AF027F803B018
:10B0500030BD4FF0FF33DEE708E7050800B1CFE76A
:10B06000704700BFF8B5CB7813B900252846F8BD66
:10B0700000F110070C460646897838460EF0FCF9B8
:10B0800005460028F1D0E0780EF084FCB06123780A
:10B090000133DBB210B1C371222383710921FFF7A1
:10B0A000DDFFB069FFF790F90D4AD2F8B437632B92
:10B0B000FBD90C480EF0B6F9B082384644F0A4FB38
:10B0C000074630B9E0780EF065FC0EF0C3FC3D4653
:10B0D000CCE7306986F8D87050F0AAFCC6E700BF0C
:10B0E000E818002040420F000B4B10B5D3F8103B7E
:10B0F00003440446987D0EF04DFC60B12E2282710F
:10B10000621CC2710121FFF7A9FF20460021BDE8A2
:10B110001040FFF739B810BDE818002070B50E4C8C
:10B12000D4F8246A002E15DD04F58164002503E0BF
:10B13000B54204F120040DD0237F0135002BF7D058
:10B14000E0680028F4D0217DFFF75AFFB54204F1F2
:10B150002004F1D1012070BD04000010F8B5037D7A
:10B1600085691F2B04464DD90168A3F120024E6862
:10B1700020209040064234D010239340C860CB601A
:10B180004B68D340DE0700F18380EFF31183502238
:10B1900082F312882A6C1168C9075AD4516889B29F
:10B1A00071B9D5E90960864250D0AF690744D760CC
:10B1B00073D9301A80B25060AE62002185F86410F5
:10B1C000116841F00101DBB2116083F3118895F839
:10B1D0006430002B44D1237D1F2B27D92168A3F194
:10B1E00020024C6808209040044200D0C8604C689F
:10B1F000042000FA02F2224203D0203B00FA03F3BB
:10B20000CB60F8BD026820201668984006421946B7
:10B210000ED010219940906091601168D940C80704
:10B22000B3D5012101FA03F39360AEE72268194612
:10B23000106808238B40184200D0936010680423E4
:10B2400003FA01F10142DCD09160F8BD012285F8DA
:10B250006420DBB283F3118895F86430002BBAD0F8
:10B2600095F87C30002BB6D195F871000EF092FB6A
:10B270002A6E938923F008031B0401211B0C938180
:10B2800085F87C100028A6D02021FFF7B9FEA2E7A0
:10B29000012303FA02F2CA6077E72E69301A80B2FE
:10B2A0005060A96289E700BF70B503792D4C002B6F
:10B2B00014BF012200228AB084F80C2803D184F83C
:10B2C000E0370AB070BD054604F6140690F9001088
:10B2D00030460EF0D1F8AD78002D37D1224B2348FF
:10B2E000C4F8A838012284F82028C4F81C580EF0AD
:10B2F00099F803464FF47A70A4F8183811F0ACFCB2
:10B30000D4F81C3813B11A689B881383184D0FCDDD
:10B31000EC46ACE80F000FCDACE80F0095E8030059
:10B320008CE80300694630460DF00AFFD4F8142873
:10B33000136A002BFCD1D4F8B417C4F8D01701223B
:10B3400084F8E02784F8D4370AB070BD28460EF0A0
:10B3500021FB05460028C1D01E23C3800921FFF729
:10B360004FFEBBE7E8180020A4200020801A06004A
:10B370004CEE050870B50C4682B01546064600280E
:10B3800039D0036803F13F4303F57E039B0A1B4A50
:10B39000134493F83C074EF063FDB2880092B2FA72
:10B3A00082F304F003028DF80420C4F381023068B4
:10B3B0008DF80520C3F11F03C4F30012C4F3411438
:10B3C0008DF80740C3F3CC0400EB840403F00703BB
:10B3D0008DF806209B00226A0F269D4006FA03F393
:10B3E00022EA03032362226A15436946256249F073
:10B3F00055FE02B070BD4FF0FF33C8E708E70508FF
:10B4000000B1B7E7704700BF2DE9F043774D05EB7A
:10B41000001683B0D6F8603B002B00F09380044602
:10B420004FEA001896F8680B4EF01AFD96F8683B44
:10B43000590903F01F0203294FF0010303FA02F335
:10B4400000F09880042900F0858002297DD005EB6A
:10B450000803013493F8640B0EF09CFAE4B28146C1
:10B4600010B112238371C47105EB080393F8650BC7
:10B470000EF090FA074610B11323C471837105EBE7
:10B48000080393F8660B0EF085FA064610B11423F4
:10B49000C47183714544484695F8672B01924A214F
:10B4A000FFF7AEFF019A38462A21FFF7A9FF019A5C
:10B4B0000A213046FFF7A4FFD5F8602B4C4B9A4287
:10B4C0005DD04C4B9A424AD04B4B9A4262D04B4B88
:10B4D0009A426AD04A4B9A4272D04A4B9A427AD0E8
:10B4E00049499088B1F8CE42B1F8CC32B1F8D65281
:10B4F0002343B1F8D0422343B1F8D24220F00300F5
:10B500002343B1F8D4420004000C2343B1F8D842DD
:10B5100090802B4310882343B1F8DA42B1F8DC1253
:10B5200000F44150234303439BB21380938B23F4D5
:10B5300000631B041B0C9383118213889BB243F09E
:10B540004003138003B0BDE8F083304A516A0B43D7
:10B5500053627CE72D4A11690B43136177E703F5CA
:10B560000033196A41F480411962196A21F480415B
:10B570001962B5E7254A116A0B43136267E703F5C1
:10B580008433596A41F480515962596A21F48051D7
:10B590005962A5E703F5FE33196A41F400411962C7
:10B5A000196A21F4004119629AE703F58233596A56
:10B5B00041F400515962596A21F4005159628FE7F0
:10B5C00003F56843596A41F480115962596A21F4BC
:10B5D0008011596284E703F56443596A41F400110C
:10B5E0005962596A21F40011596279E7E81800207C
:10B5F0000030014000380040003C00400034014071
:10B6000000500140005401408801002000380240F1
:10B61000431C00F0A8802DE9F04F00EB8003C44FDD
:10B62000DA0087B057F8029081000546019107EBD8
:10B63000C303B9F1000F04D09C68002C4BD0A17952
:10B6400011B107B0BDE8F08FD3F80CA0BAF1000F2C
:10B6500000F095819AF80630002BF2D11832B81814
:10B66000D9F80480BB50691CC0E90133C3601523BD
:10B67000A371C9B21623E1718AF807108AF806305F
:10B6800099F818004EF0ECFBB8F804302268A18855
:10B6900023F440731B041B0CA8F80430DAF80030C4
:10B6A0001183BAF804201A8311212046FFF7A8FC61
:10B6B00011215046FFF7A4FC09264FF0330B24B1AB
:10B6C0002268A1881069014231D1BBF1010B45D03C
:10B6D0004FF044FBF3E7D3F80CA0BAF1000F00F0F1
:10B6E000A4819AF80630002BABD11832BB18D9F8D8
:10B6F0000480BC50C3E90144DC6016238AF806309C
:10B700006B1C8AF8073099F818004EF0A9FBB8F8BE
:10B710000430BAF8042023F440731B041B0CA8F86F
:10B720000430DAF800301A83C2E7A1882268518316
:10B730004FF070FB2368A2881A834FF06BFB013E29
:10B74000BBD1332624B12368A28819690A420DD1DE
:10B75000013E00F0FB804FF001FBF3E7002CE4D149
:10B760004FF058FBE9E77047A28823685A834FF0EF
:10B7700051FBBAF1000F00F02481DAF80030BAF87A
:10B7800004205A834FF046FB002C00F0EE80236823
:10B79000A2881A834FF03EFBDAF80030BAF8042092
:10B7A0001A834FF037FB2368A2881B691A4240F0C6
:10B7B000A080019B2B4407EBC3039A7C002A40F036
:10B7C00095801A7C12212046FFF7D4FD019B2B4463
:10B7D00007EBC3039B7C002B00F08F803221BAF172
:10B7E000000F07D0019B2B4407EBC30350465A7C44
:10B7F000FFF7C0FD4F4B984500F0EF804E4B98454A
:10B8000000F0F6804D4B984500F0FD80019B2B44E5
:10B8100007EBC3074FF47A73BC8A03FB04F4B8F850
:10B82000043023F440731B041B0CA8F80430B8F850
:10B8300000309BB243F00103A8F80030B8F8045080
:10B8400002A849F075FC25F03F0504993C4B2D04F6
:10B85000A3FB01232D0C45EA9345A8F80450B8F842
:10B86000002022F001021204120CA8F80020354A30
:10B87000980C9442034642DC6200B1FBF2F292B2B1
:10B880000133042A38BF0422A8F82030A8F81C206D
:10B89000B8F800309BB243F00103A8F80030B8F8C4
:10B8A000003023F4816323F002031B041B0C4FF4CC
:10B8B000804143F48063A8F80030A8F80810B8F875
:10B8C000003023F080031B041B0C0022A8F800307A
:10B8D00099F81A0011464EF0D5F9002299F819008E
:10B8E000114607B0BDE8F04F4EF0CCB91A7C3221BA
:10B8F00069E7DAF800301B695BE712216FE704EBB8
:10B900004404B1FBF4F18AB2C1F30B0109B942F06E
:10B9100001020D494FF4967300FB03F3A1FB0313DF
:10B920009B09013342F40042A8F82030AEE700BF83
:10B93000E81800200054004000580040005C00401F
:10B9400083DE1B43A0860100D34D6210002C7FF4E0
:10B950000BAF4FF05FFABAF1000F5FD0DAF80030AA
:10B96000BAF804205A834FF055FA4FF053FADAF838
:10B970000030BAF804201A834FF04CFA26E7183248
:10B98000BB18D9F8048047F802A0C3E901AAC3F89C
:10B990000CA01523A371431CE37199F818004EF015
:10B9A0005FFAB8F80430A28823F440731B041B0C20
:10B9B000A8F80430236811211A832046FFF720FBE2
:10B9C0007AE64FF027FA2368A2881A834FF022FA0A
:10B9D0004FF020FA23681B69EBE603F5F2331A6A8D
:10B9E00042F400121A621A6A22F400121A620DE777
:10B9F00003F5F0331A6A42F480021A621A6A22F4DA
:10BA000080021A6202E703F5EE331A6A42F400027A
:10BA10001A621A6A22F400021A62F7E64FF0FAF983
:10BA20004FF0F8F94FF0F6F9D0E61832BB18D9F814
:10BA3000048047F802A0C3E901AAC3F80CA099F852
:10BA400018004EF00DFAB8F8043023F440731B04CC
:10BA50001B0CA8F804302FE62DE9F84307460EF03A
:10BA600067FEDFF84C8007EB8709044608EBC90541
:10BA700042F20F7604E00EF05BFE031BB3420ADCD9
:10BA80006B7E002BF7D108EBC90898F8180080F0FE
:10BA90000100BDE8F883B8F8903B013338469BB20B
:10BAA000A8F8903BFFF7B4FD0020BDE8F88300BF85
:10BAB000E818002070B500EB8003274D05EBC302AA
:10BAC00055F833305C68A38A84B09BB20393039B20
:10BAD00013F4706F1CBF01231376039B13F4E06F04
:10BAE0004FEA80060CD1A38A304423F4706305EB3F
:10BAF000C0051B041B0C0022A3826A7604B070BD33
:10BB0000238BA38823F480631B041B0CA380039B5B
:10BB10009A05E8D423889B05E5D42388D9050FD559
:10BB20002388DA05FCD423889BB243F40073238076
:10BB300023889B05FCD40190FFF76AFD0198D2E7AA
:10BB400023889BB243F400732380A38823F44073BB
:10BB50001B041B0CA380C6E7E81800200020A9E7FF
:10BB60000120A7E70220A5E72DE9F84F2F4F00EBB2
:10BB7000800407EBC404D4F80480B8F1000F04D0AB
:10BB80009A46637E03F0FF0923B14FF0000948464F
:10BB9000BDE8F88F0E46934605460EF0C9FD0A9B98
:10BBA0007600F6B2C4E908330123A67684F81BB008
:10BBB00084F81D90A37784F81CA0637684F818900D
:10BBC000B8F804209105064622D4B8F80030DA050A
:10BBD00012D442F20F7404E00EF0AAFD831BA342BC
:10BBE0001ADCB8F800309B05F6D4B8F800309BB2E8
:10BBF00043F48073A8F80030B8F804309BB24FF0DB
:10BC0000010943F44073A8F804304846BDE8F88FB2
:10BC100099464846BDE8F88FB7F8903B01339BB290
:10BC20002846A7F8903BFFF7F3FCB0E7E8180020A0
:10BC3000F8B590F871301C09013C052C0FD81B4E4B
:10BC400006EB44020546B2F86C0703F00F0340FA16
:10BC500003F2D20703D595F87C70012F01D00120A3
:10BC6000F8BD07FA03F3013B1840344450F020FFBD
:10BC700094F878270E4C104454F8302004EBC0049C
:10BC80001069A3881840EBD0EB6E002285F87C2069
:10BC900093F8212020460221FFF76CFB2A6E93893E
:10BCA0009BB243F0080338469381F8BD08E70508C6
:10BCB0007C240020094BD3F8942ED3F8981E40F230
:10BCC0002A40002350604B620B889BB243F0010373
:10BCD0000B80136843F0010313607047E8180020DD
:10BCE0001D4B1E48196C1E4A10B441F080510124AE
:10BCF000196404625321FF24CA20546250625162C5
:10BD00005B6FDB0085B017D4164804230021029135
:10BD10000290029A1A440292029A04331C2B116078
:10BD2000F5D103910390039B0393039B0E4A1A6082
:10BD300005B05DF8044B70470A4B00220192019355
:10BD4000019B0193019A084B12689A42DCD105B01D
:10BD50005DF8044B704700BF0038024000000E42FF
:10BD600000280040502800403166654210B5174C4D
:10BD700084B00139002389B2A042ADF80C30ADF88F
:10BD800006308DF80E30029113D0114B984210D02E
:10BD900003F5804398420CD003F58063984208D0A5
:10BDA00003F58063984204D00A4BD3F8AC375B08A4
:10BDB00002E0084BD3F8AC37B3FBF2F201A9013A29
:10BDC000ADF8042049F050FB04B010BD0004014060
:10BDD00000000140E818002030B50446006EA2685B
:10BDE000838923F400531B041B0C8381637995B072
:10BDF00013F0040F4FF00001019214BF4FF4805272
:10BE00000A46ADF808201A031B0203F48063ADF85C
:10BE10000C302379ADF80E1002F40052ADF80A2070
:10BE2000DA0744BF0422ADF80E209B07ADF81010CE
:10BE300005D5BDF80E3043F00803ADF80E3001A96A
:10BE400049F024FC6279236ED50700F18B8012F053
:10BE5000080F9A8A48D092B242F008029A829A89D0
:10BE600092B242F400529A812279D00732D5E06B27
:10BE7000002800F089800023E26D0893CDE90C339F
:10BE8000CDE91033CDE912334FF480750A9363691D
:10BE9000E1680E9506920793626C05924FF48063F9
:10BEA0004FF480350B9309910F9549F0A5F905A939
:10BEB000E06B49F037FAE26B216E136843F001033F
:10BEC00013608B8A9BB243F040038B8253682279C4
:10BED0009BB2636591070DD4226E93899BB243F4A4
:10BEE0000053938115B030BD22F008021204120CE9
:10BEF0009A82B4E7206C002852D02369A26D09937E
:10BF0000A36CCDE90532402300254FF4803108931E
:10BF10004FF480630B930F91CDE90C55CDE910558B
:10BF2000CDE9125507950A950E9549F065F9206CF3
:10BF300005A949F0F7F9236C226E586940F080009A
:10BF40005861186840F0160018605D60938A9BB2D3
:10BF500043F0800302F10C0193820B6843F040032D
:10BF60000B60BAE71E498B4224D0A1F54C418B42AD
:10BF70001ED001F580618B421ED102200121FEF707
:10BF800003F96279236E62E74FF6DF711980D96891
:10BF900041F02001D960D96841F01001D96099E7DA
:10BFA000226ED36843F0800302F10C01D360D4E722
:10BFB0000120E3E70020E1E701F580618B420AD030
:10BFC00001F580618B4208D001F544418B427FF43A
:10BFD0003EAF0520D2E70320D0E70420CEE700BF24
:10BFE000001001402DE9F84F4D4C04EB8004D4F8CB
:10BFF0002C4A002C7DD0E56E002D76D01F46EB6AD2
:10C000006361AB6AA3616B8EE3602B8E23616B6807
:10C010002366444B2360444BA160A366064620463A
:10C0200090460DF04BFE94F871000DF0B3FC814684
:10C0300095F8200094F870B0A24600284ED1022353
:10C04000390784F87C3036D418F0020F10D0B9F1DB
:10C05000000F0DD00B2389F80630731C89F80730C8
:10C060003B0648D495F8212048462221FFF782F963
:10C0700018F0010F04D1E26B9AB15046BDE8F88F79
:10C0800058460DF087FC0028F5D00C220136C67109
:10C09000827195F821202221FFF76CF9E26B002ACA
:10C0A000EBD195F8241095F8220089094DF0EAFDAE
:10C0B0005046BDE8F88F0136F6B2B9F1000FDAD07C
:10C0C0000B237A0689F8076089F8063009D595F8B8
:10C0D000212042214846FFF74DF9CCE74DF0C0FE44
:10C0E000ADE795F821201221F4E7AA465046BDE8B5
:10C0F000F88FA246C1E794F871000DF04BFC226E58
:10C10000938923F008031B0401211B0C938184F8FD
:10C110007C100028ACD02021FEF772FFA8E700BFFA
:10C120000400001088EE050831BC0008BFF34F8FF3
:10C130000549064BCA6802F4E0621343CB60BFF3C3
:10C140004F8F00BFFDE700BF00ED00E00400FA05DF
:10C1500008B572B6FFF7EAFF00B583B00D490022BB
:10C1600000920091009B0C330093009B1B68012BF5
:10C1700002D003B05DF804FB01920191019B0649D6
:10C180000C330193019B1A600B6883F308884B689A
:10C190009847FEE7502800400000FF1F38B5FFF722
:10C1A0009FFDFFF7D9FF012049F04EF9704A9368CF
:10C1B00023F003039360936813F00C0FFBD1136813
:10C1C0006B49002840D143F00103136041F28833EA
:10C1D0000A6895075BD4013BFAD1664C664D644B07
:10C1E000664AEA60664A596FAA60596B654821F051
:10C1F00080015963596F41F080715967196B41F49F
:10C20000CE0119635A6B5A639A6B9A631A6C024394
:10C210001A64596C5C4A0A435A640EF041FAD4F825
:10C22000AC375A4AA2FB03239B09013BB3F1807F41
:10C2300009D24FF0E022F02053610021072385F856
:10C2400023009161136138BD43F4803313600A68A1
:10C25000940341F2883304D4013BBED00A689403AE
:10C26000FAD5444C4A4A4B4BB0FBF3F3B0FBF2F027
:10C27000B3EB400F18BF18464FF48002B3FBF0F346
:10C28000C4F8B02EC4F89C0EC4F8A03E09E0394CA6
:10C29000002108220223C4F8B01EC4F89C2EC4F862
:10C2A000A03E022049F0D0F803280FD83A4BD4F82A
:10C2B000A01E03EBC0008588C2884388C4F8A85E2E
:10C2C000B3FBF1F3C4F8AC2EC4F8A43E284B3349B9
:10C2D0001A6C42F080521A640A6842F440420A60C2
:10C2E0009A689A609A6842F400429A609A6842F4A6
:10C2F000A0529A60D4F8B00ED4F89C2ED4F8A41EA4
:10C30000024342EA8112D4F8A81ED4F8AC0E4908C0
:10C3100042EA0062013942EA01425A601A6842F078
:10C3200080721A601A689201FCD51D4A40F20571AC
:10C330001160996821F003019960996841F0020148
:10C34000A2F580629960936803F00C03082BFAD180
:10C35000D4F8A00E1349D823B3FBF0F39B0143F0AC
:10C3600000530120C2F884308866FCF719FB35E7DA
:10C3700000380240E818002000ED00E00005FA0552
:10C3800000000020FFC9FE36335F0700D34D621066
:10C3900080841E0040420F00B8EE05080070004087
:10C3A000003C02400000474210B584B00023044620
:10C3B000ADF80C300068ADF806308DF80E3003F1A2
:10C3C0008043013903F5823389B29842029114D037
:10C3D000A3F58063984210D003F5804398420CD0B7
:10C3E00003F58063984208D003F58063984204D037
:10C3F000204BD3F8AC375B0802E01E4BD3F8AC37C8
:10C40000B3FBF2F301A9013BADF8043049F02CF87D
:10C410002168194A0B8819489BB243F001030B802D
:10C42000002301E050F83320914208D001330E2B55
:10C43000F8D1002004B0BDE81040FCF725BA104A3E
:10C4400002EBC30393F8D5472046FCF71DFA1B2CDB
:10C4500005D1192004B0BDE81040FCF715BA2E2C08
:10C4600008BF2C2004D104B0BDE81040FCF70CBA82
:10C4700004B010BDE818002000000140D8EE050807
:10C4800008E7050870B50468A30AA3F58013522BCA
:10C4900051D83C4D2B4493F8F4530D2D4BD8407993
:10C4A0008608002954D005EB850305EB4303B4F857
:10C4B0000CE04FEA900C33440220334E00FA0CF0AB
:10C4C00040EA0E0006EB830C80B2CCF84815CCF89D
:10C4D0005825A081EFF3118C502383F312882C236D
:10C4E00005FB03F3F118D1F8442562B3274BC1F8DB
:10C4F0006825043226482C2105FB01F1084414313B
:10C500000B4453F8041B19B1116053F8042C043286
:10C510009842F6D100235FFA8CFC13608CF31188EB
:10C520002C2303FB0565D5F868352BB1A3899BB295
:10C5300043F00103A38170BDA38923F001031B0411
:10C540001B0CA38170BD03F12402104B1A44D1E7E8
:10C55000B4F80CC005EB8503304605EB43034FF000
:10C56000020E33441FFA8CFC074E0EFA00F02CEA40
:10C570000000A08106EB8300C0F84815C0F85825DC
:10C58000A8E700BF08E70508E81800202C1E0020D7
:10C59000501E002001490248FDF760B82C1E002003
:10C5A0000000014010B5064C064804F24451FDF766
:10C5B00055F804F5DA610448BDE81040FDF74EB8BF
:10C5C000E8180020000001400044014002494FF0FB
:10C5D0008040FDF743B800BF581E002001490248C3
:10C5E000FDF73CB8841E00200004004001490248C9
:10C5F000FDF734B8B01E0020000800400149024891
:10C60000FDF72CB8DC1E0020000C00400149024858
:10C61000FDF724B8601F00200004014010B5064C4F
:10C62000064804F5CF61FDF719F804F25471044887
:10C63000BDE81040FDF712B8E818002000040140E2
:10C64000001C004001490248FDF708B88C1F00207B
:10C650000040014001490248FDF700B8E41F0020F6
:10C660000048014001490248FCF7F8BF10200020B3
:10C670000018004001490248FCF7F0BF6820002084
:10C6800000200040F8B5164D1648174F00214FF412
:10C690001A7251F0D4FF05F688064FF08041A5F1DB
:10C6A0008C043A46002301E054F8332091420BD029
:10C6B00001330E2BF8D100201C354DF0D1FBB542D3
:10C6C0000CD055F81C1CECE7084A02EBC3031C35E0
:10C6D00093F8D4074DF0C4FBB542F2D1F8BD00BFCA
:10C6E00064EF05082C1E00200000014008E7050843
:10C6F00010B50C2937D8DFE801F0973636366636A4
:10C700003636373636360700038C5488B2F80CE0DC
:10C7100023F480531B041B0C0384038CB0F804C067
:10C72000818B21F4E6414EEA040E0904148823F4B7
:10C730000053090C41EA04211B04754C1B0C43EA0D
:10C740000E33A0421FFA8CFC9BB289B200F0AE807F
:10C7500004F58064A04200F0A9809268A0F804C0AB
:10C7600081830264038410BD038CB2F80CC054882A
:10C7700023F480731B041B0C0384038CB0F804E0C7
:10C78000818B23F400731B044CEA040C21F0730129
:10C790001B0C43EA0C230904B2F800C0090C41EA5F
:10C7A0000C0C5B4988421FFA8EFE9BB268D001F5E3
:10C7B0008061884264D09268A0F804E0A0F81CC0B0
:10C7C000C263038410BD038CB2F80CC0548823F0FC
:10C7D00010031B041B0C0384038CB0F804E0018BD2
:10C7E00023F020031B044CEA040C21F4E6411B0C4B
:10C7F00043EA0C130904B2F800C0090C41EA0C2109
:10C800001FFA81FC424988421FFA8EFE9BB269D012
:10C8100001F58061884265D09268A0F804E0A0F834
:10C8200018C08263038410BD038C5488B2F80CE0F6
:10C8300023F001031B041B0C0384038CB0F804C019
:10C84000018B21F073014EEA040E0904148823F0D1
:10C850000203090C1B0421432D4C1B0C43EA0E035D
:10C86000A0421FFA8CFC9BB228D004F58064A04241
:10C8700024D09268A0F804C001834263038410BDF1
:10C88000D189548A23F4006343EA0121138A2EF4E8
:10C89000405E23434EEA031E94884FF6FF330B405D
:10C8A00043EA04231FFA8EFE9BB284E7148A2CF419
:10C8B000804C4CEA841C1FFA8CFC4EE7D489B2F8F9
:10C8C00010E023F008032343548A2CF4407C4EEA02
:10C8D000040E948823F004034CEA0E0C1FFA8CFC1F
:10C8E0002343C6E7D189548A23F0800343EA011128
:10C8F000138A2EF4406E23434EEA830E94884FF63B
:10C90000BF730B4043EA04131FFA8EFE9BB283E70A
:10C91000000001402DE9F04FA24BDFF8A49293F8FC
:10C92000C63EA14EA14F8FB0CDE90139013BDBB22C
:10C9300000930025DFF88CB2DFF88CA25B46D3466B
:10C940009A464FEA9A23A3F58013522B4CD83344CE
:10C9500093F8F4330D2B47D8FC56019B012B40F084
:10C960000181012C35D14FF000084146204611F0DD
:10C970001DFA11F0A9FA037813B1542B40F0F98095
:10C9800008F104081FFA88F8B8F1100FEDD14FF044
:10C99000000E8DB3494600200CE0334493F8F43385
:10C9A0000D2B0ED8FB56A3420ED00130A84201F544
:10C9B00080711EDA8A6813689B0AA3F58013522BD4
:10C9C000EBD90023A342F0D153799BF805209A427A
:10C9D000EBD1774B5B454BD05BF81CAF4FEA9A230A
:10C9E000A3F58013522BB2D9009B012BF1D900245F
:10C9F000B9E7BEF1000FECD15846FBF7C3FCC3B258
:10CA0000022B9BF805C000F23483431C5BB203EB9E
:10CA100043034FEA830E644B664903F5727004E0EA
:10CA2000984200F0268353F82C1F5145F8D11A790B
:10CA30006245F5D153F80E40002CF1D05E4800233A
:10CA40004268A24203F1010300F08980102B00F13B
:10CA50002400F5D14FF0FF33584A03EBC30302EB38
:10CA6000830393F8A830002BB3D1029BC3F808B01E
:10CA7000029B013503F58073042D02937FF45AAFB6
:10CA8000DFF848B10BF59E730027ABF5816A984635
:10CA9000DAF8243ABB425FDDDBF80C50002D5BD0A6
:10CAA0009BF81030A88802932B68DAF80460019391
:10CAB00003F13F41B0FA80F301F57E010393002EAC
:10CAC000C3F11F034FEA9121009340F384800023B8
:10CAD00002E00133B3427BD01C0259F804208A42A1
:10CAE000F7D14C440099029B8BF810300326013794
:10CAF000CBF80410CBF80C50CBF81840AE71EF71A6
:10CB0000636CE26C0D4649008E401E43012303FA1C
:10CB100001F111439AF800206664E1647AB303FAE4
:10CB200005F11A46236D0B432365019B89B21883D7
:10CB3000D4F8A000FBF762FC2046FBF7B5FD01230B
:10CB4000082F8BF81C308BF81D3088F811300BF152
:10CB5000200B08F118089BD10FB0BDE8F08FDBB2B5
:10CB6000013B79E7022B7FF4FEAE082C3FF4FBAECD
:10CB70002FE74FF0010E002D7FF40CAF29E703994A
:10CB8000C1F12F05009903FA05F58B4099B2236D89
:10CB90002B432365019B5883D4F8A000FBF72EFCA0
:10CBA000CAE700BFE818002008E70508E45E0608A9
:10CBB000B0F80508000001401402002088010020A0
:10CBC0000C00001000040140D0F705080C04001010
:10CBD000032B00F31F820AEB06233202186904922A
:10CBE000002800F03F8299600131CAB283F8052124
:10CBF0000692542283F80421013602680592447992
:10CC0000CAF80460FBF7BEFB934AC3B2022B92F84A
:10CC1000DDEE844600F22D82461C76B206EB460617
:10CC20008E498F48059AB600002305E00133172B83
:10CC300000F01F8251F82C0F8242F7D10879A042F0
:10CC4000F4D188590028F1D02C2101FB03F30CEB1F
:10CC50004C0C03EB8C0C814B63441969049B5344CB
:10CC6000C3E906017F4B00211E461C4663689842BB
:10CC700016D00131102904F12404F7D17A4B93F82E
:10CC80008420002A00F0E7817849794A794BCAF874
:10CC9000681ACAF8602ACAF8703A0FB0BDE8F08F77
:10CCA00001F1010C5FFA8CFC6F4B07960CF1FF3C15
:10CCB0000CEBCC0C03EB8C0C9CF8A8300593002BF0
:10CCC000E2D1049E069B8CF8A930F31103EB2620D9
:10CCD00000EB001368488C2400EB83003112674B93
:10CCE00004FB01F103EB41010AEB0603C3E93C1429
:10CCF0005421019E8CF8A8103321C3F8AC10DE60DB
:10CD0000C3F8A8005E4B04999A4209EB010400F0B5
:10CD10007681534B9A4200F0728103F580439A4228
:10CD200000F06D8103F580639A4200F0688103F59D
:10CD300080639A4200F06381474BD3F8AC07BEF1A1
:10CD4000060F4FEA500000F061814E4B4E49BEF194
:10CD5000070F18BF9C464D4B08BF8C464C4918BF67
:10CD60001946B0FBF1F1B0FBFCFC1046049A013906
:10CD70000AEB020389B20CF1FF3CA3F8B0C0A3F8A0
:10CD800068104FF000060193A165002302F15401E1
:10CD90004944A4F85C60636548F066FB019B3D4A2A
:10CDA0001B690193186803889BB243F080030380DA
:10CDB000038809920A210B914FF48072022123F01B
:10CDC0000103CDE90C121B04ADF828601B0C019E79
:10CDD0000380717909AAFFF78BFC3079002840F0B5
:10CDE0002281049B079E0AEB030200231069D2F8FC
:10CDF00018C001680A8892B242F001020A80726883
:10CE0000944503F1010300F00A81102B06F124067A
:10CE1000F5D14FF0FF33144A1F4E03EBC30302EB6F
:10CE200083031E4AD3F88C30B3420CBF4FF4001377
:10CE30004FF48003166B33431363427918480C2A6E
:10CE40009BBF184B03EB42030026B3F8CC60049B56
:10CE500053449E8200232EE0E818002008E70508CE
:10CE6000000001401402002088010020B57601086E
:10CE7000B1760108BD760108C8270020F82A0020F5
:10CE8000000401404495080010552200D0DD060042
:10CE900040771B0060000100006002400038024043
:10CEA0001406001000F80508914200F0E0800133FC
:10CEB000042B00F0E18050F83320002AF4D1DAF896
:10CEC0000C260132CAF80C260AEBC302DB00C2F8BA
:10CED000101603446A499A88059816439E80049B5D
:10CEE0000AEB030690222346FDF79EFFB069026815
:10CEF000002342F010020260C4E92533A367C4F89E
:10CF00008830C4F89C30F26962664FF48062E26750
:10CF100004214FF40032C4E9232140222267D6F8CD
:10CF2000AC206267F268049B1832A2664FF480520C
:10CF3000C4F88020D6F8A820E26603F164014FF41B
:10CF400080424944C4F8842048F0ECF9B069049B5D
:10CF5000D0F800E0C4F81CE0D0F814E0C4F820E0F9
:10CF6000D0F804E0C4F824E003F1AC01D0F808E004
:10CF7000C4F828E00023D0F80CE0C4F82CE0C4E9A1
:10CF80003733C4F8B830C4F8C030C4F8D030C4F86F
:10CF9000E430F369C4F8AC304FF48063C4F8C430B3
:10CFA0004FF4403C0423C4E935C3D6F8F430C4F848
:10CFB000BC30F3681033C4F8B0304FF40063C4F8E9
:10CFC000C830D6F8F030C4F8B4304FF48042C4F81A
:10CFD000CC20494448F0A6F9B369A8881A682263AE
:10CFE0005A6962635A68A2639A68E263DA682264E3
:10CFF0001A6842F010021A602B68019372E5214B07
:10D00000BEF1060FD3F8AC077FF49FAEDFF87CC00B
:10D010001D49A6E61B4A032382F8DC3E34E6DBB258
:10D020000593013BF7E60CF0B5FC069038B1019B87
:10D030000221DA79FEF79EF9069B5422DA80019BE1
:10D040001A68B2F844306FEA43436FEA53439BB225
:10D05000A2F84430C5E6542283F88420069A83F867
:10D06000852011E6074A022382F8DC3E0CE6DB004D
:10D070002FE700235B68FFDE00239B88FFDE00BFF5
:10D0800045840008E8180020A0BB0D00882A110084
:10D090000C2911D8DFE801F023101010191010101E
:10D0A000111010100700838B23F400631B041B0C6A
:10D0B00043EA022292B282837047838B23F00803F3
:10D0C0001B041B0C1A4382837047038B23F40063F9
:10D0D0001B041B0C43EA022292B202837047038BAB
:10D0E00023F008031B041B0C1A430283704700BF84
:10D0F0002DE9F04FDFF870B29BF8004087B024B9FB
:10D100000124204607B0BDE8F08F934ED6F8B457FF
:10D110000DF03AFB9BF8B43A0390002B00F05882D4
:10D120008E4AA2FB05328E4B5209A3FB0213DB0889
:10D1300003EB8303A2EB4303DAB204920BF23C62EB
:10D1400002EB830300930BF61C1306F1DC0401933E
:10D150004FF00009924635E03B680293009B5C3338
:10D160000093019B30461433019348F045F87A4B05
:10D1700002988C2202FB0933002583F8D05079797C
:10D180002A46FFF785FF22467979FFF7B1FA7979C8
:10D190000822FFF77DFF402344F83C3CA4F14801FE
:10D1A000304648F0BFF8336843F0100333609BF813
:10D1B000B43A09F1010999450AF15C0A04F18C04B9
:10D1C00080F2D480DBF83836039AD31A04D454F8AA
:10D1D000082C9342C0F2AB815F4B54F8587C266A0E
:10D1E0008C2202FB093393F8D030002BB4D039687D
:10D1F000736834F8542C02911FFA83FE8B89CEF1A8
:10D20000160E9BB223EA0203BEF1070F8B81A5D94C
:10D21000DBF824390133CBF82439A36A05939C4603
:10D2200000225CF8045B012190461BE0DCF8000062
:10D23000B8F1140FA0EB05031DDC13F1080548BF7E
:10D2400003F117052B1108EB25180546581E01316F
:10D2500002FA03F3012282408E4542EA03020CF1F6
:10D26000040C08D38E45E1D8C8F11503DCF8005052
:10D270004FF01508EAE7B8F1150F60D13948C2F34D
:10D280008423C2F3441100EB830300EB8101D3F844
:10D29000E830D1F8E8101B0243EA011302F01F0145
:10D2A00000EB8101C2F3C43200EB8202D1F8E81036
:10D2B000D2F8E8200B4343EA023383EA132282EADE
:10D2C000121202F00F020F2A39D1C3F30F134FF6D7
:10D2D000FF72934233D0B3F5606F00F03681019A4C
:10D2E00093819AF85820049DAA4211D00098DAF848
:10D2F00000208168521ACAF80020016BDAF8042075
:10D30000521ACAF804200022826002638AF8585038
:10D31000DAF8002000990132CAF800208A68013248
:10D320008A604FF6FF7293427FF418AFDAF8043048
:10D330000133CAF804300B6B01330B630EE7DBF8E3
:10D3400020390133CBF82039B9F1000F00F0E58026
:10D350004FF6FF73C5E700BFE81800201F85EB51AB
:10D36000CDCCCCCC00F805080400001001228BF8CD
:10D37000202ACBF83856002B3FF4C2AE974890F8DD
:10D380008C10890700F1BE80D0F8841008684979B4
:10D390008A40018C92B289B221EA02010184018C97
:10D3A00089B20A43012B02843FF4AAAE8B4991F85B
:10D3B0001821970700F1C080D1F810211068547926
:10D3C000018C012289B2A24092B221EA02010184B9
:10D3D000018C89B20A43022B02843FF491AE7F494B
:10D3E00091F8A421960700F1C180D1F89C21106822
:10D3F0005479018C012289B2A24092B221EA020141
:10D400000184018C89B20A43032B02843FF478AE75
:10D41000724991F83022950700F1B180D1F82822A5
:10D4200010685479018C012289B2A24092B221EA9B
:10D4300002010184018C89B20A43042B02843FF467
:10D440005FAE664991F8BC22940700F1A180D1F843
:10D45000B42210685479018C012289B2A24092B2A0
:10D4600021EA02010184018C89B20A43052B02845E
:10D470003FF446AE594991F84823900700F1918056
:10D48000D1F8402310685479018C012289B2A2405E
:10D4900092B221EA02010184018C89B20A43062B6F
:10D4A00002843FF42DAE4D4991F8D423920700F148
:10D4B0008180D1F8CC2310685479018C012289B283
:10D4C000A24092B221EA02010184018C89B20A438E
:10D4D000082B02847FF414AE404A92F860349B0714
:10D4E00071D5D2F858240423116850790A8C8340EE
:10D4F0009BB292B222EA03020A840A8C92B21343CC
:10D500000B84FDE5354AD2F8842010685479018CEB
:10D510000422A24089B292B23EE7059930485822CF
:10D5200051F02AF83B6802934FF6FF73D9E60024C6
:10D53000204607B0BDE8F08F284AD2F810211068C5
:10D540005479018C042289B23DE7244991F8DD2405
:10D5500002EB420201EBC2024A4492F8ED240D2A8A
:10D560007FF4BDAE019980228A77BAE61B4AD2F8D1
:10D570009C2110685479018C042289B23CE7174A37
:10D58000D2F8282210685479018C042289B24CE721
:10D59000124AD2F8B42210685479018C042289B25C
:10D5A0005CE70E4AD2F8402310685479018C0422BB
:10D5B00089B26CE7094AD2F8CC2310685479018CFF
:10D5C000042289B27CE7054BD3F8582401238BE76A
:10D5D00001228BF8202ACBF8383692E5E818002093
:10D5E000CC0900102DE9F04F002299B02F210746F9
:10D5F00010F0C0FC00B3BE4ED0F80080C6F8988E84
:10D600000446FDF715FB0246B0B1D0F804C0C6F8D9
:10D6100094CEBCF1000F0FD0B64D002329464868C8
:10D62000844501F1240103F101030FD0102BF6D141
:10D63000B14B93F8840018B1002019B0BDE8F08F09
:10D640002F2283F8842083F88500F6E7DBB2DFF829
:10D65000A892013B03EBC30309EB830393F8A8A053
:10D66000BAF1000FE8D138469768DFF8C0B22F2230
:10D67000A3F8A8200CF08EF92F220346CBF87C05E6
:10D6800020B1DA80E2792A21FDF774FE9B4A9C4999
:10D69000002301E051F83320904500F0228101334E
:10D6A0000E2BF7D100204CF0DBFBD6F8980E954AF4
:10D6B000038823F001031B041B0C9042038000F03D
:10D6C00070818E4B984216D003F58043984212D059
:10D6D00003F5806398420ED003F580639842D6F834
:10D6E000AC270AD08849B1EB520F4FEA520340F2FF
:10D6F000528100210AE0D6F8AC27834B9A4280F091
:10D7000017814FF0010C0021B2FBFCF37F4AADF80A
:10D7100004101B0A7E49A2FB03231A09A1FB021273
:10D7200052084FF000081B09ABF87A2501A95200F6
:10D730000293ABF87825ADF80C80ADF806808DF833
:10D740000E8047F091FECDE90688CDF82080A379C0
:10D75000ADF81480602204929A0740F1AF80DB009C
:10D7600003F00803ADF81E300423ADF81430D6F8EA
:10D77000980E617904AAFEF7BBFF61790822FFF7D2
:10D7800087FCB0F84430D6F8948E6FEA43436FEAD2
:10D7900053439BB2A0F8443003889BB243F080030C
:10D7A0000380A3796179028C9B074CBF042301237A
:10D7B0008B409BB292B222EA03020284028C92B2A4
:10D7C0001343038403889BB243F0010303802A467A
:10D7D00000235168884502F1240203F101037DD042
:10D7E000102BF6D14FF0FF3303EBC30309EB830992
:10D7F000484AD9F88C3048498B420CBF4FF400138B
:10D800004FF48003116B0B43136300236A68904548
:10D8100005F1240503F101035DD0102BF6D13F493A
:10D82000602200235046FDF7FFFA404647F0E4FC33
:10D83000D6F8940E036823F001030025036047F037
:10D84000DBFCCDE91455CDE91655D6F8983E0E957A
:10D8500012956279D6F8940E099734331344304AFE
:10D860000B9240220A930C924FF480434FF4805263
:10D87000CDE9102340F22A414FF440330D91139328
:10D8800009A94FF480630F9347F04CFD6379D6F8F4
:10D89000981E0C2B04D8234A02EB4303B3F8CC5058
:10D8A0008B89D6F8942E9BB21D438D81136801207D
:10D8B00043F01003136019B0BDE8F08F5B0003F074
:10D8C0000203ADF81C300123ADF812304FF4807321
:10D8D000ADF820304BE75FFA83FAA0E7DBB2013BFB
:10D8E00082E7114A02EBC30393F8D407DBE600BFDB
:10D8F000E8180020140200208801002000000140E8
:10D90000D8EE050800040140006CDC02598B4F0181
:10D91000ABAAAAAA0038024000600240FD860008B7
:10D92000B04E002000F8050808E70508E0290020AF
:10D93000254B98420BD003F58043984207D003F55E
:10D940008063984203D003F58063984222D102F1AC
:10D95000B7731E4903F55853A1FB03139B0D013BFD
:10D9600099B2194B984201F1010C3FF4CDAE03F589
:10D97000804398423FF4C8AE03F5806398423FF479
:10D98000C3AE03F5806398423FF4BEAE5308B3FBC9
:10D99000FCF3BBE6530803F1B7730C4903F5585386
:10D9A000DAE7D6F8AC270A4B9A42FFF4AAAE074949
:10D9B00002F1B77303F55853A1FB03139B0D013B11
:10D9C00099B201F1010C9FE600000140819F5E16B3
:10D9D000006CDC02F0B50C4689B03C49BDF83860FB
:10D9E0009DF83C70013B054620689BB20493884239
:10D9F0004FF00003ADF81430ADF80E308DF816304E
:10DA000013D0334B984210D003F5804398420CD08A
:10DA100003F58063984208D003F58063984204D0F0
:10DA20002C4BD3F8AC375B0802E02A4BD3F8AC3769
:10DA3000B3FBF2F203A9013AADF80C2047F014FD54
:10DA400020686179A3790FB183F001030022CDE949
:10DA50000622ADF81020602203929A0729D5DB0038
:10DA600003F00803ADF81A300423ADF8103003AA10
:10DA700001910596FEF73CFE01990822FFF708FB8D
:10DA80002268B2F844306FEA43436FEA53439BB2D3
:10DA9000A2F84430138811469BB243F0010321F8E9
:10DAA000343B63796A60C81800222860CA5009B004
:10DAB000F0BD5B0003F00203ADF818300123ADF8B0
:10DAC0000E304FF48073ADF81C30D0E700040140F5
:10DAD00000000140E81800200B4B93F89425D3F880
:10DAE00084353AB113B11A689B885383074B0022DF
:10DAF0001A827047002BF9D01A689B881383034B56
:10DB000000221A82704700BFE02900200010004068
:10DB10000B4B93F89425D3F884353AB113B11A68B6
:10DB20009B881383074B00221A827047002BF9D081
:10DB30001A689B885383034B00221A82704700BFE8
:10DB4000E02900200014004070B5384C94F8A0552E
:10DB500084B00DB904B070BD94F8A13584F8943543
:10DB600028460BF017FFC4F8840508B13823C3809A
:10DB700094F898656EB3012EECD13146FDF76EFA3C
:10DB800094F89435002B49D1D4F8843513B11A6830
:10DB90009B881383264D4FF4E072D5F86831C4F8A2
:10DBA000902503A8012284F88025039347F00EFBFB
:10DBB000D5F86C31029302A847F008FB1D491E4CB2
:10DBC0000B6C1E48002243F030030B642285028553
:10DBD000C0E728463246382110F0CCF90546002827
:10DBE000B8D0C279D4F884050221FDF709FC144AA3
:10DBF00094F89435D2F8AC27124801935208802348
:10DC000029460096FFF7E6FED4F888158023012206
:10DC1000C4F890350B6084F880259BE7D4F88435F0
:10DC2000002BB7D01A689B885383B3E7E029002004
:10DC300000F80508003802400010004000140040C1
:10DC4000E8180020682F00202DE9F0415C4CDFED42
:10DC50005D7AB4F89A35DFED5C6A94F8985504EB78
:10DC6000400007EE103AB0F8A235B4F89E056422E1
:10DC7000B8EEC77A02FB03F327EE277A07EE903A55
:10DC8000F8EEE77A02FB003327EE277A07EE903AA8
:10DC9000F8EEE77A002687EE270A0F46C4F8AC654F
:10DCA00020EE260A55B3012D01D0BDE8F081D4F84D
:10DCB000908507EE908AF8EE677A27EE800A4FF09B
:10DCC000E3FE002832D194F89435002B66D0D4F8C6
:10DCD000843513B11A689B881383B4F89C053844C3
:10DCE0000EF0BAFF94F89435002B5FD0D4F8843549
:10DCF000002BDAD01A689B885383D6E7D4F8903586
:10DD000007EE903AF8EE677A27EE800A4FF0BCFEF5
:10DD1000D4F888252D4B1060D3F8B437B4F89C158F
:10DD200019443944C4F8B015BDE8F081284A294B9C
:10DD30005062C2F82C805E62C3F82C80EFF3118130
:10DD4000502080F312881580C9B21D8081F311889C
:10DD500095811E4A9D81D2F8B437B4F89C151944B8
:10DD60003944D2F8B4379942FBD81949194A0B887B
:10DD7000D4F8840523F001031B041B0C0B801388CB
:10DD800023F001031B0400241B0C13808C8194815D
:10DD900000288AD0036882881A8386E7D4F88435FD
:10DDA000002B9AD01A689B88538396E7D4F8843561
:10DDB000002B3FF47AAF1A689B88138375E700BF86
:10DDC000E02900200AD7233CCA269B3EE818002001
:10DDD0000010004000140040034B93F8802512B15E
:10DDE000042800D830E77047E02900201648174A79
:10DDF000174938B5174C184D121A50F0BDFBD4F81E
:10DE00008820164B164842F47002C4F888201A681D
:10DE1000002142F001021A6099601A6822F08472AF
:10DE200022F480321A6058601A6822F480221A6044
:10DE30000C4AD960521B28460B4950F09DFBA56047
:10DE4000BDE83840FAF7ACBD000000100400001037
:10DE5000D70E070800ED00E0000000200038024067
:10DE600010300024880100200000000808B50021BF
:10DE7000032047F0D9FA72B6FEF758F908B52E4CD0
:10DE8000D4F8B42594F8BA0552B111689388096999
:10DE90000B40002845D1003B18BF0123002BF3D1D4
:10DEA00014200EF0D9FE2549002000BFD4F8B43567
:10DEB00063B11A689B88156994F8BA252B4062BB38
:10DEC000003B18BF01230BB1FFF7D0FFD1F8B427F7
:10DED000D1F8B837D31A322B11D8D4F8BC359342C5
:10DEE000E3D2D1F8CC3A33B11D689B886E693342D6
:10DEF00014BF6B832B833232C4F8BC25D5E791F86D
:10DF0000CB3AD1F8CC2A03F001031AB17BB91368DC
:10DF100092881A83C4F8BC05C7E7B3FA83F35B0998
:10DF2000D1E7B3FA83F35B09002BADD1B8E71368EF
:10DF300092885A83EEE700BFE0290020E81800200D
:10DF400008B547F0D5FF0F490F4B91F8C5052922B9
:10DF50000228A3F8F22BA3F8FA2B01D0012008BD68
:10DF600091F8CC35012BF9D10848C1F8D00500F162
:10DF700020014C304BF088FC054B002083F8230037
:10DF800008BD00BFE0290020E81800206804002038
:10DF900000ED00E0024BD3F8B0371B6A184700BF12
:10DFA000E81800200A4AD2F8103873B11968988826
:10DFB000096992F80D3808401BB1B0FA80F04009A9
:10DFC0007047003818BF012070470120704700BF1C
:10DFD000E8180020034BD3F8B00708B1836918474D
:10DFE000704700BFE81800200378022B12D00F49B9
:10DFF00043680269D1F8480810B41840D1F8404885
:10E00000D1F83C18931E400A04FB030008445DF855
:10E01000044B7047054B4268D3F83418D3F83008E6
:10E0200000EB410000EB5220704700BF6840002029
:10E030002DE9F04F83B012F0020E019310D078B9A1
:10E040008D4D95F8E437A5F5805413B9012385F873
:10E05000E437012363700226304603B0BDE8F08F39
:10E06000854DD5F83878BFBB4FF0FF3C834C844FCB
:10E07000E146E046E24600262368984200F0BF8071
:10E0800094F80EB0BBF1000F3CD0BBF1010F15D1DD
:10E0900006F5B17B07EB0B1B9BF807B01BF0010FDC
:10E0A0000CD11BF07E0F09D15FEADB1340F0B58085
:10E0B000D4F808B0D34501D2DA46B14601360B2E6A
:10E0C00004F11004D8D1BCF1FF3F28D1B8F1FF3FD3
:10E0D0001FD06B4CC44623E0D5F84068D5F83C48C7
:10E0E00006FB0744A042BFD395F8E43713B90123D8
:10E0F00085F8E437624B0026012230465A7003B09F
:10E10000BDE8F08FB44601360B2E04F11004B3D1F4
:10E11000D9E7B9F1FF3F18BFCC4600F08680584CD4
:10E12000D5F8C86604EB0C1841F21869013648F8B6
:10E13000090041F21C690CF5B17748F809604FEA13
:10E140000718C5F8C86644F8086004EB07164FF0D6
:10E150000008C6F8048004EB0716B679042E00F216
:10E160008580DFE806F0031A621A300012F0010819
:10E170006BD104EB0710019B90F80790D61066F363
:10E18000C719032B80F807905DD94FF6FF708342C3
:10E1900028BF034604EB07108380BEF1000F12D0A6
:10E1A000D5F8C836D5F8CC0601330130C5F8C836E5
:10E1B000C5F8CC0604EB0C1041F21C65435104EB8E
:10E1C000071304209871500705D504EB0710C37995
:10E1D00043F00103C371D30608D504EB0714E379B8
:10E1E000C3F34502013262F34603E371254B012676
:10E1F00003EB4C2330460B6003B0BDE8F08F204C9E
:10E2000006F5B17704EB071C4FEA07189CF806C027
:10E21000BCF1000F0ED1B44682E7B04601360B2E9A
:10E2200004F110047FF428AF4DE70026304603B018
:10E23000BDE8F08FB446D5F8C866013644F80860EA
:10E24000C5F8C86687E74346A4E70F4B0D49D3F8E6
:10E25000B0370E4A9D6801EB4C210023A8470028E7
:10E26000E3D004EB07140223A371F5E695F8E43735
:10E27000002B3FF4EBAEECE6684000208046002027
:10E280006830002080300020E81800201D8D000834
:10E2900070B5104E3378022B0F4B0BBF020AC0F340
:10E2A000D412C4B200F07F04D3F8300882B0104416
:10E2B0000D460023032201A9FFF7BAFE012807D16A
:10E2C0003378022B019B0CBF23F8145043F82450E1
:10E2D00002B070BD68300020684000202DE9F04F8A
:10E2E000DFF82C8198F80060032E85B00C461546A7
:10E2F00043D001288CBF00220122022E0B6801921C
:10E3000069D14FEA1329DFB24FF4807A013801282E
:10E3100020D84FF0010B9D4217D93C4ED6F8A827C4
:10E320001AB1D6F8C417994258D0D6F8300800234D
:10E330004844092203A9FFF77BFE01282CD00228BC
:10E3400017D020B123689D42E8D82560032005B08E
:10E35000BDE8F08FF7B12D4B93F8E42712B90122F5
:10E3600083F8E4270123022088F8013005B0BDE8D6
:10E37000F08F022005B0BDE8F08F01288CBF00238C
:10E38000012301930B684FF0800AC3F3D41903F003
:10E390007F07BBE7D346BEE798F800200399DDF876
:10E3A00004C0022A14D0032AE3D151F8273023F005
:10E3B0007043B3FA83F35B0963455F44236821D05C
:10E3C0005B4457452360ECD309F101090027BAE704
:10E3D00031F81730EDE74FF4807AD6E7D6F84018D9
:10E3E000013A02EB41224902B2FBF1F21344B3FBC2
:10E3F000FBF20BFB12320AB15B449B1A9D42236075
:10E400008CD8A2E7AB42A2D39FE700BF68400020B0
:10E41000683000202DE9F04FDFF86CB19BF800C0A8
:10E42000BCF1020F894683B009688246174640F066
:10E430008C800BF58053CEB2D3F83058A6EB010890
:10E4400005EB112590444FF480739844B94208F1CC
:10E45000FF38B8FBF3F84CD2A844BCF1030F07EB2C
:10E4600006040CBF80224FF48072641A9442A8EB19
:10E47000050328BF144666B994422CBF0A220B221A
:10E4800001A92846FFF7D4FD012809D003B0BDE853
:10E49000F08F0B2201A92846FFF7CAFD0128F5D10C
:10E4A0009BF800C0D9F80010BCF1020F01F1010384
:10E4B00023D0B44210D9019906F18042013A01EB10
:10E4C0008202043901EB840142F8043F914203F1D6
:10E4D0000103F9D1D9F80010A61B3144BAF1010F9C
:10E4E000C9F8001021D08F4205F101054FF0000658
:10E4F000B3D8012003B0BDE8F08FB442ECD9019845
:10E5000006F10042013A00EB4202023800EB4400FF
:10E5100022F8023F904203F10103F9D1A61B3144D6
:10E52000BAF1010FC9F80010DDD1B942DBD1BCF15D
:10E53000020F1DD004F18044019B013C4FF0FF32DB
:10E5400043F82420D9F80010CDE70BF5805301F0F3
:10E550007F06D3F83038BCF1030FC1F3D415A6EB16
:10E5600001081D44904414BF4FF4807380236CE76E
:10E5700004F10044019B013C4FF6FF72504623F822
:10E58000142003B0BDE8F08F6830002030B5044699
:10E59000C06983B010B9012003B030BD0D4600231F
:10E5A000032201A9FFF744FD0128F5D1B4F9203079
:10E5B000002B0ADA144B93F8E4270AB983F8E4072E
:10E5C000124B01225A700220E6E7019A012D4FEA10
:10E5D000431102EB431303D0022D11D1E52555540D
:10E5E000A268DA612278032A04D100221A775A77C6
:10E5F0009A77DA77626A5A83120C9A8203B030BD36
:10E60000E268DA61EEE700BF684000206830002071
:10E610002DE9F04190F83C30002982B0044614BF47
:10E6200002210021042B7BD8DFE803F0030C3D48D6
:10E630006900FFF7ABFF012870D1626B002A75D12A
:10E6400084F83C00404EDFF808814FF6F77706F576
:10E65000805516E0BA424FD84BF03EF801284FF0F3
:10E6600000011DD1206BFFF713FE012818D1019A7C
:10E67000D5F844382263511E8B4228BF0B46C5F89B
:10E6800044383278236B032A01A918469AB2E1D1A3
:10E69000434531D84BF020F801284FF00001E1D07C
:10E6A00002B0BDE8F081426B04F130010020FFF7B9
:10E6B000B1FE012832D1032384F83C302348E16ABB
:10E6C000D0F8C437D0F84028C0F8C4175B1A02FB52
:10E6D00003F3D0F8A82702EB4322C0F8A827D0F80C
:10E6E000AC2702EB4323C0F8AC37002100F5F460FF
:10E6F000FFF74CFF012811D1042384F83C3094F833
:10E700002830042B04BF002384F82830A36B8BB17E
:10E7100020469847012002B0BDE8F0810228BFD111
:10E7200094F82830042B09D00220B9E7022384F89A
:10E730003C30B9E7012002B0BDE8F081002384F845
:10E7400028300220ACE700BF68300020684000207D
:10E75000F7FFFF0F38B590F834300446052B43D847
:10E76000DFE803F01E033C0F185E006B4FF0FF3133
:10E77000FFF78EFD012837D1E06AB8BB032384F888
:10E78000343000212046FFF701FF01282CD104235B
:10E7900084F8343094F82830082B2BD0012038BD71
:10E7A000204DD5F8382800F1300102320120FFF762
:10E7B00095FD012823D00238C0B2012814D80523C2
:10E7C00084F8343094F82830082B04BF002384F8F0
:10E7D0002830012385F8E537022038BDC06A216B57
:10E7E000FFF756FD0128C9D0002038BD022384F868
:10E7F0003430F4E7002384F82830012038BDE36882
:10E80000D5F84018D4E90B2003EB4123C5F84408A0
:10E81000C4E9033002B96062012384F83430A5E70B
:10E82000004DCFE76840002010B590F8383004461E
:10E83000032B59D8DFE803F0022F38432B4AC06876
:10E84000117802F580530329D3F84018D3F8C42770
:10E850000CBF4FF0800C4FF4807C01FB0CF100EBFF
:10E860004120C4E90302D3F8A807A0EB4120C3F874
:10E87000A807D3F8AC07A0EB4121E06AC3F8AC17B6
:10E8800002EB0C01C3F8C417C4E90C2140BB62625F
:10E89000012384F8383016480021FFF777FE01285D
:10E8A00011D1022384F83830626B04F13001012069
:10E8B000FFF7B0FD012806D1032384F8383000218A
:10E8C0002046FFF763FE431EDBB2012B00D910BDCB
:10E8D00094F82830062B04BF002384F8283010BD9C
:10E8E000A2EB0C022263D3E70220ECE768300020A1
:10E8F000084800202DE9F0434368C3F308020A44A6
:10E90000B2F5007F83B004460D4605D22B44636008
:10E91000012003B0BDE8F08390F91A20501C0AD002
:10E92000414902F5B17201EB0212D1796FF3000196
:10E93000D171FF22A27694F91B20511C0FD03A49C5
:10E9400002F5B17201EB0212FF26D179C1F3450045
:10E95000013820EAE07060F34601D171E67694F860
:10E9600000C0BCF1020FD1D0DFF8C480D8F8402835
:10E97000B5EB422F4FEA422915DCD8F848781F4002
:10E980007A42AA420FDCEA194A4510D220690028CF
:10E99000BED0254A1278032A40D080B24FF6F772D3
:10E9A0009042B3D9B4E7002003B0BDE8F083227EE3
:10E9B000206912F0080626D0D8F8C427411C8A42E4
:10E9C00013D300D100214B44A5EB0905DB1BBCF19F
:10E9D000020F60613D44216163600846D7D1D8F8D9
:10E9E0005028B3EB422F91D392E798F8E42722B94D
:10E9F000012388F8E437636820690B4A01265670C2
:10EA000094F800C0DFE701A94AF066FE0128CAD1E8
:10EA10000199636894F800C02069D4E7034A9042E2
:10EA20007FF674AF74E700BF68300020F7FFFF0F78
:10EA3000684000202DE9F04790F8384082B0054644
:10EA4000032C00F2AB80DFE804F00219710BFFF732
:10EA500081FE012810D002280AD1032385F838301E
:10EA60002B6C002085F82800002B6FD098470224DB
:10EA7000204602B0BDE8F08785F838002B78022BDD
:10EA800060D0474A6B68D2F8482803EA0208C8F306
:10EA90004F282846FFF7A8FA414F0646A8EB000882
:10EAA000A7F5805901A9022200233046FFF7C0FADA
:10EAB00008EB060401281FFA84FA4FF400724FF0A5
:10EAC00000010446D4D101984FF0B9FDEB694FF431
:10EAD0000071284613B16B68002B3BD0D7F8403843
:10EAE000013B9A4506F101060DD2FFF703FF00280E
:10EAF000D8D197F8E43713B9012387F8E437012315
:10EB000089F80130CEE7C3EBC35359022846FFF71B
:10EB1000F1FE40B997F8E43713B9012387F8E437D9
:10EB2000204B01225A70022385F838302B6C0022CA
:10EB300085F8282063B1284698470124204602B072
:10EB4000BDE8F0876B68C3F34F28A2E702248FE784
:10EB500001248DE7019B4FF020324FF02E0E4FF035
:10EB6000100C1A605A6083F800E0C3F807206C6A42
:10EB70001A625A6283F80BC0C3F8272083F820E09A
:10EB800083F821E0EA6B5C835A8724FA0CF422FABA
:10EB90000CF29C8283F82BC09A869FE7002467E7DB
:10EBA00068400020683000202DE9F041B1F90430C0
:10EBB0000F2B82B00E460446174635D02046FFF78D
:10EBC00013FA94F91B80B8F1FF3F3ED0554B41F248
:10EBD000186203EB08118A58904211D1183303EBE5
:10EBE0004825B38801331BB205EB4315B38020469B
:10EBF0003D60FFF7F9F93060012002B0BDE8F08117
:10EC000003F5805292F8E41700296AD001225A7065
:10EC10002278022A69D02369002B50D100230120D9
:10EC20003B6002B0BDE8F0814FF40071FFF762FE77
:10EC3000002852D04FF6FF73B3802046FFF7D4F977
:10EC400094F91B80B8F1FF3FC0D12278022A54D03A
:10EC50002369002BDDD03349097803290EBF3249DF
:10EC60009BB24FF6F7718B4294BF00230123002B18
:10EC7000CFD138B92D4A92F8E437002B4ED0294B2A
:10EC800001225A700023112201A9FFF7D1F90128AE
:10EC900042D1019D264BEB1A48BF03F2FF13B3F597
:10ECA000B05F4FEA632230D3204A92F8E43713B9B9
:10ECB000012382F8E4371B4B01225A7027E0194ADE
:10ECC0001278032A0EBF184A9BB24FF6F77293428E
:10ECD00094BF00230123002BA0D1002002B0BDE887
:10ECE000F081012182F8E41790E7104A6368D2F8B6
:10ECF0005028B3EB422F91D2EFE70C4A6368D2F869
:10ED00005018B3EB412FB4D3F1E74FFA82F884F8EF
:10ED10001B80002D7FF465AF22787AE7012382F80B
:10ED2000E437ACE768300020F7FFFF0F68400020B1
:10ED3000803000202DE9F04790F8303088B004464C
:10ED4000042B4BD8DFE803F0030C4DD14600C54837
:10ED50004CF038F94FF6FF720123228484F83030EA
:10ED6000DFF8008304F11C0501AE04F131093246DD
:10ED700029464046FFF718FF012800F0DB800228F3
:10ED80002CD1B94901F5805595F90228531C0AD0B8
:10ED900002F5B17201EB0212D3796FF30003D37164
:10EDA000FF2385F8023895F903385F1C0FD003F56F
:10EDB000B17301EB0313DA79C2F34501013921EA9A
:10EDC000E17161F34602FF21DA7185F8031804232B
:10EDD00084F830300020E36A2070984708B0BDE81E
:10EDE000F087A24D95F81038002BF7D19D4F04F114
:10EDF0001C0901AE4FF00908324649463846FFF774
:10EE0000D3FE012840F0E8800198002800F0C2807D
:10EE10000378E52B01D0002BEED1954A821A48BF2A
:10EE200002F2FF12B2F5B05F4FEA622380F00E816A
:10EE30008D491B018F4A13449A7B042A0CD0D5F8C4
:10EE4000C8260132C5F8C8265A6004229A73D5F83C
:10EE5000CC360133C5F8CC3695F902385E1C0AD0A1
:10EE600003F5B17301EB0313FF2285F80228DA7969
:10EE70006FF30002DA7195F903385A1C0FD003F5CD
:10EE8000B17301EB0313FF21DA7985F80318C2F39C
:10EE90004501013921EAE17161F34602DA7120226C
:10EEA00000214FF0CCFB019BD4F83120D4F8351071
:10EEB00059601A60B4F8392094F83B1099721A819D
:10EEC000019B627EDA7205A802F01CFABDF81430CC
:10EED000002B40F0058144F28171019A03201182D8
:10EEE000D3811183D38284F83000237E980608D51D
:10EEF000E0690023112205A9FFF79AF801287FF4A1
:10EF00006DAF20464CF05EF82369002B68D0237E5D
:10EF100003F0F70213F0040322766ED1122A00F0F8
:10EF200083800022E36A84F828202046984708B0AE
:10EF3000BDE8F087019F002F00F09E803B78002BFA
:10EF400000F09A8097F80BA01AF0080F7FF40FAF2B
:10EF50000B22494638464FF0AFFB00287FF407AF3D
:10EF6000637E8AEA0303DB0640F1FB803E4901F53C
:10EF7000805595F902385E1C3FF415AF03F5B17367
:10EF800001EB0313FF2285F80228DA7960F300020F
:10EF9000DA7108E795F8E837022B3FF418AF95F8D7
:10EFA0001038002B7FF413AF85F82038C5F82438CB
:10EFB000C5F8283885F81C38D5F8FC37C5F814385A
:10EFC000D5F8443885F81088C5F818383846FFF762
:10EFD00031FD01283FF410AF02283FF4F8AEFDE602
:10EFE000237E19079DD5214B93F8C827002A7FF46B
:10EFF000F5AE072283F8C82793E7A568E66A0023E1
:10F0000084F8283029462046FFF774FC002840F099
:10F01000A28094F82830002B7FF4E0AE0223C4E9EC
:10F020000B6584F82830D9E6626AE16AA16304209E
:10F0300084F82800C4E90B22C4E9023384F83C3088
:10F040006363636220464BF0BDFFC7E695F8E43783
:10F0500013B9012385F8E437034901234B706FF09E
:10F060000F03E7E650480020683000206840002089
:10F070008030002080460020584901F5805595F9E0
:10F0800002385E1C0AD003F5B17301EB0313DA7981
:10F090006FF30002DA71FF2385F8023895F903381F
:10F0A000581C0FD003F5B17301EB0313DA79C2F3E7
:10F0B0004501013921EAE17161F34602FF21DA716C
:10F0C00085F80318237EDA067FF581AE44484BF0BD
:10F0D00079FF4FF6FF720223228484F8303081E6F4
:10F0E000404B05A8B3F9D48502F036F84FF47A7294
:10F0F000002306460F464DF073FC3C23054608FBF3
:10F100000355394630464FF47A7200234DF068FCBF
:10F110004FF47A7192B20023C5FB012302A802F0DA
:10F1200051F89DF80A209DF80B109DF80C3041EA2B
:10F130004211BDF80820A2F2BC7241EA42219DF8BA
:10F140000D20DB0243EA42139DF80E2043EA5203EE
:10F1500089B29BB2C1E6002E3FF440AE2046B047D4
:10F160003CE6BA8A7B8B204D43EA02436362D5F8C2
:10F170004028FB69A3605202B3FBF2F102FB11319C
:10F1800009B113445B1AE36084F819A095F90238B9
:10F190001249581C0AD003F5B17301EB0313DA7955
:10F1A0006FF30002DA71FF2385F8023895F903380E
:10F1B0005A1C0FD003F5B17301EB0313DA79C2F3D4
:10F1C0004501013921EAE17161F34602FF21DA715B
:10F1D00085F80318032384F8303086E66830002071
:10F1E00050480020E02900206840002010B5037836
:10F1F00090F818C0023B012B044602D91CF0060F00
:10F200005DD11CF0200F3CD194F91A30591C0AD062
:10F21000314A03F5B17302EB0313FF21DA796FF37F
:10F220000002DA71A17694F91B305A1C0FD02A4AD9
:10F2300003F5B17302EB0313DA79C2F34501013927
:10F2400021EAE17161F34602FF21DA71E1761CF0F7
:10F25000080F0DD0214B93F8C827072A05D093F843
:10F26000E427A2B31C4A01215170002283F8C82769
:10F27000E26A0023237084F82830FAB1BDE8104018
:10F28000104700231649E0691A018A58904206D0B7
:10F2900001330B2BB8D01A018A589042F8D10E4A8C
:10F2A00003F5B17302EB0313DA79C2F345010139B7
:10F2B00021EAE17161F34602DA71A5E710BD01218F
:10F2C000FFF764F90128F9D194F818C099E70122F1
:10F2D00083F8E427C6E700BF6830002068400020BC
:10F2E000804600204FF0FF3C2DE9F041354A36487A
:10F2F0006446002304E001330B2B02F1100216D008
:10F3000011780429F7D103F5B17100EB0111C97926
:10F31000CE07F0D4651C52F80A1C01D06145EAD230
:10F320001C4601330B2B8C4602F11002E8D1631C02
:10F3300002D10120BDE8F081234D04F5B17705EB42
:10F340000713998809BBDFF88C802601D8F8B0270D
:10F35000AB19D2F810801D4E41F2186206EB442121
:10F3600098581B4A0023C047E0B102280AD106F68C
:10F37000E87605EB0715D6F8CC360122013BC6F836
:10F38000CC36AA710020BDE8F081DFF8488005EB9B
:10F390000413D8F8B02741F21860D2681858260133
:10F3A0009047D3E706F6E87605EB0715D6F8CC3696
:10F3B000013B0322C6F8CC360123AA7186F8D03669
:10F3C000B8E700BF8E460020683000208030002063
:10F3D000958D0008E81800202DE9F04F90F82830AE
:10F3E000013B83B00446082B0BD8DFE803F0383C20
:10F3F0001E2305290A2E33000121FFF709F90128F0
:10F4000002D003B0BDE8F08F2378002284F82820D2
:10F41000002BF6D0D4E901138B4238BF0B46226C87
:10F42000A360032184F82810E262204603B0BDE8FF
:10F43000F04FDBE6002103B0BDE8F04FFFF7E8B87E
:10F4400003B0BDE8F04FFFF7EFB903B0BDE8F04FF0
:10F45000FFF780B903B0BDE8F04FFFF7EBBA03B098
:10F46000BDE8F04F66E4534F4368D7F84858016B46
:10F47000D7F840281D406818B0EB422F4FEA4226CB
:10F480009C46C0F0938094F800E0DFF82C91A7F53B
:10F49000805A4FF6F778BEF1020F14D02069002889
:10F4A00057D1D4F804C0A368E26A634538BF634605
:10F4B0000021A36084F82810002AA2D0204603B0BF
:10F4C000BDE8F04F1047D4F804C0D7F85028BCEB83
:10F4D000422FE8D22069227E12072CD5D7F8C42704
:10F4E00000F1010C624522D297F8E42722B90123EA
:10F4F00087F8E4376368216B01228AF8012094F8C9
:10F5000000E0891B294433445B1B8E42C4E904C0DC
:10F51000636021639C464FF00005BCD9BEF1020F29
:10F520003ED020690028BED0DFF890B01FE0E8D1BF
:10F530004FF0000CE5E701A94AF0CEF801287FF46E
:10F5400060AF2069DDF804C094F800E06368216BC7
:10F55000D7E79AF80020032AD3461AD082B2424550
:10F5600094BF00220122002AB5D0D4F804C09BF831
:10F570000030032B0EBF104B80B24FF6F77398424A
:10F5800094BF0020012000288DD18C44C4F804C011
:10F5900089E7484594BF00220122002A9BD0E4E776
:10F5A000D7F85028B3EB422FEFD37CE794F800E074
:10F5B000B4E700BF68400020F7FFFF0F683000206D
:10F5C00010B5194C1948442200214FF038F823781F
:10F5D00004F580544FF6FF70D4F84C28A4F80208C4
:10F5E000022B4FF0030118BF03234FF0100C84F8D7
:10F5F000001804F5FD600021C4F8F82784F8E83706
:10F60000C4F80C2884F801C8FFF774F948B994F8D5
:10F61000103833B9022284F81028C4F81438C4F81A
:10F620001838012010BD00BF68300020504800206D
:10F6300043F201020121028043F20112002343F24E
:10F64000015C017282804FF47F41FF22A0F802C06A
:10F6500043818381C381018282747047154BFF22ED
:10F660004FF0FF3CF0B5C2700271027242724273F9
:10F67000827303F10C076646172516244FF0150E0A
:10F68000002202EB820281189F4200F802E04C70D7
:10F690008D70CE7081F804C00BD093F9062093F8DA
:10F6A00007E01C7A5D7A93F90A6093F90BC0063380
:10F6B000E7E7F0BDA4F905084FF0000C0121022294
:10F6C000032380F805C08171C2710372704700BFC7
:10F6D00000230222037043708370C370027170476D
:10F6E0004FF0010C2C210222002380F800C0417051
:10F6F0008270C370704700BF4FF4F07140F22E4C1F
:10F7000001804FF47A71A0F81EC041844FF4FA6C66
:10F710004FF4F561A0F820C0818440F2262C42F21B
:10F720002011A0F81CC0418142F2267C41F62A71CA
:10F730000023A0F808C0C18143F6381C0E2107221F
:10F74000A0F80CC080F8261040F2012C43718371A0
:10F750004374438240F2034140F205638270A0F893
:10F7600014C0C18203838276704700BF8388C3F3CD
:10F770000B039342A8BF134670B51A461D460C46AC
:10F78000064680684EF0F8FE62199442B569074B50
:10F7900008D0074814F8011B00FB03F3A24283EAD8
:10F7A0000103F7D12B60012070BD00BFC59D1C81F6
:10F7B000930100010023037043708370C37070478E
:10F7C0000023037043708370C370704700220123CD
:10F7D0004FF02B0C812180F800C042708270C27003
:10F7E000017143718371C371704700BFFF23002211
:10F7F000027043708370C370704700BF00230621FE
:10F800004FF47A72C0E9012301700373704700BF9F
:10F8100001234FF0000C03213E2280F801C0C37089
:10F82000017082700371704710B50023411CFF22E4
:10F8300000F8132001F8132001330B2BF8D10B4BE8
:10F840004FF0FF3103F10F0400228C4605E093F9DD
:10F8500004C093F9051013F8032F00F812C000EB51
:10F86000420E9C428EF80110F1D110BDB8F9050886
:10F870004FF0260C80F800C04FF0270C00B580F840
:10F8800003C04FF02A0E4FF0200C80F806C080F81D
:10F8900012E04FF0210C4FF01F0E80F809C080F8E5
:10F8A00015E04FF0380C4FF02F0E0122022180F8A6
:10F8B0000CC080F818E04FF0390C4FF02E0E0023EA
:10F8C00042700271C1718172417380F80FC001747E
:10F8D0004FF0030CC2748275C27780F81BE0FF22E0
:10F8E00013214FF0180E837043710372C372837338
:10F8F00043740375C37580F819C080F81CC0827604
:10F90000427780F81EE080F8203080F8211080F8DF
:10F9100022C080F823205DF804FB00BF032303709E
:10F92000704700BF0A44914219D000B501F1FF3C75
:10F9300002F1FF3E41F221011CF8012F082380EA69
:10F94000022010F4004F81EA40020ABF400090B24A
:10F9500080B2013BF5D1E645EED15DF804FB70477E
:10F96000704700BFD0ED007AD0ED016A30EE677AC3
:10F97000E6EE877AB0EE670AC0ED007A704700BF06
:10F98000D0ED017AD0ED026A30EE677A90ED000A90
:10F99000E6EE877A37EEC07AC0ED017AA6EE870AE6
:10F9A00080ED000A704700BF90ED017AD0ED036A48
:10F9B000D0ED027A30EE470AA6EE807A90ED000A8A
:10F9C00080ED017A37EE676AE6EE867A37EEC07A26
:10F9D000C0ED027AA6EE870A80ED000A704700BFEC
:10F9E000DFED277AB4EEE70AF1EE10FA0CDDDFED79
:10F9F000256A9FED257AF0EE407AF4EEC77AF1EEB3
:10FA000010FA30EE660AF6DCDFED207AB4EEE70A93
:10FA1000F1EE10FA0CD5DFED1B6A9FED1D7AF0EECA
:10FA2000407AF4EEC77AF1EE10FA30EE260AF6D4F8
:10FA3000DFED187AB4EEE70AF1EE10FA14DDDFED2F
:10FA4000107A37EEC00A60EE006A9FED136A9FEDF0
:10FA5000137ADFED137AA6EE867A20EE266AE6EEBA
:10FA6000877AA6EE270A7047DFED0E7AB4EEE70A32
:10FA7000F1EE10FA44BFDFED057A37EEC00AE2E797
:10FA8000DB0F4940DB0FC940E4CB1641DB0F49C017
:10FA9000E4CB16C1DB0FC93F92E741B99730083C70
:10FAA00015A82ABEDB0FC9BFD0ED056AD0ED017ADB
:10FAB00090ED007A90ED066AD0ED025A90ED035A6F
:10FAC00080ED050A66EEA77AC0ED066AE7EE007AD9
:10FAD00090ED077AE5EE867A90ED086AD0ED045A4B
:10FAE00080ED087AE5EE477AE5EEC67AB0EE670A71
:10FAF000C0ED077A704700BFD0ED057A90ED006A3F
:10FB000090ED067AD0ED035AE6EE007A90ED016AA8
:10FB1000F0EE406AA6EE267AB0EE670AD0ED047ADF
:10FB200090ED026A67EEC07AA5EEC07AE6EE267A1C
:10FB300080ED057AC0ED067A704700BF2DE9F047E9
:10FB4000089F3C460E4614F8011B002B054614BFC7
:10FB50004FF030094FF0200941B3002A2CDD234635
:10FB600000E0B2B113F8010B9046013A0028F8D139
:10FB7000A8F102086AB1C24649462846B047534632
:10FB8000002B0AF1FF3AF7DC397828EAE8720132F3
:10FB900049B1D71B2846B047E01914F8011B0029CA
:10FBA000F8D1BDE8F0871046BDE8F087002A02F1E1
:10FBB000FF38E0DC0846F4E70022EAE703685A1C55
:10FBC00002601970704700BF024B186803681B6819
:10FBD000184700BF585F0020884210B54FF001045D
:10FBE0003ED301FB04F4B0FBF4FC8C45F9D2CCB15C
:10FBF00022BB08E0A14203F801EBB4FBF1F211D8FB
:10FC0000B0FBF2FC1446BCF1090F0CF1570E0CF1DD
:10FC1000300204FB1C00EDDCA14203F8012BB4FB15
:10FC2000F1F2EDD900221A7010BDA14203F801EBE8
:10FC3000B4FBF1F2F6D8B0FBF2FC1446BCF1090FAC
:10FC40000CF1370E0CF1300204FB1C00EDDCA1427C
:10FC500003F8012BB4FBF1F2EDD900221A7010BDAC
:10FC60008446002AEAD1CEE7002870B503DA2D23B6
:10FC700001F8013B4042092886464FF0010307DDA9
:10FC800003EB83035B00B0FBF3F2092AF8D8EBB176
:10FC9000104CBEFBF3FCA4FB0320C008BCF1090F11
:10FCA0000CF130060CF15705024607D8092B01F874
:10FCB000016B03FB1CEE09D90346EAE7092B01F8A7
:10FCC000015B03FB1CEE01D91346E2E700230B7036
:10FCD00070BD00BFCDCCCCCC0378202B024600F108
:10FCE0000100F9D0092BF7D02D2B28D02B2B03BFE7
:10FCF0005378B7EE000A0246B7EE000AA3F13001CE
:10FD0000C8B209289FED567A10D8F2EE046A07EEC1
:10FD1000901AF8EEE77A12F8013FE7EE267AA3F19F
:10FD20003001C8B20928B0EE677AF0D92E2B5ED028
:10FD300003F0DF03452B07D020EE070A7047537806
:10FD4000BFEE000A0246D9E710B451782D2978D0C9
:10FD50002B296AD0A1F13003092B02F101026BD8E3
:10FD60000024002303EB830301EB430312F8011F7C
:10FD7000A1F130000928A3F13003F3D9B3F59A7F3C
:10FD80001A4628BF4FF49A72072B66D9DFED356A01
:10FD90001346F7EE007A083B072B67EEA67AFAD8EF
:10FDA00002F00702DAB1F2EE046A012A67EEA67ADF
:10FDB00015D0022A67EEA67A11D0032A67EEA67A3A
:10FDC0000DD0042A67EEA67A09D0053A67EEA67A26
:10FDD00005D067EEA67A012A18BF67EEA67A6CB343
:10FDE00087EE277A5DF8044B20EE070A70475378B8
:10FDF000A3F13001C8B2092802F1010298D8F2EE4D
:10FE0000046AF0EE665A07EE901AF8EEE77A12F8F6
:10FE1000013F87EEA66AA3F13001C8B2092866EE59
:10FE2000A56A37EE067AEED982E79178A1F1300320
:10FE3000092B02F1020293D9F7EE007A27EE277A16
:10FE4000D0E79178A1F13003092B02F1020288BFBB
:10FE5000F7EE007AC4D8012483E7F7EE007AA1E731
:10FE60000000000020BCBE4CF8B5164D6B78BE2BD0
:10FE700025D1022229464FF6FF70FFF753FD124F9E
:10FE8000AC1C22884AB1A618BE4218D2052A16D93F
:10FE90002146FFF747FD3446F3E721460222FFF7EC
:10FEA00041FD0222A118FFF73DFD0634074B641BFC
:10FEB0009C8041F60F53C31A58425841F8BD0020A8
:10FEC000FCE700BF0040000800800008585F0020E9
:10FED000F0B5067906F0E003402B03D145794FF0E9
:10FEE000FF3406E0602B4FF00105F8D1447905FAA4
:10FEF00004F40023012006F00706AB4200D1F0BD58
:10FF0000052E0FD8DFE806F00308101D242448B1A1
:10FF1000C85CD75C78400FE020B1C856D756C71BE5
:10FF2000784278410133E8E70028FBD031F813002C
:10FF300032F81370784080B220420CBF01200020BC
:10FF4000F0E70028EED031F9130032F91370E6E73C
:10FF50000028E7D051F8230052F82370DAE703793C
:10FF600003F01803102B1CD004D82BB1082B06D09B
:10FF700000207047182BFBD1B0F80B007047104BD6
:10FF8000B0F80B0093F90030591C06BF0D4B1B7ADB
:10FF9000DBB203EB830203EBC20300EB830080B20E
:10FFA0007047074BB0F80B0093F901305A1C06BF9D
:10FFB000044B5B7ADBB2C3EB031300EB4300EEE7C9
:10FFC00010050020585F0020114A002330B503605F
:10FFD000838002F10C054FF448744FF0290E4FF066
:10FFE000280C03EB430300EB430100F813C081F836
:10FFF00001E0D3788B70AA428C8008D092F9063049
:020000040801F1
:1000000092F807C092F808E054890632E9E730BD5B
:10001000CCF90508092900D001B9704701394B0016
:1000200003F00802930001F00301A3EB9203C1EB7C
:100030000111C3EB0313C1EB011100229B008900E6
:10004000026081804380704784B04FF46173ADF8E3
:1000500004300199ADF80C10BDF80C1081814FF4FB
:10006000007C41F201420023A0F800C042804FF41E
:100070000D7C01220093A0F806C08360C28104B009
:10008000704700BF144B154910B5044618681B791A
:10009000206284F82430152204F125004EF020FB64
:1000A0000F4B1A7E4FF0010E84F83AE012B984F833
:1000B0003B2010BD03F11C0CBCE80F002060616008
:1000C000A260E360BCE80F0084F83BE0206161615E
:1000D000A261E36110BD00BFF45E0608FC5E060885
:1000E000585F002010B50021382204464EF0A7FAD0
:1000F0000D490E4A0E482061C4E905120D480E4A0A
:10010000E061012341F61E614FF0090CE18484F89F
:1001100008C0A37384F82130A26221460748BDE8D5
:10012000104030F045BB00BF1A046C07001975037E
:100130006400DC0543080E001E7D01010C5F06080B
:10014000B5EEC00ADFED347AF1EE10FACCBF30EE36
:10015000270A30EE670ADFED317A20EE270A70B504
:10016000FDEEC07A86B017EE904A054684EAE47048
:10017000002303A9A0EBE470CDE90033029346F01D
:10018000EBFC002CACBF20232D2303A88DF80030FE
:100190004BF062FF01286E4628D0022832D0032897
:1001A0001CD003A930464EF052FA30464BF054FFB3
:1001B0000338C4B22246314628464EF0DDF900230A
:1001C0002B5528464BF048FF2E232B540130311974
:1001D00028444EF058FA284606B070BD302303A9D3
:1001E00030468DF801304EF032FADEE743F230024D
:1001F000302303A93046ADF801208DF803304EF0CE
:1002000026FAD2E743F2300303A93046ADF80130B5
:100210004EF01DFAC9E700BF6F12033A00007A449E
:1002200008F0F8BE13B568B14C1E14F8011F21B9CF
:1002300002B0BDE8104008F001BF019008F0EAFEEE
:100240000198F2E702B010BD08B520214EF00EFA79
:10025000034620B11A78202A00F10100F8D0184690
:1002600008BDF8B5D0B1104B0138C70003EBC00092
:10027000CA4390F8406090F8415002F0010282EACF
:100280000604A5420AD0C06B28B185880068B24236
:1002900014BF058345833B4483F84140CB0701D419
:1002A000FBF756FFF8BD00BF585F00202DE9F34172
:1002B000124D134F002305F85C3F044600EB810606
:1002C000B44203D10F4802B0BDE8F0813946284658
:1002D0004EF0BDF9214668464EF0D5F94FF00008C2
:1002E000202168464EF0C2F928B9694628464EF0EA
:1002F000AEF90434E4E780F80080F1E7585F0020AD
:100300009FB30608B45F0020024BD3F880003BF097
:10031000EDB800BF585F0020084B09498B420246E8
:100320000AD2184602E01C30884205D20388C3F383
:100330000B039A42F7D170470020704790EC0608F3
:100340006CF5060870B50546B0F80900FFF7E4FF44
:10035000064B93F8846004462846FFF700FE16B16A
:10036000E368184470BDA368FBE700BF585F002036
:1003700038B505460C46FFF7E5FF2B7903F0E002A0
:10038000602A03F007032AD1052B0CD8DFE803F01D
:10039000030B0F0B1B1B6A7901239340DBB202781E
:1003A00014B11343037038BD22EA0303FAE76A79F4
:1003B000012393409BB2028814B113430380F2E7F8
:1003C00022EA0303FAE76A79012303FA02F20368D7
:1003D00014B113430360E6E723EA0203FAE7052BAF
:1003E000E1D8DFE803F00303050507070470DAE747
:1003F0000480D8E70460D6E770B585880B460446CC
:10040000C5F30B052A46002118464EF018F961691C
:10041000084A9142034602D3074A914205D319B1D3
:10042000BDE870401846084770BD2A46BDE87040D8
:100430004EF0A2B86CF506087BF7060838B5064CF6
:10044000064DAC4206D2A16820461C34FFF7D4FF0B
:10045000AC42F8D338BD00BF90EC06086CF5060836
:100460004840082310F0800F82EA40010ABF400094
:10047000C8B2C0B2013BF5D1704700BF30B50568C6
:100480008D4219D901F1FF3E6C1E00231EF801CFE9
:10049000082183EA0C0313F0800F82EA430C0ABFA1
:1004A0005B005FFA8CF3DBB20139F4D17445EDD116
:1004B0006A1C02602B7030BD00236A1C02602B7026
:1004C00030BD00BF07EE901AB8EE677ADFED7C7A98
:1004D00027EE000A60EE277ABDEEE77A17EE103AB3
:1004E0002033402B00F2DB809FED767AB4EEC70A12
:1004F000F1EE10FAB0EE677A0CDDDFED735A9FED86
:10050000736AF0EE476AF4EEC66AF1EE10FA37EE5F
:10051000657AF6DCDFED6E6AB4EEE67AF1EE10FA9B
:100520000CD5DFED695A9FED6B6AF0EE476AF4EE89
:10053000C66AF1EE10FA37EE257AF6D4DFED666A78
:10054000B4EEE67AF1EE10FA00F39D80DFED636A17
:10055000B4EEE67AF1EE10FA44BFDFED5D6A36EEF6
:10056000C77A27EE075ADFED5E5A9FED5E6ADFED30
:100570005E6ADFED5E4AA5EE256A27EE054AE5EEE6
:10058000066AF7EE005AA4EE267AF0EE656AE7EE08
:10059000646AE7EE245A86EEA54A9FED4F7A77EE1D
:1005A000877ABDEEE77A17EE103A2033402B6FD8EA
:1005B0009FED4F7AB4EEC70AF1EE10FA0CDD9FED15
:1005C000426ADFED426AB0EE677AB4EEE67AF1EEA7
:1005D00010FA77EEC67AF6DC9FED3D7AF4EEC77A34
:1005E000F1EE10FA0CD59FED386ADFED3A6AB0EE05
:1005F000677AB4EEE67AF1EE10FA77EE867AF6D400
:100600009FED357AF4EEC77AF1EE10FA4CDD9FEDEE
:10061000397A77EE677A67EEA74A9FED317A9FEDD8
:10062000315ADFED316AA4EE875A67EEA43AE4EE60
:10063000856AB7EE006AE3EEA67AB6EE007A36EE89
:10064000676AB8EE005A67EE857A26EE077AB7EE4B
:10065000005AC5EE256A0023836143610362C361CA
:1006600080ED044A26EE877A26EE866A66EEA77A41
:1006700080ED095A80ED007A80ED016A80ED027A02
:10068000C0ED037A7047DFED1B6A36EEC77A68E784
:10069000DFED197AB6EE007AB7EE006AD7E7B7EE6B
:1006A000004AF0EE445A78E79FED0C7AF4EEC77AF0
:1006B000F1EE10FA44BF9FED067A77EE677AAAE76B
:1006C00027D4D2360024F448DB0FC940E4CB1641CE
:1006D000DB0F49C0E4CB16C1DB0FC93FDB0FC9BF3D
:1006E00092E741B99730083C15A82ABEF304353F7C
:1006F00000247448DB0F4940000000009FED2E7A73
:1007000070EE077AFDEEE76A16EE903A2033402B42
:100710004FD8B4EEC70AF1EE10FA0CDD9FED276A50
:10072000DFED276AB0EE677AB4EEE67AF1EE10FA02
:1007300077EEC67AF6DC9FED237AF4EEC77AF1EE17
:1007400010FA0CD59FED1D6ADFED1F6AB0EE677AD7
:10075000B4EEE67AF1EE10FA77EE867AF6D49FEDF3
:10076000167AF4EEC77AF1EE10FA1DDC9FED177AD7
:10077000F4EEC77AF1EE10FA44BF9FED127A77EEED
:10078000677A27EEA76ADFED125ADFED126A9FED56
:10079000127AE6EE256A67EE865AA6EE267AE5EE2E
:1007A000877AB0EE670A70479FED0C7A77EE677A2A
:1007B000E7E79FED0B0A7047DB0FC93FDB0FC9402E
:1007C000E4CB1641DB0F49C0E4CB16C1DB0FC9BF38
:1007D00092E741B99730083C15A82ABEDB0F494083
:1007E00000000000F0EEC07AB0EEE07AB4EEE77AF6
:1007F000F1EE10FAB4BFB0EE676AB0EE476AB5EE3C
:10080000406AF1EE10FA46D0B4EEE77AF1EE10FA53
:100810008CBFF0EE675AF0EE475AC5EE866ADFED00
:100820001F2ADFED1F3ADFED1F4A9FED1F5A9FED94
:100830001F3A9FED1F4ADFED1F5AE6EEE23AA6EEA1
:10084000834AE6EEA34AB7EE006AA6EEA45AA6EEE5
:10085000846AE6EE855AC5EE866AB4EEE77AF1EE72
:1008600010FA48BFDFED147AF5EEC00A48BF77EE04
:10087000E66AF1EE10FA48BFDFED107AB5EEC00A75
:1008800048BF77EEE66AF1EE10FA48BFF1EE666A0D
:10089000B0EE660A7047DFED076ADEE739094E3DC4
:1008A000E3B59E3E88FA163E45FE7F3F99FB243F06
:1008B00069A2163EA7DFA834DB0FC93FDB0F494012
:1008C00090ED005A9FED4C0A35EE000A08B5FDEE9A
:1008D000C07A17EE903A2033402B7BD8FFF780F890
:1008E000F0EE403AFDEEC57A17EE903A2033402BF9
:1008F0007FD8B0EE450AFFF773F8B0EE405AD0ED5E
:10090000014A9FED3D0A34EE800AFDEEC07A17EEF3
:10091000903A2033402B69D8FFF762F8F0EE405A46
:10092000FDEEE47A17EE903A2033402B5BD8B0EE20
:10093000640AFFF755F8F0EE404A90ED023A9FED59
:100940002E0A33EE000AFDEEC07A17EE903A2033FD
:10095000402B45D8FFF744F8B0EE404AFDEEC37A8D
:1009600017EE903A2033402B37D8B0EE430AFFF70A
:1009700037F8F0EE407A24EE233A27EEA36A24EE0D
:10098000057A67EE856AB0EE462AF0EE432AA7EEB6
:10099000242AE6EEE42AA6EE247AE3EE646A24EE44
:1009A000254A65EEE77A25EE655A65EEA35A81ED94
:1009B000004AC1ED017AC1ED024A81ED032AC1ED81
:1009C000042A81ED055AC1ED066A81ED077AC1ED71
:1009D000085A08BDDFED093A84E7DFED087ACAE777
:1009E0009FED064ABAE7DFED054AA6E7DFED035AB9
:1009F00096E79FED025A82E7DB0FC93F0000000037
:100A00002DE9F04389B0541C03941478002C00F0B5
:100A100007810025074688461E46A94609E021466B
:100A20003846C047039A0135531C03931478002CB1
:100A30003DD0252CF3D1931CCDE9033950783028D3
:100A400000F09480A0F13003DBB2092B4FF00004DA
:100A500040F297806C2838D0782822D857282AD995
:100A6000A0F15803202B1CD8DFE803F0B41B1B1B9C
:100A70001B1B1B1B1B1B1B959D1B1B1B1B1B1B1BCA
:100A80001B1BAF1B1B1B1B111BA71B1BB40056F80A
:100A9000043B049A0093002341463846FFF74EF882
:100AA0000544039A531C03931478002CC1D12846A3
:100AB00009B0BDE8F0830028F9D02528F1D125211F
:100AC0003846C0470135039AAEE7039B5A1C039290
:100AD00019787829A8D8572958D9A1F15803202B7B
:100AE000A2D801A050F823F0ED0B0108290A010853
:100AF000290A0108290A0108290A0108290A010806
:100B0000290A0108290A0108290A0108290A0108F5
:100B1000290A0108970B0108050C0108290A010898
:100B2000290A0108290A0108290A0108290A0108D5
:100B3000290A0108290A0108290A0108290A0108C5
:100B4000CD0B0108290A0108290A0108290A010810
:100B5000290A01088F0A0108290A0108110C010855
:100B6000290A0108290A0108ED0B0108D31C039387
:100B70009078A0F13003DBB2092B4FF001043FF66F
:100B800069AF04AA03A946F09DF963E700298ED056
:100B9000252994D048E756F8041B3846C9B2C04707
:100BA0000135039A40E756F8040B05A9FFF75CF8F6
:100BB00005AB0093049A23466EE756F8040B05AB89
:100BC00000220A21FFF708F8F2E7039A56F8043BDF
:100BD0001D6029E7A0F15802B2FA82F256F8040B20
:100BE000520905AB1021FEF7F7FFE1E7A1F158022A
:100BF000B2FA82F256F8040B520905AB1021FEF747
:100C0000EBFFD5E756F8040B05A9FFF72DF8CFE762
:100C100056F8040B05AB00220A21FEF7DDFFC7E7FB
:100C2000254644E773B5144C01920646D4F8880073
:100C30000D46C0B11149FFF7F5FAD4F888003146E6
:100C4000FFF7F0FA0E49D4F88800FFF7EBFA0D49E8
:100C5000019BD4F888002A46FFF7D2FE0A49D4F84F
:100C60008800FFF7DFFA94F88C3013B1012384F881
:100C70008D3002B070BD00BF585F002068A4060828
:100C800073A806082102010875A406080EB400B571
:100C900084B005AB019053F8042B0649039301A8D7
:100CA000FFF7AEFE019B00221A7004B05DF804EB62
:100CB00003B07047BDFB00082DE9F043002483B06A
:100CC0000646048021463046013437F0EBFD082CFF
:100CD000F8D10023DFF8688086F8EA30C6F8EC30F7
:100CE000C6F8F030C6F8F430C6F8F8301F46FC36C7
:100CF00099463A46414601A8FFF7C8FF3546032406
:100D000001AA12F8013B6BB1013C05F8013BF8D197
:100D10000137082F85F8009006F10406E9D103B0E9
:100D2000BDE8F083284622462021254401374DF0B6
:100D300086FC082F85F8009006F10406D9D1EEE76D
:100D4000185F0608F7B5114E07463046002300F835
:100D50008E3F0C460E4B0F49002F08BF1946154613
:100D60004DF075FC0C4F04EB45058E36AC4202D1BC
:100D70000A4803B0F0BD394634F8022B6846FFF745
:100D800085FF694630464DF062FCEFE7585F002072
:100D900082A4060879A406088BA40608E65F002052
:100DA000F7B50C4E0C4F002306F8BF3F044600EB8E
:100DB0004105AC4202D1094803B0F0BD394634F8D0
:100DC000022B6846FFF762FF694630464DF03FFC54
:100DD000EFE700BF585F0020B6A5060817600020A7
:100DE000F8B5084F4E1E054601F11F0416F8012FF5
:100DF00028463946FFF74AFFA64205F10205F5D11C
:100E0000F8BD00BF90A4060803685A1C0260197060
:100E10000368090A5A1C026019707047026811467B
:100E2000531C036011F802CB0160D31C517803609E
:100E300093781B0443EA0123111D0160D07843EA33
:100E40000C0343EA00607047A0F13003092B07D977
:100E500020F02000413819288CBF00200120704765
:100E600001207047303809288CBF002001207047CE
:100E7000413819288CBF002001207047613819289B
:100E80008CBF002001207047202805D00938042895
:100E90008CBF00200120704701207047A0F1410362
:100EA000192B98BF20307047A0F16103192B98BF10
:100EB0002038704710B500F100440246013C04E0C0
:100EC000B3EB0E0015D1A24214D012F8013BA3F1EE
:100ED0004100192811F8010BA0F1410C98BF2033F3
:100EE000BCF1190F00F1200EEAD91B1A04D1002819
:100EF000E9D110BD002010BD184610BD02B310B5D9
:100F00008446841804E0B3EB0E0014D1A44513D03A
:100F10001CF8013B11F8010BA3F14102192AA0F1C1
:100F2000410298BF2033192A00F1200EEBD91B1A79
:100F300004D10028EAD110BD002010BD184610BD14
:100F40001046704770B5044608460D464BF084F8CD
:100F5000064602E014F8013F43B1204632462946D6
:100F6000FFF7CCFF0028F5D1204670BD1C46204677
:100F700070BD38B507490546FFF7E4FF0649041E72
:100F8000284618BF0124FFF7DDFF08B144F0020432
:100F9000204638BD95A4060887BA06082DE9F04119
:100FA000044686469EF800C0BCF1200F7046ACF1A6
:100FB00009050EF1010EF5D0042DF3D9BCF12B0F6C
:100FC0005BD0BCF12D0F3BD1102A4FF0010600F190
:100FD000010E58D19EF800C0BCF1300F5FD04FF029
:100FE00010086FF070450F2742460EF1010E0020E9
:100FF0000DE0ACF1300C5FFA8CFC94450FDA8542C1
:1010000074462DD32AD008FB00C01EF801CBBCF1DA
:10101000390FEED94CF0200CBCF1600F0BD801B1A8
:101020000C600EB323B1B0F1004F28BF4FF0004069
:101030004042BDE8F081ACF1570C5FFA8CFCDCE774
:10104000102A864649D04FF0FF35B5FBF2F502FB7A
:1010500005F7FF43FFB290460026C6E76745D2D2A8
:101060001E404FF0FF30D0E7002BE2D06FF000437E
:10107000984228BF1846BDE8F081102A4FF00006BC
:1010800000F1010EA6D04FF0FF35B5FBF2F502FBE3
:1010900005F7FF4390F801C0FFB29046A5E79EF820
:1010A00001C0ACF1410019280EF10104624601D8DB
:1010B0000CF12002782A4FF0100805D0A6466FF0F8
:1010C00070450F27424690E79EF802C06FF07045CA
:1010D0000EF1020E0F27424687E700267AE700BF8F
:1010E00001230A22002159E770B50D461446FFF787
:1010F000ABF80646A0B1FFF7F3FF40F63403984281
:10110000A8BF1846B0F5617FB8BF4FF46170A0F575
:1011100061731920B3FBF0F32B7023780133237034
:101120003046FFF791F80646A0B1FFF7D9FF40F629
:1011300034039842A8BF1846B0F5617FB8BF4FF49A
:101140006170A0F561731920B3FBF0F36B70237825
:1011500001332370304670BD10B40288C378174C39
:10116000A2F5FA6202F0030140F2B55C9208013B7D
:101170000CFB0233827801EB4101013A02EB810260
:1011800004EB420102798C8F4179234403EB430342
:1011900002EBC30384790A4A0089C3EB031301EB12
:1011A0008303C3EB0313224402EB830200214FF4B9
:1011B0007A73C2FB03015DF8044B7047A4F905087C
:1011C00080436D382DE9F04117461E4605464FF421
:1011D0007A720023384631464BF002FC4349444AB8
:1011E000014482FB0143C8170B44C0EB631382FB2D
:1011F00003021A44D8173F4CC0EB621284FB02046E
:101200004FEAE27C3C48CCEBA40C80FB0C404FEA5C
:10121000EC74C4EBE010C3EB0314A1EB8401A971DF
:10122000C2EB0211A3EB81036B710CEB4C03A2EB3D
:10123000C30240F2B55303FB10CCBCF5896F2A7191
:101240004FEA800044DA40F2DA239C4547DCBCF5E3
:10125000B77FB4BF00220122284B02EB420103EB0F
:10126000C1034FEA4208B3F8523091B2244C08EB64
:10127000020E04EBCE0416344FF00B0E01E034F8EE
:10128000023D63451FDDBEF1010EF8D11B4B424408
:1012900003EBC2024FF0010E938F85F802E000F5D8
:1012A000FA600CF1010C0844ACEB030C288085F8C3
:1012B00003C04FF47A720023384631464BF090FB5E
:1012C0002A81BDE8F0810EF1010E5FFA8EFEE4E79F
:1012D000032140F296530A464FF00608C6E7022162
:1012E00040F229430A464FF00408BFE780BC92C78A
:1012F00089888888ABAAAA2A73B06D16A4F9050854
:10130000E0F9050808B50C4BD3E93A2352EA030C7F
:1013100009D1002340F2011242808380837103804F
:101320000381184608BD054909688A1843F100037E
:10133000FFF748FF012008BD585F00209C200020D7
:1013400090422DE9F0410B46044615460AD2B0FB07
:10135000F5F6134A05FB16441846135D00F8013BE9
:10136000BDE8F081B0FBF2F69642B6FBF2F706D28A
:101370000B4A05FB1767D15D03F8011BEAE7BA4288
:10138000B7FBF2F807D9064A05FB187812F80810DF
:1013900003F8011BEDE74046FFF7D2FF0346F2E7F3
:1013A000205F060830B5874CB4F8FC33B4F800046D
:1013B000B4F80214B4F80424B3F57A7F84BF4FF470
:1013C0007A73A4F8FC33B4F8FE33B3F57A7F84BFA4
:1013D0004FF47A73A4F8FE33B0F57A7F84BF4FF4EC
:1013E0007A70A4F80004B1F57A7F88BF0021B4F8C0
:1013F000063488BFA4F80214B2F57A7F84BF4FF494
:101400007A72A4F80424B3F57A7F84BF0023A4F889
:10141000063488429CBF0021A4F800149A4298BF69
:101420000023B4F8122498BFA4F80434B4F8143498
:101430009A4284BF0023A4F81234634B1B8883B004
:101440002BB3627B614D012A48D9AA78062A97BF3F
:101450005F499FED607A01EB820191ED277A29794E
:10146000002940F08A8094F81C1407EE903A06EEAA
:10147000901AF8EEE77AB8EEE66AAB79C6EE276A1C
:10148000002B72D1B4EEE67AF1EE10FA37DC637A13
:10149000032B14D8504AC3EB031302EB4302237A05
:1014A000C4F82424032B12D84C4A03EB830103EB2A
:1014B000C10302EB8303C4F8283403B030BD00231A
:1014C0006372237A444AC4F82424032BECD9434B97
:1014D000C4F828340022227203B030BDAA79002A51
:1014E000B3D0AA78072A2AD0B3F57A6FAED994F888
:1014F0001C140229B8BF022184F81C14A6E767EE69
:10150000277ABCEEE77A8DED017A9DF8042007EE8C
:10151000102AB8EEC77AF4EEC77AF1EE10FAC4BF1B
:101520000132D2B2002A3CD0102AA8BF1022D2B277
:101530008A42134638BF0B4684F81C34A7E70622BC
:10154000B3F57A6FAA702ED82A79002A9FD194F821
:101550001C1407EE903A07EE101AF8EEE77AB8EE90
:10156000C76A9FED1F7AC6EE276A37EE077AB4EE98
:10157000E67AF1EE10FA8ADDC1E7042A02D8002AE1
:1015800085D002E0053A032A81D9B7EE000A80EE41
:10159000070A4CF079FA2B88984228BF1846288011
:1015A00075E70122C3E794F81C242979022AB8BF01
:1015B000022284F81C2400297FF469AF9FED087A89
:1015C00051E700BF585F0020C00A00109C27002090
:1015D000A4F905086F12033848600020C06000209D
:1015E00017B7D1382DE9F04FAD4E85B096F82C34B1
:1015F000A3F11702022A00AF00F2CC82A94BBB6014
:10160000DFF8C09296F83C14DFF8BCB2A64D09F1A1
:101610006C0A4C464FF0000834E010F0010C4ED13B
:10162000142A00F0B3824308820802F0333203F038
:1016300077331344C20802F01132C31A9B1A03EB2A
:10164000131303F00F33ABFB03E2D209C2EB022208
:101650009A1A830302D5012A00F09882012A0ED932
:10166000082A00F29382BCF1000F01D0284206D173
:10167000F96049F067FFF968002800F087820C34B0
:10168000544521D094F904202068A2F11E03DBB256
:10169000012BC2D8A379022BA8BF0223A371E3793F
:1016A000022BA8BF0223E371237A022B20F0410012
:1016B000A8BF0223206023724FF0000CB3E708F1AB
:1016C00001085FFA88F8AEE708F1FF38B8F1020FB9
:1016D00000F25C820024022086F8DC4411F074F9E8
:1016E00096F8E034022B00F0ED82002800F05983D8
:1016F0006E4B96F8AD8503F5247B4FF47A7E4FF060
:10170000000C5A88B2F57A7FB3F8462088BFA3F858
:1017100002E0B2F57A7F9A8888BFA3F846E0B2F576
:101720007A7FDA8888BFA3F804E09988B2F57A7FD7
:1017300084BF0022A3F806C09142B3F85A10B3F850
:101740005C2098BFA3F804C0914293F86B2088BF37
:10175000A3F85AC0013A632A84BF642283F86B203D
:1017600093F86C200132D2B2092A88BF83F86CC08A
:1017700003F16600194600228D7A10F8014B013200
:10178000A54238BF00F801CC032A01F10601F3D1CC
:10179000B8F1010F18BF83F885C0A4339B45B0D1C1
:1017A000434B9B78042B00F0D5823BB9404A138809
:1017B000B3F5F07F84BF4FF4F0731380FFF7F2FDB1
:1017C0003C4896F8C015FEF725FC96F8DF1510305A
:1017D000FEF720FC96F8ED150E30FEF71BFCB6F870
:1017E000FA25B6F8F8351343B6F8FC2513431BB2B7
:1017F00013B10123A6F8FE35D6F89C352E4A1A40BF
:10180000002A00F0E482DA0700F14E825D0440F124
:10181000DF812A49D6F8A0250B400A40C6F89C353E
:10182000C6F8A02513F4004200F02182002286F8B9
:10183000432486F85324D90440F1238296F80B36CA
:10184000DFF87CB0022B04BF012386F80B360BF1C6
:1018500078045B4602E00633A3420CD01A78072ACC
:10186000F9D19978DA78914202D35A79002AF2D0E4
:10187000072022F00FFF00234FF4806086F8DC344D
:1018800011F0A2F8002800F07F820D4DA84698F8CC
:10189000051031B398F8000008B35B4619E000BFAB
:1018A000585F0020A4F90508BC020200C0600020B7
:1018B0009C2700202865002009600002F6DFFFFD5C
:1018C00068650020C46300208180808006339C42CC
:1018D00007D01A788A42F9D15A79002AF6D022F034
:1018E000D9FE08F106084445D1D1BB4B93F802B0AC
:1018F000BBF1080F00F0048296F8AD3596F8F92395
:10190000A3F10103B3FA83F35B0986F8883696F8EE
:10191000AE35A3F10103B3FA83F3032A4FEA53135D
:1019200088BF002286F88C36D6F8A03588BF86F8A6
:10193000F923AA4AC3F3C03186F88A1603EA0201E2
:10194000D6F89C35C6F8A0151340B27DC6F89C3574
:10195000002A00F0E081B6F8A036002B40F0E781C5
:10196000D6F8A43613F07F4F1CBF0023C6F8A43668
:10197000D6F8AC3623F4007323F002031BB140F217
:101980000223C6F8AC3696F8A836013B042B84BF78
:10199000012386F8A836ABF1050B914BBBF1030F81
:1019A00093F8901540F25A8111B30023FB608A4BE3
:1019B0007C606FF00702A2EB0308444603F1080BBA
:1019C000884604E004EB0B03984540F21D811BF8A8
:1019D000010B0028F6D00CF0B1F90028F2D0837981
:1019E0009B07EFD5FA687C680123002A40F012813A
:1019F000794B9B7913B1784A00239371B6F8B636C8
:101A000013F00C0F03D1C3F30313022B03D94FF4CC
:101A10002063A6F8B636B6F8B83613F00C0F03D12B
:101A2000C3F30313022B03D940F60123A6F8B836FB
:101A300096F8313796F825279A4296F8243705D933
:101A4000002286F8252753B1A6F8282796F83027D4
:101A50009A4204D2002386F82437A6F8283796F84D
:101A60001A3896F826275F49FC609A4288BF0023FF
:101A7000BC6888BF86F8263701F1780B11F8013C65
:101A800003EB430323444FF0030893F870E293F809
:101A900071C293F872020B461A787245A8BF72465B
:101AA00003F8012B5A796245A8BF62465A719A78A9
:101AB0008242A8BF0246B8F101089A70ECD11E31EB
:101AC0008B45DBD1D6F86424FC68002A00F039810C
:101AD000002001212B78282B07D16B78043301FAE1
:101AE00003F313421CBF9A4301200635AC42F1D1E7
:101AF00008B1C6F864243C4D05F108042B4613F8E0
:101B0000012B072A00F293809C42F8D1EB4688B063
:101B10006B46FF21184620224CF091FD32490346C6
:101B200011F8012B53F82200013040F087808C42DD
:101B300043F82220F4D1B6F8A625B6F8A4359A4287
:101B4000DD4602D3294BC6F8A435FF23284986F881
:101B50004C3899F90430142B05D0D9F8002031EA1B
:101B6000020200F0F48009F10C09D145F1D1214ABB
:101B70005379012B04D0022B04D11F4B1B790BB9D5
:101B8000002353711437BD46BDE8F08F1B4810F099
:101B9000CFFE9FE51A4ABA601146DA0001EBC30393
:101BA00093F8B81021B1D3F8BC30002B00F0E880D6
:101BB000BB68134493F8B920002A3FF421AD93F891
:101BC0009831002B7FF41CAD182386F82C3417E5D0
:101BD0001C0772D50B491DE69C270020FEDDDDFDAC
:101BE000C00A00104B600020AF270020AE014A0160
:101BF00001000200A02F0020A82F0020C4630020B5
:101C0000A4F90508FE9FFFFDFA687C680023002AFE
:101C10003FF4EEAE73494A7C002A7FF4EFAE4A7976
:101C2000012A3FF4E5AE002B7FF4E2AEE6E6EB4698
:101C300088B02022FF2168464CF001FD05F8018B99
:101C400008F10108B8F1080F3FF475AF05F8018BF2
:101C500008F10108B8F1080FF0D16CE7614A0023E0
:101C60001371002900F0AA800123FB609FE696F81B
:101C7000431400293FF4DFADD90486F853243FF51F
:101C8000DDAD1A067FF5DAAD96F82C14182906D8C2
:101C9000554B01228A401340002B7FF4CFADDFF873
:101CA0005CB10BF17804E6E55049D6F8A0250B406D
:101CB0000A40C6F89C35C6F8A02598047FF5B2AD59
:101CC0004B49A7E500283FF413AD4A4B96F82D1574
:101CD00090F904504FF0FF0C03F16C0093F90820C9
:101CE000AA4204D1013983F808C0C9B201240C33D7
:101CF0008342F3D1002C3FF4FBAC86F82D15F7E4BA
:101D00001A469B79002B3FF4F7AD537C012B04BF9F
:101D100002235374F0E5384A1343C6F89C35B6F8ED
:101D2000A0361143C6F8A015002B3FF419AE96F863
:101D30009C060CF003F800287FF412AEA6F8A0066B
:101D40000EE6282022F0A6FCD6F86424C0E686F829
:101D50004C380CE7D6F89C35224A23F48053C6F859
:101D60009C35D6F8A03523F48053C6F8A035538CA3
:101D7000B3F57A7FBFF422AD4FF47A7353841DE537
:101D8000172386F82C3413E7D6F89C3523F000632C
:101D9000C6F89C35D6F8A03523F00063C6F8A03508
:101DA00073E5D6F89C25D6F8A03522F0800223F002
:101DB0008003C6F89C25C6F8A03599E4537C002B17
:101DC0007FF41CAE5379012B7FF418AE10E6D6F8E1
:101DD000A02543F0080342F00802C6F89C35C6F877
:101DE000A02510E59C27002000410001F79FFFFD82
:101DF000F6BFFFFD88640020200415006865002000
:101E00002DE9F04F784F794BD7F85C2802F2DC527D
:101E1000C7F85C28764A934283B080F0E18003F1F2
:101E20001C059B46734B744E4FF0010A03F10208E8
:101E3000704B5A88002A00F0BC8008EB0203B342C2
:101E400080F0B780444608E01A881C461344002AF4
:101E500000F0AF80B34280F0AC80052A40F2A98048
:101E600035F81C2C6188C2F30B029142ECD16279E7
:101E70009207E9D1238855F8141C94F80490019333
:101E80005846FEF7B9FA35F81C2CB9EB123F00F0B2
:101E900098804FF0000A35F8181C55F8140CC1F35F
:101EA0000B0146F025FD55F8043C1860504B0BF132
:101EB0001C0B9B4505F11C05BAD3D7F89C35C7F818
:101EC000A035FFF78FFB3B7A4C4D4D4C03EB830263
:101ED00003EBC2037A7AA5F17801C2EB021201EB9F
:101EE000420205EB8303C7F82424C7F8283421F005
:101EF000E9FD4FF0FF33D7F8280463602DF050FB65
:101F000022F01CFC05F5956305F5A46102E006339B
:101F10008B4260D01A78002AF9D19D78D878854212
:101F200002D358790028F2D097F80836227203EBD2
:101F3000830303EB83039B00632BB7F80C26314923
:101F4000D8BF6423C7F85438642303FB02F2632A22
:101F5000D6BF1A46C7F85828C7F85838C7F87028A7
:101F60000023294AC7F85C38C7F86038C7F86438D6
:101F7000C7F86838C7F86C38A7F8743887F8763827
:101F8000C1F814272EF0D0FCB7F8780897F87A1823
:101F900023F056FA39F04AFB17F0CAFE1B4A1268C2
:101FA000C7F85C280123504687F8753803B0BDE8B0
:101FB000F08F55F8141C5846FEF71EFA4FF0000A31
:101FC00069E7019BA11D9A1F5846FDF7CFFB00282A
:101FD0007FF461AF5DE7FA7D003A18BF0122A3E705
:101FE0004FF0010A69E700BF585F002090EC060837
:101FF0006CF506080040000800800008C060002062
:1020000010050020C00A0010506500209C20002010
:102010001C4B0122032870B51B4D83F81C27064674
:102020001ED9711CC9B249004029184A28BF402155
:10203000002302244FF0140ED454023302EB030C9D
:1020400099420CF801ECF7D8FF2E08BF0221294471
:10205000FF2381F87C38BDE870400E2010F0DABE16
:1020600000EB800005F5B47306EBC00003EB8000C5
:10207000C5F828042E722DF093FA23F097FD23F073
:102080006BFECEE7C00A0010585F0020D467002026
:10209000054BD3F8C028012142F4001283F8BD1883
:1020A000C3F8C028704700BF585F0020F8B5046827
:1020B000C4F30D0406460F460CB335683F6843F081
:1020C0005FF9092840F08780444C236923F440736A
:1020D0002361236943F400732361236943F00103FF
:1020E00023612F6043F04CF92369092823F0010391
:1020F000236170D1336804333360002034E0384BFF
:10210000384A93422AD302F58042934225D302F5FE
:102110008042934229D3344A934228D902F580322F
:10212000934226D902F50032934224D902F50032B7
:10213000934222D902F50032934220D902F50032AF
:1021400093421ED902F5802293421CD9B3F1016F4C
:102150001BD348F04FFB47F0D9FD082443F010F99A
:10216000092814D04FF0FF30F8BD1024F6E71824EA
:10217000F4E72024F2E72824F0E73024EEE73824BF
:10218000ECE74024EAE74824E8E75824E6E7134D63
:102190002B6923F440732B612B6943F400732B618B
:1021A0002B6923F0F8032B612B691C4344F00204D4
:1021B0002C612B6943F480332B6143F0E1F82B69E8
:1021C00023F002032B612B69092823F0F8032B610C
:1021D0003FF473AFC6E76FF00100C5E7003C024073
:1021E0000040000800400008FFFF00082DE9F04112
:1021F000574F3B78B12B8AB06FD1FDF735FE80F099
:102200000104E4B2534B544DB3F87F32534EADF852
:10221000003004F00104B54261D3002C00F0968038
:102220001022002106A84CF00AFA4D4B0497DB1B44
:1022300005934C4B1A69002A04DA4B4A5A6002F1A2
:1022400088325A6001228DF82420F322DA60694630
:10225000022204A80025089549F0FEFB02226946E7
:102260004FF6FF70FDF75EFB3B4F0446B74243D38A
:10227000022201A904A80025ADF8045049F0ECFBA6
:10228000022201A92046FDF74DFB40BAC043ADF83C
:102290000800022204A802A949F0DEFB079868B1F1
:1022A00006ABC0F10402294618444CF0C8F908985E
:1022B00018B906A904A8FFF7F9FE08909DF8243084
:1022C000089823B1274A136943F000431361B0FA19
:1022D00080F040090AB0BDE8F081012492E7A988A6
:1022E000A868C1F30B0146F003FBAB691B681C3502
:1022F000834218BF01248EE7B7F804808DF80D5093
:10230000C8F30B0808F10603ADF808303B88C3F3A7
:102310000B02ADF80A201B0B062202A904A88DF8B7
:102320000C3049F099FB062202A92046FDF7FAFA83
:10233000B9680446424604A849F08EFBB9682046B5
:102340004246FDF7EFFA1C3704468FE70120C1E74C
:1023500000400008A4F9050890EC06086CF5060892
:1023600000800008003C02402301674510B5194C6D
:10237000FFF738F9D4F85C38012203F2DC53C4F8D3
:102380005C3884F8C428FFF731FF10B9FFF72EFF3F
:1023900050B1114B1B78B12B02D1FDF765FD58B937
:1023A00048F028FA47F0B2FCFFF720FF0028F0D1F0
:1023B00048F020FA47F0AAFC084A0023116884F884
:1023C000C4380122C4F85C1884F8752884F8C5382C
:1023D00010BD00BF585F0020004000089C20002076
:1023E00010B50B4A0B4C012382F81C37A375FFF77D
:1023F000BDFFFFF705FD41F20242FF23A4F87C2850
:1024000084F87E380E20BDE8104010F003BD00BFF8
:10241000C00A0010585F002090F88730DFED6A5A3C
:1024200003EE903A90F88B3006EE103A90F889302F
:1024300004EE103A90F88A30F8EEE33A04EE903A5F
:1024400090F88D3063EEA57AB8EEC66A03EE903A46
:1024500026EE256AB8EEC44AF8EEE44AF8EEE33A0E
:1024600026EE276A24EE254A64EEA54A63EEA53AD5
:10247000F0B5564D24EE064A64EEA74A63EEA73A3D
:1024800000210626F7EE002AA5F10C0C00F1660EDD
:1024900006FB01F2B7EE005AAC1890F886700244C1
:1024A000F0EE456A15E0012904F1060402F1060286
:1024B000EED190F8883007EE903A90F8903006EE22
:1024C000903AF8EEE77AF8EEE66A27EEA55A66EE5D
:1024D000A56A237807EE103A66EE867AB8EEC77AD8
:1024E00027EE277AFDEEC77A17EE903AFA2BA8BFAF
:1024F000FA2323EAE3731372637807EE103A66EE69
:10250000847AB8EEC77A27EE277AFDEEC77A17EEFF
:10251000903AFA2BA8BFFA2323EAE37353725CF8CC
:10252000213007EE903A002BF8EEE77A49DDA378E8
:1025300007EE103AB8EE477A90F88C3037EE677AAB
:1025400003EE103A87EE272AB8EEC33AB0EE627A6D
:1025500023EE253AA2EE037A64EEA77A66EEA36A2A
:1025600067EE857A27EE877AFDEEE77ABDEEC77AC9
:1025700017EE103AFA2BA8BFFA2323EAE3739372FB
:1025800017EE903AFA2BA8BFFA2323EAE3730EF86A
:102590000130A38807EE903AF8EEE77A013167EE52
:1025A000A67AFDEEE77A17EE903AB3F57A7FA8BFE8
:1025B0004FF47A7323EAE3738F429381BFF673AFCC
:1025C000F0BDB7EE007AC7E70AD7233C60FE0508E6
:1025D00090F88E306BB3B0F85A308BB190F88F20F2
:1025E00002EB82036421C3EB0313B3FBF1F3A0F806
:1025F0005A30962312FB03F3B3FBF1F3A0F85C30DF
:1026000043884BB190F88F3003EB8303C3EB031384
:102610006422B3FBF2F34380B0F846304BB190F83C
:102620008F30962213FB02F36422B3FBF2F3A0F87F
:102630004630704790F821304BB3438B83B190F80C
:102640002230FA2213FB02F203EB8303B3F57A7F05
:10265000A8BF4FF47A7364218383B2FBF1F2428303
:10266000838843B190F82230FA2213FB02F36422EC
:10267000B3FBF2F38380C3884BB190F8223003EBB5
:102680008303B3F57A7FA8BF4FF47A73C380704792
:1026900070B50B4C002504F5247694F8863013B100
:1026A0002046FFF7B9FE2046FFF792FF013530467E
:1026B000FFF7C0FF042D04F1A404EED170BD00BFEC
:1026C000C0600020034BD3F8C80D08B106F0B6BCBB
:1026D000704700BF585F002008B50B460549024609
:1026E000D1F8C80D28B10449FEF78AF9BDE80840C1
:1026F000E8E708BD585F002021020108024B0146AF
:10270000D3F8C80DFDF78EBD585F002008B504460C
:102710000848FFF7F3FFFFF7D5FF074BD3F880001A
:1027200010F0F6FA0AF084FA012C01D147F0EEFA23
:10273000F9F70EFD9DA40608585F00200048DDE76C
:102740000EB006080CB4C30607B500D561B90498ED
:1027500005A90191FFF7C0FFFFF7F0FF012003B0CB
:102760005DF804EB02B070470020F8E708B5FFF70A
:10277000C5FFBDE80840E1E710B504460348FFF790
:10278000BDFF2046BDE81040F0E700BFA9A4060841
:1027900008B50948FFF7F0FFFFF794FF074B002447
:1027A00083F8CC4DC3F8CC4E83F8D04E23F0A4FB75
:1027B0002046FFF7ABFF00BFAEA40608585F00201D
:1027C000034B0146D3F8C80D08B106F023BC70478F
:1027D000585F00200CB407B510F020000BD079B979
:1027E0002320FFF7EDFF049805A90191FFF774FF7F
:1027F000FFF7A4FF012003B05DF804EB02B07047BF
:102800000020F8E70FB407B504A951F8040B0191B3
:10281000FFF762FF03B05DF804EB04B0704730B51A
:102820002B4885B0FFF76AFF2A4B1B7923B92A484A
:1028300005B0BDE8304099E7FBF7B4FB08B927487D
:10284000F6E7FBF7C7FB08B92548F1E7254B1B68FE
:10285000DB6998470028F7D0FBF79CFB0268037DF3
:1028600081790446407C0290207C0190608A00902F
:1028700052081D48FFF7C6FFE51D0C3415F8010B83
:10288000FFF79EFFA542F9D1184C1948FFF736FF14
:102890006378022B06D007D9032B10D11548FFF718
:1028A0002DFF0CE01448FAE704F580541348FFF7B5
:1028B00025FF94F8E437022B05D0032B05D005B093
:1028C000BDE830403AE70E48E9E70E48E7E700BFC9
:1028D000D5A40608A82F0020DFA40608EEA4060849
:1028E000FCA40608982000200BA5060868300020EC
:1028F00039A5060849A506084FA506085CA50608DF
:1029000062A506087BA506080FB407B504A951F80F
:10291000040B0191FFF7E0FEFFF710FF03B05DF835
:1029200004EB04B070472DE9F041037903F0E002B5
:10293000402A50D004D85AB1202A29D0BDE8F081CD
:10294000602A4BD0802AF9D182794179254812E05A
:1029500003F00703052B16D8DFE803F01015101558
:102960000309D0F805102048BDE8F041CCE7D0F8C5
:10297000052051421D48BDE8F041C5E7B0F80720E9
:10298000B0F80510F6E7B0F90720B0F90510F1E747
:102990004679174D174805EBC605FFF7AFFE95F8CA
:1029A000D47400240123A74202D8BDE8F041C5E653
:1029B000D5F8D06456F824204FEA84084AB113B9F8
:1029C0000D48FFF79BFE56F808100C48FFF71AFF5A
:1029D00000230134E7E741790948C5E7BDE8F04144
:1029E000084891E7DCA506088DA50608A3A50608FA
:1029F000A4F90508BAA50608BCA80608D3B80608B5
:102A0000CBA50608F3A506080249034801F5216194
:102A10000EC979E70070FF1F0BA6060810B57521D7
:102A200004462EF055FA01460948FFF76DFF1A21BA
:102A300020462EF04DFA01460648FFF765FF1B21A0
:102A400020462EF045FABDE81040014602485BE7FB
:102A50001FA6060832A6060845A6060838B50C4D7E
:102A600095F8FB0310F0FD0405D10A48FFF74CFF71
:102A70002046FFF7D3FF95F8FB33013B012B06D827
:102A80000548FFF741FFBDE838400120C6E738BDE3
:102A9000585F002058A6060863A606082DE9F04FE7
:102AA000754B76491A68764BB2FBF3F299B08046C3
:102AB0007448FFF7A7FE744BDFF840C20FCBDCF879
:102AC00008700CAD85E80F00704B0793BC08704B85
:102AD000089314F00204C7F3810718AB18BFDCF8A1
:102AE000046003EB870318BFC6F3805653F8301C0D
:102AF000002C00F0BF8018AB03EB860353F8442C86
:102B0000644C6548654D664FDFF8BC91FFF77AFE6F
:102B1000B4F8D22E4FF47A73B2FBF3F103FB112217
:102B20000A20B4F9D43E92B2B2FBF0F25D48FFF74E
:102B3000EBFE5D4A5D495E48FFF764FEFFF7FEFD70
:102B4000A17D5C4A5C4B5D4805EB8101D31AD1F84D
:102B5000B016A288FFF7D8FE5948FFF7CFFD94F8CA
:102B6000D61E5848FFF74EFE5748FFF7C7FD94F8AA
:102B7000D71E5648FFF746FEFFF7E0FD5448FFF723
:102B8000BDFD00210A4694F817340B4113F0010FE4
:102B900001F1010608D012B14846FFF7AFFD3146FA
:102BA0003846FFF72FFE0122072E3146EBD1494E62
:102BB00096F86A1506F5EC7306F13C02012918BF78
:102BC000134693F8DC30032B02D04348FFF71AFE7C
:102BD000424B96F86A15A3F5CE72012918BF134629
:102BE00093F8DC30012B02D13D48FFF70BFE3B4B45
:102BF00096F86A15A3F5CE72012918BF13461B6912
:102C00005B7B012B02D93748FFF7FCFDDFF8F09022
:102C1000FFF794FDD4F8D83E0393002709F1200A6A
:102C200059F8041B00296DD0012303FA07FB039B0D
:102C30001BEA030F1CD01BF01F0F19D02A4B5AF8A8
:102C40002720D85D52F8202037B12848CDE904125A
:102C5000FFF754FDDDE904122548FFF7D3FDBBF172
:102C6000020F05D196F8411A11B12248FFF7CAFDAB
:102C70000137D5E7204A43E79420002076A60608CE
:102C800040420F007BA606084400060898A60608E6
:102C90009DA60608585F0020A2A60608A4F905080C
:102CA00052A70608AAA60608F0FF001000080000B8
:102CB000CBA606080080000800400008EFA6060822
:102CC0001EA7060830A7060838A706083AA7060870
:102CD00042A70608C00A00105BA70608980C00105F
:102CE00063A7060868A7060858050020BCA80608C0
:102CF00070A7060876A7060810B00608003802403C
:102D00005C000608FFF71AFD94F8221DD4F8242D64
:102D10007B48137A527A05EB8101D1F8EC16FFF764
:102D2000F3FD78497848FFF76DFD78497848FFF75B
:102D300069FDFFF703FD774B774819684FF47A7305
:102D4000B1FBF3F1FFF75EFD09A8FEF7DBFA38B13E
:102D500009A910A848F07CFF704810A9FFF752FDA0
:102D6000FFF7ECFCD4F8642F002A00F0858007EE12
:102D7000902ADFED6B6AB8EEE77AC6EE877AFDEE51
:102D8000E77A17EE903A674FB7F8640558B107EE47
:102D9000900ADFED636AF8EEE77A86EEA77AFDEE39
:102DA000C77A17EE900AD4F8E41E59B107EE901ACC
:102DB000DFED5B6AF8EEE77A86EEA77AFDEEC77A7A
:102DC00017EE901AB6F87C6A642ECDE90001314600
:102DD0005548A8BF6421FFF797FD97F8663597F827
:102DE0006725B7F86815514805EB8303D3F800371A
:102DF000FFF78AFD4E4B4F48198889B2FFF784FDD3
:102E00004D494046FFF70BFD4C48FFF777FCD4F8DF
:102E1000A0351B0660D597F89435032B8CBF484826
:102E20004848FFF76BFC94F8E034022B26D1464863
:102E3000FFF764FC97F89435042B44D84348FFF718
:102E40005DFC97F8A435002B44D005EBC303D3F801
:102E500058173F48FFF7D6FCFFF770FC3D483E4F40
:102E6000FFF74CFCD4F8C0480126002C38D1FFF7FE
:102E700065FC19B0BDE8F08F134684E702200FF01F
:102E8000C5FD064608B93548D2E738F0B5FB96F9D6
:102E9000041005EB80000131D0F814273048FFF70B
:102EA000B1FC94F8E334012B04D12E48FFF726FC43
:102EB0002D48BDE7B3792D4805EB8303D3F81417EC
:102EC000FFF7A0FCF4E794F8E2340BB92848B6E722
:102ED0002848B4E72849BCE72848FFF70FFCBBE7C0
:102EE00094FAA4F3B3FA83F306FA03F205EB83032F
:102EF0003846D3F88C1724EA0204FFF783FCB4E7C2
:102F00007AA706088CA70608ADA70608BBA706087F
:102F1000C1A706089C200020C7A70608E1A706084D
:102F20000024744950700020F4A706083AA8060847
:102F30007824002061A8060810B0060870A80608CA
:102F400076A8060882A8060892A8060899D206085C
:102F5000CFA80608EBA80608DBA8060898A806086C
:102F6000A2A80608B6A80608BBA8060895B20608D7
:102F7000BFA80608E3A406086EA60608DFA8060890
:102F80002DE9F04FDFF8788198F80B3099B0002BDD
:102F900000F098805148524EDFF868B1DFF8689130
:102FA000DFF868A1FFF7E2FB00252F460BA9E8B286
:102FB00017F01AF99DF83430002B53D0139C54B1FC
:102FC00007EE904A9FED470AF8EE677A80EE270AEF
:102FD0004AF05AFD04460B9A29465846FFF712FC60
:102FE000109A002A70D002FB04F04FF47A73B0FB01
:102FF000F3F30993DDF848C0BCF1000F66D00CFB79
:1030000004F142F21073B1FBF3F198F80B30082D84
:1030100018BF7F18002B5BD0179807901598069063
:10302000169805900A2311984FF47A7EB0FBFEFEA5
:103030000998CDF810E0B1FBF3FE03FB1E11CDE9BA
:1030400002E10999B1FBF3F103FB1100CDE9001096
:10305000BCFBF3F321465046FFF756FC0023C6E9BC
:103060000D33B36201351E2D06F140069ED198F84E
:103070000B3023B31C4C1D48D4F8AC25D4F8A8154C
:10308000D2084FF47A73B1FBF3F3D4F8B015FFF71D
:103090003BFC0A221648B7FBF2F102FB1172FFF764
:1030A00033FC144B1B78432B06D1D4F8B425D4F849
:1030B000B8151148FFF728FC0023C4F8B03519B043
:1030C000BDE8F08F0D4866E7099293E761469CE7FB
:1030D00021464846FFF718FCC0E700BF01A90608D3
:1030E000346E00208096184B50700020A8A9060866
:1030F000C8A9060858220020ECA906085FA90608FE
:10310000585F002069A906086FB8060878A9060864
:1031100013B52C48FFF7F2FA2B4B93F85534002BDC
:103120004ED02A4C2A48FFF721FB94F8143B2BB1D0
:1031300094F8163B13B194F8153B83B9254B2648F8
:1031400093ED280A8DED010AFFF7D8FA234B9DED88
:10315000010AB3F8643533BB2148FFF707FBB4F825
:10316000181B2048FFF74EFB94F8143B13B31E487E
:10317000FFF7FCFAB4F81C1B1C48FFF743FB94F85C
:10318000163BCBB11848FFF7F1FAB4F81A1B1848F0
:10319000FFF738FB94F8153B83B1134802B0BDE844
:1031A0001040FFF7E3BA4AF06FFC81B21148FFF715
:1031B000ABFBD4E71048DBE70F48E4E70E48EDE748
:1031C0000E48EBE716AA0608585F0020C00A001058
:1031D0002CAA06084015001033AA060850700020DB
:1031E0004DAA06085CAA06087CAA06088CAA06084E
:1031F000A6AA060857AA060885AA0608B1E906087D
:103200000EB403B503AA52F8041B0192FDF70AFDA0
:10321000064BD3F8C82D22B90549D3F88800FDF72D
:1032200001F802B05DF804EB03B07047585F00206E
:103230000EB006082DE9F04798460B7903F0E0043C
:10324000402C81460F46164631D1684DDFF8A081EB
:10325000DFF8C091002422E03B7903F00703013B33
:10326000042B04D8DFE803F006080B0E2000315DC4
:1032700028460AE03157FBE736F81410F8E736F92C
:103280001410F5E756F824104046FFF7BBFA7B7997
:10329000013BA34202DD4846FFF730FA01347B7957
:1032A000A342D9DCBDE8F08756F82410E0E703F02C
:1032B0000703052B58D8DFE803F0030C1416193167
:1032C0003578602C5ED045D8002C66D0202C7CD080
:1032D000E8E796F90050602C54D03BD8002CF5D18B
:1032E00048E03588EDE7B6F90050F4E7D6F800A0DD
:1032F000202C554669D02BD8002CD3D151463C48C0
:10330000FFF780FAD7F805108A4518D8B8F1000FF2
:10331000C8D03848BDE8F047FFF774BA202C3568AC
:1033200053D015D8002CBDD129463048FFF76AFA92
:10333000D7F80510A94202DB4B42AB42E6DDFFF7AE
:10334000FDF93A682C492B464846BDE8F04757E757
:10335000602C17D0802CA5D13178284B2848002923
:1033600014BF31461946D5E7202C2DD007D8002CA4
:1033700098D12546B7F90540B7F9076011E0602CF0
:10338000E8D100257B7945FA03F3DB07BDE8F04778
:103390004CBF1C481C48FFF735BAB7F80540B7F8D2
:1033A000076012482946FFF72DFAAC42C7DCAE424F
:1033B000C5DBB8F1000F3FF475AF32462146134824
:1033C000BDE8F047FFF71EBA00257A79104B03EBF2
:1033D000C20393F8D4249542B1DAD3F8D03453F829
:1033E0002500BDE8F047FFF789B900BFB7A506087B
:1033F000A0A50608C6AA0608CCAA060811D3060886
:10340000D3B8060808A60608B1E9060887B3060877
:10341000A4F9050838A7060813B504460846019222
:103420000091FCF78FFFDDE900130246204602B051
:10343000BDE81040FEE60EB403B503AA52F8041B23
:103440000192FDF7EFFB054B0549D3F88800FCF727
:10345000E9FE02B05DF804EB03B07047585F00204E
:103460000EB0060801490246E5E700BFE6AA0608D5
:103470002DE9F041144BD3F80C3A88B00446F3B16F
:103480001A6804A9D56A18466A46A847064688B14C
:10349000DFF8408004AC6D46002735F8022B34F885
:1034A000021B40460137FFF72FFABE42F5DC08B099
:1034B000BDE8F08105492046FFF7BDFFF7E7044965
:1034C00008B0BDE8F041B6E7585F002017AB06082A
:1034D0002FAB0608FDAA060813B50446084601915D
:1034E00048F0BAFD024670B10F2804D1019909488D
:1034F0004BF0E2F838B1074B074A0849204602B0C2
:10350000BDE8104097E70349054802B0BDE8104008
:10351000FFF7FAB9FC5E060836AB060841AB0608B1
:103520006BAB060813B504460846019148F094FDBC
:103530000199024668B1042803D109484BF0BCF850
:1035400038B1074B074A0849204602B0BDE8104091
:1035500071E70349054802B0BDE81040FFF7D4B950
:10356000F45E060879AB060841AB060889AB06088D
:103570002DE9F04306469BB008460C4648F06CFD2A
:10358000002705461C22394602A801974BF057F840
:1035900025B3402D07D0394940232A4630461BB079
:1035A000BDE8F04347E70DF1040804F140090222A9
:1035B000214668464BF094F80023102209A968467A
:1035C0008DF80270FDF7EAFC099B0DF102029342AF
:1035D00022D10234A14508F8010BE8D100213D2297
:1035E0000AA809914BF02BF8002D3AD0244C257EE7
:1035F000D5B1202204F11C0101A84AF0F6FF98B1D0
:1036000004F11C0109A8FDF7EBFB1E4A1E4909AB9A
:103610003046FFF710FF04E01A781C493046FFF7E8
:103620000AFF1BB0BDE8F08394F88430CBB9C5B96C
:1036300001AD0FCD164C0FC495E80F0084E80F00C4
:10364000144B012209A8A4F1100183F8BC25FDF751
:10365000C7FB1148FFF790F8104809A9FFF754F984
:10366000DFE70C4B93F8BC351BB9054B1B7E002BD9
:10367000F2D0074909A8FDF7B3FBEDE79CAB0608BC
:10368000585F0020DAAB060841AB0608BEAB06085F
:10369000745F002050700020E4AB0608F3AB06080E
:1036A0002DE9F74F834608460D4648F0D5FC3B4FC1
:1036B0000446D7F89C95B8B939483A4D3A4FFFF7C8
:1036C0001DF8012655F8041B49B106FA04F313EA64
:1036D000090F02D03846FFF795F80134F2E703B03E
:1036E000BDE8F04FFFF72AB8024630492846FDF7FB
:1036F00005FC78B92E482B4C2E4DFEF7FFFF54F8F1
:10370000041B0029EBD00B78002BF8D02846FFF7DC
:1037100079F8F4E72B782D2B224B03BF013504F108
:10372000FF344FF0010A4FF0000A002653F8048BD3
:10373000B8F1000F06D120492A46584603B0BDE82B
:10374000F04F78E62246414628460193FDF7D6FB26
:10375000019B00BB0123B3409A0505D5174803B070
:10376000BDE8F04FFFF702B8BAF1000F0DD029EA1B
:1037700003031348C7F89C35FEF7C0FF0D484146C8
:1037800003B0BDE8F04FFFF7BFB849EA03030D48A7
:10379000C7F89C35F0E70136C8E700BF585F002046
:1037A00000AC0608980106080AAC060864A90608D9
:1037B0000EAC0608DBA8060819AC06082AAC0608F9
:1037C00036AC06083FAC06082DE9F74F814608469F
:1037D0000E461746984648F03FFC0446E8B93F4875
:1037E0003F4DFFF70FF820460EF0A4FE3B6818424D
:1037F00006D020460EF0B0FE01462846FFF702F83C
:103800000134182CEFD13B6813B93648FEF776FF28
:1038100003B0BDE8F04FFEF791BF02463249304693
:10382000FDF76CFB0546A8B93048FEF767FF2C464C
:103830002F4D20460EF07EFE10EA080F06D02046DF
:103840000EF08AFE01462846FEF7DCFF0134192CF3
:10385000EFD1DDE733782D2B48F0807303BF0136BD
:1038600004F1FF34012500254FF0000A0193504672
:103870000EF072FE2246834601463046FDF73EFBBF
:1038800000BB50460EF056FE019B03421AD08DB18C
:10389000BAF1180F1CBF3B6840EA03081548C7F887
:1038A0000080FEF72BFF1248594603B0BDE8F04FE9
:1038B000FFF72AB8BAF1180F1CBF3D6885433D6079
:1038C0000D48EEE70AF1010ABAF1190FCFD10B4901
:1038D0003246484603B0BDE8F04FACE547AC0608B9
:1038E000DAA8060851AC060864A906080EAC06085A
:1038F000DBA8060836AC06083FAC060819AC06087B
:10390000014A40F202235FE704660020014A6FF09B
:103910007F4359E7FC65002008B50A4B93F8C025A2
:10392000032A0AD193F8C135092B06D12CF0C8FF20
:10393000BDE808400448FEF7E7BFBDE8084003497A
:1039400079E500BF5070002058AC060863AC06084B
:1039500070B5054608461646FDF7C2FB0D4B93F8B9
:1039600090259042044605D201460B48FEF7CCFF55
:10397000204670BD2EB1FF2803D10848FEF7C4FFD2
:10398000F6E70749013A2846FFF755FD4FF0FF34A7
:10399000EEE700BFC00A001072AC060883AC060850
:1039A00096AC06082DE9F04F074691B08248834D4A
:1039B0000E46FEF7A9FF8249C5F8E0D5002385F839
:1039C000E4350622012391F890153046402485F80D
:1039D000E54509F0F5F80A2009F03EF995F8E435D7
:1039E0000C2BDAB240F2E4809DF80C50FE2D30D062
:1039F000FF2D0BBF15240F2401260026944240F012
:103A0000D780611EC9B268463CF032FD04F1400324
:103A10000DEB030414F8413C834240F0C48006F1EE
:103A2000FF385FFA88F8B8F1010F9DF80D3012D910
:103A300003F01F0761375C096248FEF75FFE022E44
:103A40006AD0013C042C65D8DFE804F00B5E6064AA
:103A500062000226D2E79DF80E709DF80F401D46C9
:103A6000EAE75948DFF8BC91DFF8BCB1FEF77EFE0B
:103A70005648FEF743FE6C464FF0000A14F8011B4F
:103A800048460AF1010AFEF7BDFEBAF10C0F49D112
:103A9000FEF754FE022E4FD06422B5FBF2F102FB7A
:103AA00011524B483B46D2B2C9B2FEF72DFFB8F1D6
:103AB000010F71D8474A484B9DF810104748484DB0
:103AC000002914BF11461946FEF71EFF9DF811107C
:103AD000444B4548002914BF19462946FEF714FFF8
:103AE000022E59D19DF812404048FEF707FE4CB314
:103AF000FF2C37D00A22B4FBF2F102FB11423C4802
:103B0000D2B2FEF701FF20E03A48ABE73A48A9E716
:103B10003A48A7E73A48A5E700238DF83F300DF172
:103B20001F009FE7374B03FB0AF2B2F1553FA5D8C0
:103B30005846FEF7E3FDA1E733483A462946FEF72B
:103B4000E3FEB7E72846FEF711FE9DF813402F4825
:103B5000FEF7D4FD44B1FF2C21D02D482146FEF7BD
:103B6000D3FE04E02B48EEE71D48FEF7FFFD1C4E98
:103B7000284FDFF870800DF11305002415F8013F80
:103B80007BB1FF2B0CBF3A46424621462248013406
:103B9000FEF7BAFE042CF1D111B0BDE8F08F1D483C
:103BA000E3E73246F1E71D493846FFF744FCF3E707
:103BB0001B48FEF7DBFDEFE7DCAC06085070002089
:103BC000C00A0010EDAC0608F8AC06081EAD0608E9
:103BD00030AD0608BCAC0608C5AC060867AD0608E3
:103BE000CCAC06085ABA06087EAD060885AD0608B4
:103BF00099AD0608FFAC060807AD06080FAD06082C
:103C00006EA60608ABAAAAAA4CAD0608A1AD060886
:103C1000B7A50608D0AC0608B1AD0608BCAD0608CD
:103C2000CCAD060890A4060811D306082DE9F84F7C
:103C3000DFF8A880DFF88890DFF8A4A007460C46DC
:103C4000204648F009FA064660B91D4B1D4893F816
:103C50002C241D4B03EB8203D3F86C18BDE8F84FFE
:103C6000FEF752BE024641462046FDF747F960B1D5
:103C7000DFF860B000255BF8041BB1B92246384676
:103C80001249BDE8F84FFFF7D6BB1148114C124D51
:103C9000FEF734FD54F8041B19B12846FEF7B2FDB7
:103CA000F8E7BDE8F84FFEF749BD32462046FDF77C
:103CB00025F901350028DED189F82C545446BFE798
:103CC000585F0020D5AD0608A4F9050819AC060810
:103CD0000EAC060814020608DBA8060864A906084C
:103CE00010B0060838B50D4604461A490522284684
:103CF000FDF704F968B9184B93F88C2022B901211B
:103D000083F88C1083F88D20BDE838401348FEF707
:103D10002DBD134903222846FDF7F0F8A0B90E4D3A
:103D200095F88C3063B195F88D304BB10D49204634
:103D3000FFF781FB002385F88C3085F88D3038BD86
:103D40000948FEF713FDF5E720460849BDE838406D
:103D5000FFF771BB9CB90608585F0020DFAD06086D
:103D600003BB0608F5AD06082CAE060840AE0608F3
:103D7000F8B5174C94F88C3005467BB194F88D302B
:103D800063B11449FFF757FB28461349FFF753FB6C
:103D9000002084F88C0084F88D00F8BD0F4E96F852
:103DA000BC7597B1207E0028F7D10D4D0FCD06F5DB
:103DB000BD640FC495E80F0084E80F00012386F866
:103DC00023360AF021F93846E7E70120E5E700BF8E
:103DD000585F0020F5AD06084FAE06085070002071
:103DE000745F002008B5FFF7C3FF50B1054B0122F7
:103DF0009A75FEF7BBFA0448FEF7BEFC0020FEF7FA
:103E000085FC08BD585F00206DAE060808B5034666
:103E100010462AB1DB0600D511B1FEF7ADFC00203B
:103E200008BDF8B50D4E96F88430054693B9F8BD37
:103E300025B12388C3F30B039D4204D0D4E90201CA
:103E4000A2884AF099FB1C34BC42F1D3002386F8C7
:103E50008430ECE7024C034FF6E700BF585F0020C8
:103E600090EC06086CF506082DE9F04F85B0164673
:103E700001911A46824600213046FFF7C7FF324CB7
:103E800006F0100305464FF000090293FEF71AFCF6
:103E90002379019A03F01803934203D0002A48D1F2
:103EA000182B46D1284B4FF00D0B0BFB0933B3F801
:103EB0000900FCF731FA80462046FCF750F8D8E9B3
:103EC00002210746024401442046FCF701F880F035
:103ED00001012A460390C9B23046FFF797FFDDE99A
:103EE0000223054602B123BB174A0BFB09FB52F81C
:103EF0000BB0B2060FD573B9144803935946FEF7B9
:103F000081FCD8F80820039B3A4421465046FFF72D
:103F100091F9FEF713FC0E485946FEF773FCD8F8EA
:103F20000C2000233A4421465046FFF783F9FEF760
:103F300005FC09F1010940F26A23994504F10D04D9
:103F4000A4D105B0BDE8F08F6013060874AE060872
:103F500075AE06080149FFF76EBA00BF7FAE0608CE
:103F600038B50C46054615492046FCF7A3FF30B985
:103F7000FEF78EFB1248BDE83840FEF7F7BB11494B
:103F80002046FCF797FFA0B90F4A82F8EE0182F8AD
:103F9000F60182F8920282F89A0282F8360382F8D9
:103FA0003E0382F8DA0382F8E20382F81904074834
:103FB000E1E72846BDE83840CCE700BF8EAE0608F2
:103FC00094AE0608AFAE0608585F0020B7AE0608EC
:103FD0002DE9F043064687B008460C4648F03CF809
:103FE000082843D1671E03AD073429463A46A84640
:103FF00012F8010FFCF758FFA24201F8010BF7D1AC
:104000000023DFF87C908DF8143017F8010FFCF7CF
:104010004BFFC1B205F8010B484601914AF026FB5F
:1040200020B1019928464AF021FB28B13046FFF71C
:1040300091FF07B0BDE8F083A742E6D10F494046A3
:104040002CF0B6FB0D480E49082310F8012B11F88F
:10405000014B18326A44013B02F80C4CF5D1094877
:104060008DF8143003A9FEF74FFCE2E70028E9D0F1
:10407000304607B0BDE8F043FFF7F4B98C63002089
:104080001C720608D3AE06082DE9F74F064601AAB2
:1040900008462F49DFF8C880DFF8C890DFF8B0A0E5
:1040A0004AF0A0FA4FF0000B04465D4601271CBB06
:1040B000BBF1000F28D1274C002D44D026482946BB
:1040C000FEF722FC94F884300BB904F0B7FEFCF73D
:1040D000B5F9002384F88D30FEF7DAFA15B12846D9
:1040E000FFF79FFE9FB13046FFF742FE78B1FEF723
:1040F0003DF90020FEF70AFBBBF1000F0AD0204675
:10410000FCF7EEFF85B2C5B93046FFF723FF03B0D9
:10411000BDE8F08F41462046FCF714FF80B94946C0
:104120002046FCF70FFF0028EED05F4601AA51465B
:1041300000204AF057FA0446B9E74FF0000BF5E7C4
:104140004FF0010BF2E70548FEF716FBBFE700BF93
:104150009FB30608585F0020E3AE060806AF0608C6
:10416000DAAE0608D3B9060807B5009313460A4627
:104170000249FFF760F903B05DF804FB1CAF0608C5
:1041800020B10078B0FA80F04009704701207047F4
:104190002DE9F34106460846FFF7F2FF0D460746B4
:1041A00070B1002401A9204642F0D6FC013401463A
:1041B0003046FFF7EDFF122CF4D102B0BDE8F081DC
:1041C0000846FCF78DFFC4B2112C71D8681CFCF7AF
:1041D0003BF83B4D8046E8B93A4B03EB440393F878
:1041E00024168A1E51425141364B03EB440393F887
:1041F0002426AA5C002954D093F82536192040F2D1
:10420000EE2100FB03133048214602B0BDE8F04127
:10421000FEF77ABB017828464AF028FA70B1032CE1
:1042200094BF00220122294902EB4202431B0A44A7
:1042300052FA83F393F8DC78032F04D1304602B0AE
:10424000BDE8F04186E64046FBF7FEFF08B3022FCB
:10425000F4D1FCF745FF40F6CA0280B29042194BF8
:10426000A8BF104640F2EE22904203EB4403B8BFD1
:104270001046A0F2EE201922B0FBF2F083F82506DA
:10428000BB1E594259410F4B03EB440383F824767C
:10429000AAE7022FF4D1304602B0BDE8F041FFF7A3
:1042A000E1B80B48214602B0BDE8F041FEF72CBB57
:1042B000084911233A46304602B0BDE8F04153E7C1
:1042C000D07306085070002035AF0608A4F9050821
:1042D00045AF060852AF06082DE9F04F024691B0EF
:1042E0000846FFF74DFF0B46044628B1104611B0B3
:1042F000BDE8F04FFFF7B6B84FF0FF32CDE9082028
:10430000A74ADFF8E482D2F88020DFF8E09292F842
:104310003810DFF8DCA2CDE90C10CDE90E02CDE9B2
:104320000A00A04907AA18464AF05CF92746054644
:10433000049426464DB9089A0C9FBA4262D19A4815
:10434000FEF7E2FA11B0BDE8F08F062F12D8DFE8D1
:1043500007F0041E2328454C510051462846FCF71F
:10436000F1FD78B14FF480600EF050FB90F904300D
:10437000089301248B4907AA00204AF033F901373A
:104380000546D7E72846FCF7ABFE0890F2E728463B
:10439000FCF7A6FE0990EDE72846FCF7EAFD0A9037
:1043A000E8E7284647F058FE414602460590284671
:1043B000FCF7A4FD18B3059A49462846FCF79EFD74
:1043C00006460028D6D02846FCF78AFE0428064672
:1043D000D0D901467548FEF797FAB3E72846FCF7AF
:1043E0007FFE00230C900F93C4E72846FCF778FE6D
:1043F0000D90BFE72846FCF7BCFD0E90BAE70123FD
:104400000493B7E7DFF8EC8151B2434613F9010B8F
:10441000884208D00135092DF8D1002164480131C6
:10442000FEF772FA8EE763480121FEF76DFA7AB261
:10443000002318F9011B8A4200F00D810133092B7A
:10444000F7D13A460121E9E7A7F11402534253415B
:10445000059308AD002303F10108EB68A3BB95F9B0
:1044600000B058460EF09AFAD5F804A020B1D0F862
:104470000090B9F1000F5ED1BAF1000F19D14FF4DD
:1044800061436B604FF0010AAB680BB90323AB606B
:104490000023D5F8049002932A7A1946CDE90092B8
:1044A00058461A460EF0BAFBE86028B94248414621
:1044B00091E74FF0000AE7E74A464146BAF1000F9C
:1044C00037D03E48FEF79EF9B8F1020F05F110050E
:1044D0004FF00103BFD1059BDDF83C800B9D53B12C
:1044E0003748FEF743F9D8F800301B6A1BB135494D
:1044F0002A4640469847049B002B4ED03249334B06
:10450000142F18BF19463248FEF7FEF9142F09D1AF
:10451000049B03B936B12B68DB691BB12D493246C8
:1045200028469847002C67D100224146284642F091
:10453000C7FA2948C6E7C5F80C90BAF1000F25D094
:10454000264841465246FEF75DF95146484603F07B
:10455000C1F8D5F808A0BAF1000F0FD099F80420DF
:1045600092450BD01E4853464146FEF74BF9D9F809
:1045700000305FFA8AF19B6948469847D9F82C3099
:10458000002BA1D00023C9F82C309DE7D9F80820D2
:1045900014484146FEF736F9DBE70C49B3E700BFA4
:1045A000585F00209FB3060890AF060878AF060852
:1045B000D4B00608A9AF0608B5AF0608D1AF060803
:1045C00088B00608D57601085AAF060810B006086C
:1045D000B1B0060863020108F5AF060811B006087D
:1045E00063B006083EB0060872AF060853AC060872
:1045F00067AF060860FD050805F094FA052008F08D
:104600002BFB1A4FDFF86C9000264FF0030A99F845
:104610009035B34288D917F801BBBBF1000F15D014
:10462000584609F08BFB044680B1584605F0B2F9B4
:1046300008B1A0F806A001210490F6F70FFDA379B8
:10464000049813F0010F03D0F5F7C4FE0136DEE73E
:10465000F5F7BAFEFAE706483A460221FEF754F9A2
:10466000099B002B3FF4F0AE0023F1E6A4270020C5
:10467000A9AF0608C00A001010B5044608460B464C
:10468000FFF77EFD28B9094903221846FCF736FCDE
:1046900028B90748FEF770F80120FEF737F82046E2
:1046A0000449BDE81040FEF7C6BE00BFE6B00608EC
:1046B000EAB0060840AE06082DE9F74F0546084661
:1046C000FFF75EFD0B46044618B9334A92F8487668
:1046D00027B9284603B0BDE8F04F3BE42F49DFF887
:1046E000C880DFF8C890DFF8C8A001AA184649F0D2
:1046F00079FF264610B905F023FA08E056B90122E1
:1047000001462846FFF724F9421C04461BD103B09A
:10471000BDE8F08FFCF7E4FC2F28834636D80FB1B4
:1047200005F000FABBF1060F14D01D49012391F8E2
:1047300090155FFA8BF2E0B208F042FA594648460B
:10474000FEF7E2F80027154901AA0020013649F0DA
:1047500049FFCFE7DAF8A0351B0113D5FF2C0FD0A6
:10476000E1B22846FFF71EF9E8E72846FFF71AF9F5
:1047700001370B4B93F89025F9B28A42F5D8DDE763
:104780000027F6E70748FDF7F1FFD7E72F2241465C
:104790002846FEF750FED6E7507000209FB306086B
:1047A000C00A001063AC06081DB106080CB106086B
:1047B000585F00202DE9F04F064685B00846FFF708
:1047C000DFFC0B46044628B1304605B0BDE8F04F8B
:1047D000FEF748BE3149DFF8D490DFF8D4A0DFF807
:1047E000D4B003AA184649F0FDFE27460546A04668
:1047F00065B92B4B3A46D3F88000A1B241F0ECFEEC
:1048000068BB28493046FEF716FE28E0B8F1000FD5
:1048100006D0B8F1010F25D03046FEF723FE1EE08A
:10482000284647F019FC4946024601902846FCF705
:1048300065FB50B3019A51462846FCF75FFB30B345
:10484000019A59462846FCF759FB10B3019A1649BC
:104850002846FCF753FBF0B13046FFF77BFB05B071
:10486000BDE8F08FBB1E5A425A4129463046FFF739
:104870006FF8421C0446F2D0084903AA002049F010
:10488000B1FE08F101080546B2E74746F4E7012703
:10489000F2E70227F0E70327EEE700BF9FB3060821
:1048A000585F002049B1060846B106083DB1060828
:1048B00040B1060843B106082DE9F7438046084693
:1048C000FFF75EFC0B46054628B14046FEF7CAFDE1
:1048D00003B0BDE8F0832E49DFF8B49001AA184672
:1048E00049F080FE2F4604462E467CB9022DECD1BD
:1048F000A7F57A73B3F57A7F21D926494FF4FA6385
:104900004FF47A724046FFF72FFCE1E74DB1012DDD
:1049100010D001AA4946002049F064FE0135044642
:10492000E3E7012221464046FFF712F8431C064602
:10493000EFD1CDE72046FCF7D3FB0746E9E7164D5C
:10494000D5F8203AB8B25B689847FF2EBCEEC00A93
:10495000124B0BD195F89025F8EE407AA24212DC6A
:1049600010EE101A0E48FDF7CFFFB1E7F8EE407ACF
:1049700003EB860310EE102A0A48C3ED007A314695
:10498000FDF7C2FFA4E7E3EC017A0134E6E700BFDC
:104990009FB3060857B20608C00A00109C76002094
:1049A00074B1060867B10608F8B507460846FFF770
:1049B000E7FBC8B11F4B1E6D013630460DF0CCFD34
:1049C00034460546F0B90134192CA8BF002420460E
:1049D0000DF0C2FD0546A8B9B442F4D138461649D7
:1049E000BDE8F840FEF727BD0846FCF779FB044612
:1049F0000DF0B2FD054628B921461048BDE8F84043
:104A0000FDF782BF0B4B1C650EF0CEF90C482A4611
:104A10002146FDF779FF182C09D80A480C2101FB23
:104A2000040090F8E408BDE8F8400EF0F3B9002067
:104A3000F9E700BF1005002083B1060897B106080A
:104A4000ADB10608A4F9050838B5124D044608466C
:104A5000FFF796FB60B1104B104893F900104B1C08
:104A60000ABF0F4BC9B2197ABDE83840FDF74CBFF9
:104A70000846FCF735FB032804D8C0B2FDF7C8FA96
:104A80002946E4E720460749BDE838400322FEF7FF
:104A9000D2BC00BF10B0060810050020C6B1060841
:104AA000585F0020D6B1060838B5124D04460846B6
:104AB000FFF766FB60B1104B104893F901104B1CD7
:104AC0000ABF0F4BC9B2597ABDE83840FDF71CBF89
:104AD0000846FCF705FB032804D8C0B216F0FEFC1C
:104AE0002946E4E720460749BDE838400322FEF79F
:104AF000A2BC00BF10B0060810050020C2B1060815
:104B0000585F0020D1B106082DE9F74F444BDFF87C
:104B100028A11A7A8AF800205A7A93F884308AF801
:104B20000120054688460BB904F088F9FBF786FC9E
:104B300000263C4CB1460D233A4A7343414652F895
:104B400003B05846FCF7FEF9002841D0B9F1000F38
:104B500001D0FDF7F3FD34485946FDF753FE00221E
:104B600021462846FEF758FCFDF7E8FD237903F0BF
:104B70001803082B46D0102B49D02046FDF7D3FE52
:104B8000284A0D2303FB0623B3F80900FBF7C4FBF7
:104B90000746D8B12046FBF7E2F9D7E90221009099
:104BA000024401442046FBF793F978B90190594635
:104BB0001E48FDF727FE019AB9681346009A284659
:104BC0000A442146FEF736FBFDF7B8FD09F101095D
:104BD000013640F26A239E4204F10D04ABD100205D
:104BE000FFF71FF9FF238AF800308AF80130B9F186
:104BF000000F11D10E494246284603B0BDE8F04FE0
:104C0000FEF719BC0B492846FFF71EFFB5E7094917
:104C10002846FFF749FFB0E703B0BDE8F08F00BFBB
:104C2000585F00206013060879AE0608F1B1060847
:104C300019AC060810B00608100500202DE9F74F42
:104C4000074608460E4647F007FA044620B10128F9
:104C500026D132782A2A23D1B348B44EDFF8E8921D
:104C6000FDF784FD0025B2464FF00D0B40F26A2897
:104C70000BFB05F348465AF80310FDF7C3FD221E4F
:104C800018BF0122314638460135FEF7C5FBFDF756
:104C900055FD454506F10D06EAD103B0BDE8F08F9C
:104CA0003D21304649F0E2FC002800F03781014602
:104CB0000A4611F8014D202CFAD0921B0130814692
:104CC00010F8011B2029FAD0DFF860B25FFA82FAEF
:104CD0004FF000080D2303FB08F10BEB01045246D3
:104CE0005BF8011000913046FCF708F905460028F2
:104CF00057D10099084647F0AFF9824551D126793E
:104D000006F0E001402900F0CC800ED8002956D0F2
:104D1000202900F09E8038468549FEF78CFB20460E
:104D200003B0BDE8F04FFDF7FEBD602900F09280B2
:104D30008029F0D1484647F08FF9E379A679DB075F
:104D400005460CD52046FBF7FDFA0378014633B142
:104D50002A46484649F0B0FC002840F0D980002D92
:104D600000F0D680AE42C0F0D3800D2303FB08B321
:104D7000204693F805A0FBF7E5FA3246002149F0FA
:104D80005EFCAA452CD86B492A46484649F094FC5B
:104D900030B32046FBF7D6FA2A46494649F0ECFBE9
:104DA0001EE008F1010840F26A23984592D1624959
:104DB0003246384603B0BDE8F04FFEF73CBB06F084
:104DC0000703042B1CD10B460A224846FCF7E6F8E1
:104DD000D4F80530834201469DD32046FBF7C8FA3C
:104DE0000D2303FB08F855485BF80810FDF70AFD92
:104DF00000222146384603B0BDE8F04FFEF70CBB59
:104E0000052B0FD101230A224846FCF7C7F8D4F836
:104E1000053083420146FFF67EAF5B4283423FF797
:104E20007AAFDAE74846FCF75BF9B4F80550B4F816
:104E3000071016F0050FAAB218BF2AB28BB218BF1E
:104E40000BB29042FFF667AF98423FF764AF01465E
:104E5000C3E765793A4A02EBC505002695F8D424E4
:104E60000092B2463346009AB24202D9BAF1000F1C
:104E700003D0002B3FF44FAFB2E7D5F8D01451F870
:104E8000260060B149460193FCF714F8019B30B944
:104E9000314620464FF0010AFBF76AFA53460136C5
:104EA000E1E76379009306F00706013E009BAB4201
:104EB00096DD4846814610F8013B202BFAD020466B
:104EC000FBF740FA8246042E04D8DFE806F0031010
:104ED00010161F004846FCF703F90AF8050048467B
:104EE0002C2149F0C3FB013500F10109DEE74846FA
:104EF000FCF7F6F82AF81500F1E700230A22002152
:104F00004846FCF74BF84AF82500E8E70123F5E7A7
:104F10000C4932463846FEF78EFAFCE631463846F2
:104F200003B0BDE8F04FEFE501B2060860130608D4
:104F30004FB2060811D3060819AC060844B2060899
:104F4000A4F9050814B2060879AE06082DE9F04F59
:104F5000914689B00C461A4600218046FEF756FF5E
:104F6000DFF8ECB006464D460027B9F1000F6CD0D3
:104F700029460622204649F038FB0028324614BF55
:104F80000121002140460CBF4FF0010A4FF0000AFA
:104F9000FEF73CFF0646287814F09EFE079010B3FB
:104FA000687914F099FE079BEA785B790793AB78F0
:104FB00095F801E04FF461714FF0190C1CFB0313DD
:104FC0001CFB0212297900B14079CDF804E0CDE94B
:104FD0000232079B0093CDE904103B465A465146E6
:104FE0004046FDF7F7FB207814F076FE079010B3EB
:104FF000607914F071FE079BE2785B790793A378E0
:1050000094F801E04FF461714FF0190C1CFB03138D
:105010001CFB0212217900B14079CDF804E0CDE902
:105020000232079B0093CDE904103B465A46514695
:105030004046FDF787FB0137142F04F1060405F104
:10504000060592D109B0BDE8F08FCA46CBE700BF94
:105050005DB206082DE9F041064686B00846FFF726
:105060008FF80F46054638B100235D491A460120E6
:1050700006B0BDE8F04169E70846FCF731F81328AF
:10508000044600F3A38006264643781C8DF817508B
:10509000FBF7DAF8534D074670B1FCF721F8C0B2C0
:1050A00014F030FE40B1AB19027983F810269DF858
:1050B000173001338DF817303846FBF7C5F807462F
:1050C00068B1FCF70DF80D2809D8062303FB04533B
:1050D00083F811069DF8173001338DF81730DFF88B
:1050E0000081B11C0DF1170241443846FBF7FCFF6B
:1050F000FBF7AAF8074668B1FBF7F2FF012809D8C9
:10510000062303FB045383F814069DF8173001337C
:105110008DF817303846FBF797F880B1FBF7E0FFC2
:10512000C0B214F0EFFD50B1062303FB0453027923
:1051300083F815269DF8173001338DF817309DF848
:105140001720042A4FF006032FD103FB045300223B
:10515000A3F814261FF0F2FA062303FB04554FF4BC
:10516000617695F8100614F0B7FD95F8132695F8BA
:1051700012761923804695F8150613FB076713FB73
:10518000026614F0A9FD437998F80520039395F879
:1051900014360097CDE90163134895F8113621467E
:1051A000FDF7B2FB06B0BDE8F081052A05D103FB8F
:1051B0000453002283F81526CCE7062ACAD008EB50
:1051C0000602002348F806309380C3E707491323FB
:1051D0002A46304606B0BDE8F041FEF7C5BF00BF25
:1051E00068650020585F00205DB2060876B20608A8
:1051F0002DE9F04F174689B01A460C46002181462A
:10520000FEF704FE3B4EDFF8F4B007F16C03804676
:105210003D46079394F90410374A002392F9080099
:10522000884263D00133092B02F10C02F6D1079BAF
:105230000C359D4204F10C04ECD109B0BDE8F08FAF
:1052400029460C22204649F0D0F90028424614BFD6
:105250000121002148460CBF4FF0010A4FF0000A1F
:10526000FEF7D4FDEA7995F9043006EB8202804618
:10527000D2F8142704922A7A06EB82025146D2F819
:1052800014270392AA7906EB82024846D2F8142723
:1052900002926A7906EB8202D2F8142701922A68F8
:1052A00000925A46FDF796FAE27994F9043006EB3B
:1052B00082025146D2F814270492227A06EB820227
:1052C0004846D2F814270392A27906EB8202D2F85C
:1052D00014270292627906EB8202D2F81427019217
:1052E000226800925A46FDF72DFAA0E7002FA7D1B9
:1052F000BA46D9E7A4F90508886400207CB20608FC
:105300002DE9F04380468BB00846FEF739FF38B1EF
:1053100000234D491A4601200BB0BDE8F04367E772
:10532000CDE90700099008464D1CFBF7D9FE44B2B1
:1053300020460DF0E7FA0646002843D08DF82040BD
:1053400001242846FAF780FF054638B100230A22D7
:105350001946FBF723FE01340790E4B2DFF8F09022
:1053600000272846FAF770FF054618B3FBF7B8FE8A
:105370003649002251F804CB6045D3B203D0013244
:10538000102AF7D1002309EB8302D2F814279042A8
:1053900010D1022F1DD0032F20D05A1E012FD2B2C0
:1053A00012D00B2A03D88DF821300134E4B2013732
:1053B000042FD6D1052C17D840460BB0BDE8F043DA
:1053C000FEF750B80446BCE7042AF0D88DF8223026
:1053D000EBE7052BEBD88DF82430E6E79A1E0D2A73
:1053E000E5D88DF82330E0E707AB03CB9DF8232009
:1053F00030601868164B716003EB8202B060D2F81F
:10540000142704929DF8242003EB82020021D2F895
:10541000142703929DF8222003EB82020846D2F85B
:10542000142702929DF8212003EB8203094AD3F846
:1054300014370193079B00939DF92030FDF782F903
:105440000BB0BDE8F08300BFC4630020B8000608BD
:10545000A4F905087CB206082DE9F04F8BB00C4684
:10546000089200211A460746FEF7D0FCDFF8B4B0D8
:10547000089D099000264FF019094FF46178089BA8
:10548000002B4BD029460A22204649F0AEF80028CE
:10549000099A14BF0121002138460CBF4FF0010AC0
:1054A0004FF0000AFEF7B2FC2A890692EA880592BC
:1054B0002A790492EA780392AA78099019FB028269
:1054C00002926A7819FB028201922A78009233468E
:1054D0005A4651463846FDF77DF922890692E28800
:1054E000059222790492E2780392A27819FB028253
:1054F0000292627819FB0282019214F80A2B009240
:1055000033465A46514638460136FDF71BF91E2EE2
:1055100005F10A05B3D10BB0BDE8F08FDDF820A08E
:10552000DBE700BF99B206082DE9F04380468BB057
:105530000846FEF725FE0F46044638B100236549AC
:105540001A4601200BB0BDE8F04385E70846FBF79B
:10555000C7FD1D28054600F3B3800A264643781C84
:105560008DF82740FAF770FE044630B1FBF7B8FD1E
:105570009DF8273001338DF827302046FAF764FE76
:10558000554C074668B1FBF7ABFD0D2809D80A2337
:1055900003FB054383F86C069DF8273001338DF833
:1055A0002730DFF83091711C0DF12702494438464D
:1055B000FBF79AFDFAF748FE074668B1FBF790FD46
:1055C000222809D80A2303FB054383F86F069DF8B8
:1055D000273001338DF827303846FAF735FE074675
:1055E00068B1FBF77DFD0D2809D80A2303FB0543AD
:1055F00083F870069DF8273001338DF827309DF829
:105600002730062B0CD009EB0602002349F80630A0
:10561000404653601381FDF725FF0BB0BDE8F083D2
:105620000A2606FB054600233846A6F87236A6F879
:105630007436FAF709FE074640B1FBF751FD9DF8B5
:105640002730A6F8720601338DF827303846FAF76E
:10565000FBFD58B1FBF744FD0A2303FB0543A3F808
:1056600074069DF8273001338DF827301B4B4FF01F
:10567000FF325A600A2202FB05424FF46170B2F811
:1056800074360693B2F87236059392F87036049326
:1056900092F86F36039392F86E16192313FB0101EB
:1056A000029192F86D1613FB0103019392F86C3688
:1056B000009300210A4A2B460846FDF743F8ACE761
:1056C00008491D23224640460BB0BDE8F043FEF7D3
:1056D0004BBD00BFBC76002050700020100500209C
:1056E00099B2060876B206082DE9F04F2DED088B29
:1056F000DFF82CA195B0804691461F460C46164611
:105700004FF0000B94ED008AB5EE408AF1EE10FAEE
:105710007FD0D4ED019A94ED029AD4ED038AB9F1C9
:10572000000F49D0D6ED00BA96ED01BAD6ED02AA27
:1057300096ED03AAB4EE6B8AF1EE10FA6ED1F4EE98
:105740004B9AF1EE10FA69D1B4EE6A9AF1EE10FAC2
:1057500064D1F4EE4A8AF1EE10FA0CBF0121002167
:105760003A460D46404681F00101FEF74FFBB0EE90
:105770006B0A074611A8FAF7E3FCB0EE4B0A079054
:105780000EA8FAF7DDFCB0EE6A0A06900BA8FAF74D
:10579000D7FCB0EE4A0A059008A8FAF7D1FC0599A3
:1057A000069A079B039002910192009352465B4632
:1057B00029464046FDF70EF8B0EE480A11A8FAF760
:1057C000BFFCB0EE690A05460EA8FAF7B9FCB0EEC8
:1057D000490A06900BA8FAF7B3FCB0EE680A0590E8
:1057E00008A8FAF7ADFC069B059A0390CDE9005393
:1057F00002925B465246002140460BF1010BFCF73A
:10580000A1FFBBF1080F04F1100406F110067FF4AC
:1058100079AF15B0BDEC088BBDE8F08F00219FE794
:10582000BCB206082DE9F74FDFF898A1DFF898B170
:1058300007460D462846FEF7A3FC064638B100236E
:1058400059491A46012003B0BDE8F04F4CE7052244
:1058500051462846FBF752FB60B9534B00221A60B1
:105860001A611A621A631A641A651A661A6703B013
:10587000BDE8F08F4D4904222846FBF73FFB044664
:105880002846002C44D1FAF7DFFC80460028EED0F1
:1058900046F0E2FB464BC2B253F8049BB9F1000F4D
:1058A00007D144492A46384603B0BDE8F04FFDF71A
:1058B000C2BD49464046CDE90023FBF71FFB01343A
:1058C000DDE9002306460028E6D1374A034615469F
:1058D00000210133082B42F8101BFAD10BEBC40452
:1058E000D4F8BCC0BCF1000F03D094F8B8E0764502
:1058F00005DB3148314D4946FDF706F89AE70CEBD8
:1059000006130FCB05EB061484E80F000136EEE713
:10591000FBF7E6FB072804463DD82846FAF794FC37
:10592000064658B3FAF7D8F91F4B03EB041383ED7F
:10593000000A01253046FAF787FC064638B1FAF727
:10594000CBF9194B03EB041383ED010A0135304603
:10595000FAF77AFC064638B1FAF7BEF9124B03EBB8
:10596000041383ED020A01353046FAF76DFC38B9AD
:10597000384603B0BDE8F04FFDF774BD0546D9E7E2
:10598000FAF7AAF90848032D00EB041484ED030A82
:105990003FF455AFECE70A4907233246384603B0D7
:1059A000BDE8F04FFEF7E0BB64680020D0B2060807
:1059B0001402060819AC0608D5B2060810B006088D
:1059C00076B2060872AF0608A4F905082DE9F74F6C
:1059D00092460C461A4600218146FEF717FADFF878
:1059E00070B0804656460025BAF1000F2ED03146E1
:1059F0000422204648F0F9FD0028424614BF012148
:105A0000002148460CBF01270027FEF7FFF97388E5
:105A100001933AF82530009380462B465A46394682
:105A20004846FCF7D7FE6388019334F8043B0093A3
:105A30005A462B46394648460135FCF783FE042D6D
:105A400006F10406D0D103B0BDE8F08F5746EAE76F
:105A5000DFB206082DE9F34105460846FEF790FB44
:105A60000C46074638B1002333491A46012002B0DC
:105A7000BDE8F041AAE731492046FBF71BFA03468F
:105A800070B92D4A4FF47A704FF4FA610133042B48
:105A90001080518002F10402F8D102B0BDE8F0811B
:105AA0002046FBF71DFB0328064641D82046FAF79F
:105AB000CBFB074670B1FBF713FB4FF00108044620
:105AC0003846FAF7C1FB48B9284602B0BDE8F041B4
:105AD000FDF7C8BC40F2EE248046F1E7FBF700FB7F
:105AE000B8F1000FF0D0A4F2EE2240F2DC539A425B
:105AF00003D8A0F2EE229A420AD9114940F6CA030D
:105B000040F2EE22284602B0BDE8F041FEF72CBB81
:105B10000C4B0D4A03EB86030021A3F89847A3F82A
:105B20009A07CDE9004033460846FCF70BFEB4E780
:105B3000064903233A46E5E7E877002072AF0608F6
:105B4000F0B2060850700020DFB2060852AF060817
:105B50002DE9F04F89468FB0174600211A460646B8
:105B6000FEF754F9DFF878A0054600240DF1240B68
:105B700059F824300293594602A840F04FFF67B30A
:105B800057F82430029A0393934218BF01212A4602
:105B900008BF002130460CBF4FF001084FF000084D
:105BA000FEF734F904A9054603A840F037FF04A91D
:105BB00000912346524641463046FCF70BFE2346F1
:105BC000CDF800B05246414630460134FCF7BAFDEC
:105BD000202CCDD10FB0BDE8F08FB846EFE700BF65
:105BE000FEB20608F0B5074689B00846FEF7C8FAC7
:105BF0000E46054638B1002319491A46012009B05E
:105C0000BDE8F040A4E70846FBF76AFA1F280446FF
:105C10001DD83046FAF718FB0146204635F07AFECB
:105C200078B10F4803AE314600EB840040F0F6FE39
:105C30000C4A0096234629462846FCF783FD09B006
:105C4000F0BD384609B0BDE8F040FEF783B906491B
:105C50001F232A46384609B0BDE8F040FEF784BA53
:105C6000F8770020FEB2060876B206082DE9F04F5C
:105C7000924685B00C461A4600218146FEF7C6F8CA
:105C8000DFF874B0804655460026BAF1000F31D0D7
:105C900029460422204648F0A8FC0028424614BFAA
:105CA0000121002148460CBF01270027FEF7AEF86E
:105CB000EB780293AB7801932B88009380463346B0
:105CC0005A4639464846FCF785FDE3780293A378A7
:105CD000019334F8043B00935A463346394648460C
:105CE0000136FCF72FFD102E05F10405CDD105B0CE
:105CF000BDE8F08F5746E8E708B30608F0B5074659
:105D000085B00846FEF73CFA0E46054638B100233A
:105D10001C491A46012005B0BDE8F040A6E7084638
:105D2000FBF7DEF90F28044623DC3046FAF78CFA3D
:105D30000146204635F06CFDA8B1134B04F120025A
:105D400003EB8203294693F8AB27029293F8AA2724
:105D50000192B3F8A83700930C4A23462846FCF773
:105D6000F1FC05B0F0BD384605B0BDE8F040FEF7E7
:105D7000F1B807490F232A46384605B0BDE8F04080
:105D8000FEF7F2B9787800205070002008B30608BA
:105D900076B206082DE9F04F87B0144603911A46F3
:105DA00000210546FEF732F8DFF830B106464FF025
:105DB0000008062303FB08F7C0374FF00009039BD8
:105DC000DB5D0493002C00F08580E35D049A05936D
:105DD0009A4218BF0121324608BF002128460CBF55
:105DE0004FF0010A4FF0000AFEF710F8059B064637
:105DF000CDE900935A46434651462846FCF7EAFC53
:105E0000049B5A46CDE9009351464346284609F182
:105E10000109FCF797FCB9F1060F07F10107CED194
:105E200008F10108B8F1060FC3D1DFF8B0B0E427DC
:105E3000039BA7F1E40913F807A0002C4CD0E35D05
:105E400004939A45324614BF0121002128460CBF15
:105E50004FF001084FF00008FDF7D8FF049B0646FD
:105E6000CDE900935A46062341462846FCF7B2FC8A
:105E7000CDE9009A194A0623414628460137FCF726
:105E800061FCEF2FD4D1039B93F8EF70B4B194F879
:105E9000EF804745324614BF0121002128460CBF40
:105EA00001240024FDF7B2FF002300930B4ACDF834
:105EB0000480072321462846FCF78CFC002300932E
:105EC000064A0197072321462846FCF73BFC07B00A
:105ED000BDE8F08FA24693E7A046C9E71AB30608CB
:105EE000F0B5054687B00846FEF74AF90B4604466A
:105EF00038B100231C491A46012007B0BDE8F04024
:105F000048E71A49194F02AA184648F06BFB03AE3E
:105F1000B8B1032C04D12846FDF7A4FA07B0F0BDB0
:105F2000FBF7DEF802AA46F8040B394600200134DC
:105F300048F058FBECE70E4832462146FCF7E4FCFB
:105F4000ECE7032CE7D1DDE90346059B01931A46F4
:105F50003146E0B235F0A0FC019B0028EBD1284689
:105F6000FDF7F8FFDAE700BFF87700209FB30608D7
:105F70001AB306082DE9F04F0F4689B016460021E6
:105F80001A460546FDF742FFDFF83CB10790B846D8
:105F900034464FF00009002E7ED021460C224046A8
:105FA00048F023FB0028079A14BF0121002128464E
:105FB0000CBF4FF0010A4FF0000AFDF727FF94F9DC
:105FC0000B20049294F90A200392B4F9082002925B
:105FD000B4F906200192B4F90420079000924B46D0
:105FE0005A4651462846FCF7F5FB98F90B200492D7
:105FF00098F90A200392B8F908200292B8F906200D
:106000000192B8F9042000924B465A465146284660
:1060100009F10109FCF796FBB9F1080F08F10C082A
:1060200004F10C04B7D1DFF8A49000240C2303FB87
:1060300004FA9EB34FF00008012303FA08FB56F858
:106040000A2057F80A3053403BEA030314BF0121EA
:10605000002112EA0B0F08D0CDF8008023464A46F3
:1060600028460791FCF7B6FB079957F80A301BEA58
:10607000030F06D0CDF8008023464A462846FCF799
:1060800061FB08F10108B8F10E0FD5D10134082CDD
:10609000CCD109B0BDE8F08FB246A6E7B04657F8BC
:1060A0000A20012303FA08F3134207D0CDF8008039
:1060B00023464A4601212846FCF744FB08F1010823
:1060C000B8F10E0FEBD1E1E72EB3060846B3060890
:1060D000F0B506468BB00846FEF752F80D4604466A
:1060E00020B300233F491A4601200BB0BDE8F04021
:1060F00040E72D2B03D0A3F13002092A4BD8052C01
:1061000005DD30460BB0BDE8F040FDF7ABB92846E1
:10611000FAF7E6FF0AAB621C03EB440424F80C0C0C
:1061200015F8013F303B092BFAD914462B78002B88
:10613000DFD1062CE5D1BDF81C20BDF91C30072AA3
:10614000DFD8BDF91E10A1F5FA7292B2B2F5FA6F5E
:106150001AD8BDF92040A4F5FA7292B2B2F5FA6FDE
:1061600012D8BDF92270B9420EDCBC420CDBA14250
:106170000ADCBDF924C00CF1640292B2C82A03D82B
:10618000BDF92650112D11DD174930460BB0BDE881
:10619000F040FDF750B9202B02D101352246C4E76B
:1061A00030460BB0BDE8F040FDF7D4BE0F4A0C20DE
:1061B00000FB03226DB2A2F89C18A2F89E48A2F838
:1061C000A07882F8A2C882F8A35800910021CDE9F6
:1061D00003C5CDE90147064A0846FCF7B3FA0BB000
:1061E000F0BD00BFE87800205BB3060850700020C7
:1061F0002EB306082DE9F04F89468DB016460021D2
:106200001A460746FDF702FEDFF8DCA0054600242B
:10621000C4EBC40309EB030259F803009188927997
:10622000089040F30748ADF824108DF82620B8F107
:10623000000F54D0002E55D0F218F0589188937961
:106240000A90ADF82C1007220AA908A88DF82E3064
:1062500048F0CBF900282A4614BF01210021384616
:106260000CBF4FF0010B4FF0000BFDF7CFFD9DF879
:106270002E3006939DF92D3005939DF92C30049313
:106280009DF82B3003939DF92A3002939DF8293015
:1062900001939DF8283000930546234652465946FF
:1062A0003846FCF797FA9DF8263006939DF925307D
:1062B00005939DF9243004939DF82330CDE90283A2
:1062C0009DF8213001939DF82030009352462346DB
:1062D000594638460134FCF735FA102C98D10DB0E8
:1062E000BDE8F08FB346DEE771B306082DE9F04F45
:1062F0009D4FDFF8A882DFF8A8928DB006460D46C4
:10630000284645F0A9FE034630B9984902460120C7
:106310000DB0BDE8F04F6DE7052239462846FAF783
:10632000EDFD0446C8B9924D0146702205F6F8000D
:1063300048F085F9C5F89848C5F8A448C5F8B048AC
:10634000C5F8BC48C5F8C848C5F8D448C5F8E04801
:10635000C5F8EC480DB0BDE8F08F04224146284650
:10636000FAF7CCFD044638BB2846F9F76DFF8246A4
:106370000028EFD045F070FEDFF828B202465BF847
:10638000041B39B97B492A4630460DB0BDE8F04FB1
:10639000FDF751B85046CDE90012FAF7AFFD019A6A
:1063A00040B9204629F0CAF90099734D4846FCF7D8
:1063B000ABFAA5E70134E2E7704907222846FAF76D
:1063C0009DFD074600287AD12021284648F04EF945
:1063D000044670BB6A486B4DFCF714FA2146284608
:1063E0000134FCF70FFA0E2CF8D1FCF7A7F9DFF80F
:1063F000B891654FDFF8B481002421464846FCF788
:1064000001FA0C26DFF8A8A166430025F2595F487F
:106410000123AB40134214BF414651460135FCF7FE
:10642000F1F90E2DF2D10134FCF788F9082CE4D1F2
:1064300090E75749564D03AA48F0D4F804AC002819
:1064400048D0022F11D1049A072A07D805990D299F
:1064500004D80378722B13D06E2B22D04D49082319
:1064600000223046FDF780FE74E7FAF739FE03AAF2
:1064700044F8040B29460020013748F0B3F8DEE762
:106480003B4B0C2000FB0233012000FA01F1D3F852
:1064900098080843C3F8980838493046FFF726FFA4
:1064A00058E7334B0C2000FB0233012202FA01F1C2
:1064B000D3F8982822EA0102C3F89828ECE7284686
:1064C0003349334F03AA48F08DF804AD0024A8B136
:1064D000082C03D13046FCF7C5FF3BE7FAF700FE76
:1064E00003AA45F8040B39460020013448F07AF835
:1064F000EDE729493046FCF79EFF2BE7082CE9D150
:10650000049B0F2BF5D8DDF814E0BEF1070FF0D88F
:10651000DDF818C0BCF10D0FEBD8079F07F164023E
:10652000C82AE6D8089DFF2DE3D809986428E0D84A
:106530000A996429DDD88842DBDA0B9C032CD8D871
:10654000C3EBC3020A4B134483F8FD1883F8F8E841
:10655000094983F8F9C883F8FA7883F8FB5883F877
:10656000FC0883F8FE4898E772AF060848790020D7
:106570005070002019AC060810B006088EB306084B
:10658000D4B8060896B30608E87800209BB306083E
:106590009FB30608A1B306085BB30608D0B206088D
:1065A000D5B2060814020608B7A5060859B30608AE
:1065B00049BB06082DE9F04F89B00C46079200212F
:1065C0001A460746FDF722FC0026079DDFF8A0B01B
:1065D0000690B2464FF019094FF46178079B43B318
:1065E00029460622204648F000F80028069A14BFE3
:1065F0000121002138460CBF4FF0010A4FF0000A7C
:10660000FDF704FC6A79069019FB028205922A794B
:1066100019FB02820492EA780392AA7802926A78BD
:1066200001922A78009233465A4651463846FCF782
:10663000D1F8627919FB02820592227919FB028254
:106640000492E2780392A27802926278019214F89E
:10665000062B009233465A46514638460136FCF71F
:1066600071F80A2E05F10605B8D109B0BDE8F08F22
:10667000A7B306082DE9F04F80468BB00846FDF71A
:106680007FFD8946074638B1002355491A46012047
:106690000BB0BDE8F04F8DE7524C084694F81A381D
:1066A00094F830B794F831A70793FAF719FD092841
:1066B000054600F38B800626464309F101008DF85C
:1066C0002770F9F7C1FD074658B1FAF709FD0D2803
:1066D00007D8A31983F8240A9DF8273001338DF8D1
:1066E00027303846F9F7B0FD074668B1FAF7F8FCED
:1066F000834509D3062303FB054383F8250A9DF848
:10670000273001338DF827303846F9F79DFD0746CD
:1067100068B1FAF7E5FC504509D8062303FB0543A9
:1067200083F8260A9DF8273001338DF82730384644
:10673000F9F78AFD074670B1FAF7D2FC079B83424E
:1067400009D3062303FB054383F8270A9DF8273066
:1067500001338DF82730DFF88890311D0DF12702C5
:1067600049443846FAF7C0FC9DF82730062B0BD079
:1067700009EB0602002349F8063040469380FCF7F7
:1067800071FE0BB0BDE8F08F03FB05444FF461715F
:1067900094F8292A192313FB0212059294F8282A47
:1067A00013FB0213049394F8273A039394F8263AC0
:1067B000029394F8253A019394F8243A0093002127
:1067C000094A2B460846FBF7BDFFDAE707490923CC
:1067D0003A4640460BB0BDE8F04FFDF7C5BC00BFE0
:1067E0007C690020585F0020A7B3060876B206082F
:1067F0002DE9F04F0F4689B0144600211A4606468F
:10680000FDF704FB0546002C00F0DB8022783B7886
:106810009A4218BF0121024608BF002130460CBF32
:106820004FF001084FF00008FDF7F0FA23789B4A7B
:10683000054641463046FBF7CDFF3B78974A414637
:106840003046FBF77FFF002C00F0BD8062787B783C
:106850009A4218BF01212A4608BF002130460CBFCA
:106860004FF001084FF00008FDF7D0FA63788C4A2A
:10687000054641463046FBF7ADFF7B78884A4146E6
:106880003046FBF75FFF07F1CA030493822304F14C
:10689000CA0B05934FF002094FF0000A3B785345AD
:1068A00000F39380002C00F0F38097F8EA3094F81E
:1068B000EA209A4218BF01212A4608BF002130462B
:1068C0000CBF4FF001084FF00008FDF79FFA94F855
:1068D000EA30744A054641463046FBF77BFF97F89D
:1068E000EA30704A41463046FBF72CFF07F1EC09CD
:1068F000002C00F0CF8004F1EC034A4604F1FC01C7
:106900004FF001089A4633F802CB32F8020B844567
:1069100018BF4FF000088B42F5D188F001012A46DC
:10692000C9B23046FDF772FA082105465046FAF71B
:1069300037FA5D4A034641463046FBF74BFF97F86E
:10694000EA104846FAF72CFA574A034641463046C1
:10695000FBF7F8FE002C00F09F804FF0FC094FF091
:10696000010807EB090104EB0900FAF7A3FA09F1A2
:106970000409002818BF4FF00008B9F58E7FF0D148
:1069800088F001012A46C9B23046FDF73FFA0821D6
:1069900004F1FC00F9F78AFC444A034641463046BC
:1069A000FBF718FF97F8EA1007F1FC00F9F77EFCF7
:1069B0003E4A03464146304609B0BDE8F04FFBF77A
:1069C000C1BEA04639E7A04657E7059B3B44069366
:1069D000002C5BD0059B0698234419460793FAF7D1
:1069E00069FA049B1A789BF800309A4206BFB0FA05
:1069F00080F84FEA58184FF000084B4609F1100292
:106A0000F85AE15A0233884218BF4FF00008934207
:106A1000F6D188F001012A46C9B23046FDF7F6F9F1
:106A2000627804EB090105469BF81800FAF78AF929
:106A300002909BF800300193079B00931C4A0AF1D7
:106A4000010341463046FBF7C5FE049B7A78187E69
:106A5000079307EB0901FAF775F9079B049A02906F
:106A60001B7801930132069B04920AF1010A0093FC
:106A70000F4A534641463046FBF764FE059B0933F7
:106A80000BF1010B09F11009059307E7A046DCE7BC
:106A9000A04624E7A04652E7A04683E7C0B3060815
:106AA000D2B3060800B4060818B406082FB40608C6
:106AB000E7B306082DE9F04F8FB0044602AA084656
:106AC000AF4947F08FFD064640B903460246AD493F
:106AD0004120FFF78DFE0FB0BDE8F08FAA49FAF70D
:106AE000E9F9074620BBA64902AA47F07BFDFAF761
:106AF000F7FA0828054606D9A44908233A4620464D
:106B0000FDF732FBE7E7A24C94F83037834202DC12
:106B100084F83057DFE7064604F5E6673146384625
:106B200031F0C0FE94F830370136B342F6DCEFE7BF
:106B300098493046FAF7BEF90546E0B9904902AAED
:106B400047F050FDFAF7CCFA0828064603D99249D7
:106B500008232A46D3E78E4C94F83137834202DC6F
:106B600084F83167B7E72846314601353FF02EFFFC
:106B7000082DF8D1F4E789493046FAF79BF9074622
:106B800000BB7F4902AA47F02DFD0028A3D0FAF7E9
:106B9000A7FA0828054603D9814908233A46AEE7F3
:106BA0007B4C94F81A38834209DD014604F5E6600F
:106BB00031F0C2FE294604F5E66031F0CBFE84F8E0
:106BC0001A5888E777493046FAF774F9054618BB32
:106BD0006F4BDFF8AC9193F81A7806AE014610229D
:106BE000304647F02CFDB046BD4202AA80F20E812D
:106BF0004946002047F0F6FC10B96B493A460EE1D1
:106C0000FAF76EFA013528F8020BEDE796E80F0067
:106C1000664C84E80F005EE765493046FAF74AF9AA
:106C2000054600283BD15A4B0DF1180893F81A98E5
:106C3000464607464F45524902AA4FF0000080F2EF
:106C4000F28047F0CFFC014610B95A494A46E6E0C7
:106C50000322304647F044FDB2464FF0000B304669
:106C600045F0FAF9584502D801370436E2E79AF8B8
:106C70000000FAF719F90BF1010B0AF8010BEEE726
:106C80004D494A46CBE041462046032231F0F2FD11
:106C90000135043408F10408AF42F4D11BE7474939
:106CA0003046FAF707F90546002840F0AC80384F27
:106CB000334997F8308702AA47F094FC00283FF444
:106CC0000AAFFAF70DFA461E01D4B04503DC3C4981
:106CD0004346012213E72A4902AA002047F082FC1A
:106CE000014600283FF4F7AE4FF00008082203A841
:106CF000CDE903888DF8148047F0F2FC0DF10C0902
:106D000003A845F0A9F940451CD81D4902AA002056
:106D100047F068FC00283FF4DEAE90F800A097F83A
:106D20003197DFF8ACB04FF000084D45144902AA86
:106D30004FF000007EDA47F055FC024658B9214971
:106D40004A466CE099F80000FAF7AEF808F101083D
:106D500009F8010BD4E7002D40D11378303B092B03
:106D60003CD919490192FAF7A5F8019A90B3104657
:106D70005946FAF79FF8019A002838D013494EE097
:106D80009FB306088866002046B406084CB406087F
:106D9000585F002057B4060860B406086EB40608B1
:106DA0007AB406088CB406087BB506087467002020
:106DB000B6B406089BB50608C2B40608E0B40608D7
:106DC000E5B40608BBB506087AA40608F8B40608B8
:106DD000F1B406084FF001084FF0FF35104601925C
:106DE000FAF77EF90028019A03DA214917E0A8464C
:106DF000F2E70EAB03EB4503013523F8200C94E7D3
:106E00001C494A460BE01C49324608E01B49002059
:106E100047F0E8FB00283FF4F9AE19493A4620460E
:106E2000FCF709FB57E647F0DDFB00287FF428AFAD
:106E3000144C31E747F0D6FB0028E1D1124C06EBA9
:106E4000C6008230082203A9204431F013FD5046C9
:106E5000FAF72AF837446A0087F8FA0704EB0610B5
:106E600006A9023047F088FB87F8128833E600BF96
:106E70002DB5060842B5060865B506089FB3060895
:106E800098B4060884670020886600202DE9F04F3A
:106E900089B00F4691460021139A98460646FCF7A2
:106EA000B5FF87EA09096FEA0903DFF884900693C2
:106EB0000446002528460BF03DFB129B184230D0BB
:106EC000069BDFF870B0034014BF4FF0010A4FF08B
:106ED000000A049310EA070314BF4A465A4628469C
:106EE000059307920BF038FB079A039000904346F6
:106EF00051463046FBF76EFC049BB3FA83F1224601
:106F000049093046FCF782FF059A039B009304462B
:106F10004346002A14BF5A464A4651463046FBF7BC
:106F200011FC0135182DC5D109B0BDE8F08F00BFA7
:106F3000CAB20608E0B5060837B50446084601910E
:106F400045F08AF80199054602462046F9F7D6FF32
:106F500070B9625D1046F9F797FF00B932B9013593
:106F60002C44204601340378202BFAD003B030BDE6
:106F70000020FBE7F0B5032985B005460C46164610
:106F800014D80B4F3970FBF7D9FB0A492846FDF797
:106F90005BFD0949224601A8F9F778FE01AB3246AC
:106FA00008212846FCF760FFFF233B7005B0F0BDC9
:106FB0001005002010B00608C6B10608F0B5032978
:106FC00085B005460C46164614D80B4F7970FBF772
:106FD000B5FB0A492846FDF767FD09492246684680
:106FE000F9F754FE6B46324610212846FCF73CFF69
:106FF000FF237B7005B0F0BD1005002010B006081F
:10700000C2B1060810B586B0104B0493104B039321
:10701000104B0293104B0193104B1149114A0093EE
:107020000446114B1148FBF7EDFBFBF787FB1049BA
:107030001048FBF769FC3CB10F4A1049104806B0F4
:10704000BDE81040FBF760BC06B010BD27B60608CF
:107050002CB6060836B606083FB60608BBA70608D3
:10706000F1B50608E7B50608675F0020FCB506081D
:107070004BB6060853B60608FC5E0608F45E060822
:1070800064B606080120BDE72DE9F04F0A4687B037
:1070900000210646FCF7BAFE3B4C05903B4A23789C
:1070A000608802EB8303D3F830ABF9F735F98368D6
:1070B0000493374BC16893F88420002A4BD0DDF845
:1070C00010800491002721796279049B07FB01223B
:1070D00013F80290B8F1000F3FD018F80250059A4B
:1070E0004D4514BF0121002130460CBF4FF0010B6C
:1070F0004FF0000BFCF78AFE013705907DB305F0D9
:107100000F022D0940350292CDE90075214A534600
:1071100059463046FBF75EFBB9F1000F2AD009F063
:107120000F024FEA1919029209F14002CDE90072EB
:107130005346184A59463046FBF704FBA279012A08
:1071400038BF0122BA42BEDC134B0834A342A5D19A
:1071500007B0BDE8F08F9046B4E74546BFE7B8F109
:10716000000FD9D00D4A0097534659463046FBF7D9
:1071700031FBD1E77306E1D4084A009753465946DC
:107180003046FBF7DFFAD9E7B4030608A4F905088F
:10719000585F002091B60608D4040608A7B6060872
:1071A00038B50C4B03EBC0050C4695F8102A0A487D
:1071B00003EB8203D3F8301BFBF724FB95F8163A58
:1071C00033B1611C0548BDE83840C9B2FBF71ABBB2
:1071D00038BD00BFA4F90508D3B80608B6A506084F
:1071E00073B50E4611490546F9F764FE18B93070BB
:1071F000012002B070BD2C78602C8CBF613C413CFA
:10720000072C10D8013501230A2201A92846F9F7D5
:10721000C5FE019B9D4206D00F2804D8013440EAE8
:1072200004143470E4E70020E3E700BFF6B6060874
:107230000246531C084605D1044B1A681B790A60A4
:107240000B7170470249F9F721BD00BFF6B6060879
:10725000B7A506082DE9FF471E46C368BDF8307084
:10726000DDF8348004468946924643B3CBB20D2BF9
:107270009ABF1A4AD5560025BAF1FF3F21D023689C
:10728000174A3146CDE9005A3846C0475246207960
:107290005FFA89F1F3F758FC024600B10288D3B2D5
:1072A0000393C2F30323120BCDE9005202930D4A5C
:1072B000236831463846C04704B0BDE8F0874D1C0E
:1072C000DAE77B06F8D42368074A0C95314638463E
:1072D000C44604B0BDE8F047604700BFE45E06085E
:1072E000BBB60608C8B60608ECB606082DE9F0419C
:1072F000154686B06A1C8846BDF830600D9F194659
:1073000023D0030900F00F044033CDE90045164AAD
:1073100005933046B847A8B198F80510D8F8000092
:107320002A46F3F759FC68B1028801780391C2F349
:107330000321120BCDE900420291059B0B4A00216B
:107340003046B84706B0BDE8F0817306FAD40309A9
:10735000074A00F00F000C9040333046BC4606B0A0
:10736000BDE8F041604700BFFBB606080DB7060850
:1073700036B706082DE9F04F2DED028B0A468BB08B
:1073800000218246FCF742FD6F4D814605F1800BDE
:1073900000266E4B93F88440AB7AB34200F395809D
:1073A0001035AB45F4D140F21620F8F7B5FFD0E91F
:1073B00002530CB12C461D460DF1100B1522002175
:1073C000584647F03CF900272E78002E44D06978C3
:1073D0000391304605F0C6FF95F9023002935A1C1E
:1073E000534208EE100A5341002C00F0A980039983
:1073F000002214F802C0B44504EB020040F09C8067
:1074000090F90280029A424540F0948042788A4284
:1074100008BF012301220BF8072003F001034A46AD
:1074200083F0010150460393FCF7F0FC039B814677
:107430004CB1474A18EE101ACDE900A23046424638
:10744000FFF754FF039B434A18EE101ACDE900A240
:107450003046029AFFF74AFF0137152F05F1030561
:10746000B2D16CB33A4FDFF8EC8004F13F061BF861
:10747000013B02930BBB2078F8B194F90220013252
:107480001BD0617805F06EFF4A4605460121504643
:10749000FCF7BCFC94F90220029B29468146207827
:1074A000CDE900A7FFF722FF2078029BCDE900A8D5
:1074B0004FF0FF322946FFF719FF0334B442D6D10B
:1074C0000BB0BDEC028BBDE8F08FE888F8F724FF25
:1074D000D0E902230CB114461A46297A6B7A06FBCE
:1074E000013312F9038014B3E756B8450CBF0123EA
:1074F00000234A4614BF0121002150460293FCF7A5
:1075000085FC029B814644B1114A3146CDE900A277
:1075100028463A46FFF79EFE029B0E4A3146CDE9C9
:1075200000A228464246FFF795FE013631E74FF0AC
:10753000FF37DAE700236DE703323F2A7FF459AFC4
:107540004FF0FF386BE700BF64050020585F002054
:10755000D527010845270108224BB0F5FA6F1A68B4
:107560000346A8BF4FF4FA63B3F57A7FB8BF4FF470
:107570007A73D20416D540F2DC52904215D007EE51
:10758000903A40F2DB529042F8EE677A1FD8DFED76
:10759000166A9FED167A9FED160A77EEE67AA7EE49
:1075A000870A7047B0F57A7F02D89FED120A7047BC
:1075B00007EE903ADFED106A9FED107A9FED100A0A
:1075C000F8EE677A77EEE67AA7EE870A7047DFED86
:1075D0000D6A9FED0D7A9FED0D0A77EEE67AA7EE24
:1075E000870A7047F864002000007A44D62000C063
:1075F00000E082440000000000407A446610004031
:107600000000404200A0BB44D6200040000083445C
:1076100010B584464FEA810E102312F4004F14BFB8
:107620000E2407245200013BCCF8004092B2F444EF
:10763000F3D100EB81128C01035142F8213012206A
:1076400010BD00BF10B584464FEA810E0424130B11
:1076500003EB430318331201013CCCF8003092B223
:10766000F444F4D100EB01130A01845043F82140A3
:10767000062010BD704700BF704700BF034B00EBF2
:10768000400003EBC000407C704700BF480500107D
:1076900000233D22027043708370C370704700BFA7
:1076A000704700BF00207047704700BF0020704740
:1076B00001207047704700BF704700BF704700BF90
:1076C000704700BF9FED010A704700BF0000000037
:1076D0000020704703681B69184730B5084B00222B
:1076E00093F900405D7801190132CD729D780555FE
:1076F000062ADC788C7503F10403F1D130BD00BF9C
:10770000C4320608002383700370C370437070474F
:10771000C36B33B15B68426D9BB29A4205D3D01AFA
:107720007047D0E907239A42F9D2C0681044C01AC2
:10773000704700BFD0E909120369914238BFC918E8
:107740008A1A016C39B14968013B12FA81F29342FD
:1077500004D9981A7047013B981A70470020704767
:10776000036C13B190F864007047D0E90903181A4C
:10777000B0FA80F040097047C26B10B4034662B1A2
:10778000426DC1685C69881A013A205C5DF8044B5F
:1077900008BF0A46C0B25A657047006A5C69411C5E
:1077A000205CDC68A14238BF0A46C0B25DF8044BD9
:1077B0001A627047836E70B504460D460BB1984748
:1077C000B8B1636AA269D554636A2169226C013336
:1077D0008B4228BF0023636232B3EFF31183502240
:1077E00082F31288226C1168C90703D5DBB283F3D8
:1077F000118870BD516889B271B9D4E909508542C8
:1078000018D0A6690644D66018D9281A80B25060EC
:10781000A562002184F86410116841F00101DBB217
:10782000116083F3118870BD226ED36843F080032A
:10783000D36070BD012284F86420D7E72569281A37
:1078400080B25060A162E4E7836E03B118477047CD
:10785000F8B590F87C30012B1CD0002A164619DDB3
:107860000269436A05460F46D41AB442A869A8BF04
:10787000344639461844224646F07EFE6B6A2A6931
:107880002344361BB3FBF2F0002E02FB10336B6275
:107890002744E9DCF8BD00BF90F87C30012B0DD007
:1078A000036C43B3EFF31183502282F31288026C0E
:1078B0001168C90703D5DBB283F31188704751689B
:1078C00089B270B471B9D0E90954A54219D086695A
:1078D0002644D6601CD92C1BA4B2546085620021BA
:1078E00080F86410116841F00101DBB2116083F38C
:1078F000118870BC7047026ED36843F08003D36078
:107900007047012280F86420DBB283F31188F0E72E
:1079100005692C1BA4B254608162E0E7084900238A
:1079200001E0152B09D003EB4302013311F802C02B
:1079300084450A44F5D1104670470020704700BFC7
:107940000024002070B5094C236873B10546002659
:1079500006E099681A681E7321609047236823B176
:107960005A68AA1A002A1846F3DA70BD7CAB0020C8
:1079700008B5254B1B68DB040AD5B5EE400AF1EECD
:1079800010FA12D19FED210A46F07EF880B208BDB0
:10799000DFED1F7AB4EEE70AF1EE10FA1CDA9FED84
:1079A0001D0A46F071F880B208BDDFED197AB4EE19
:1079B000E70AF1EE10FAE5D49FED177AB4EEC70AA4
:1079C000F1EE10FA14D870EE677A9FED147A9FEDFD
:1079D000140AA7EE870AE4E770EE677A9FED117A42
:1079E0009FED110AA7EE870A46F04EF880B208BD57
:1079F000DFED0E7A9FED0E7A70EE677A9FED0D0A3D
:107A0000A7EE870ACDE700BFF86400200080BB44E2
:107A10000000404200007A4400E0824466BEFFBE9F
:107A20000060BB4438DFFF3E00407A4400008344DE
:107A300066BEFF3E00A0BB442DE9F04F6D4B1B78A6
:107A400087B0002B00F0D0806B4D6C48A968DFF840
:107A5000F0A1FAF759FF69686948FAF755FF694BD1
:107A60006948D3E90031C91A684B5A68B1FBF2F290
:107A7000FAF74AFFFAF762FE6548FAF777FE6548BB
:107A8000FAF774FE4FF00008634B1B785FFA88F436
:107A9000A34222D8614C624FFAF750FE26460025D9
:107AA00056F8041B38460135FAF7ACFE162DF7D10F
:107AB000FAF744FE5A4E0125234661681B6830469A
:107AC000C91A0135FAF79EFE162D04F10404F3D10C
:107AD00007B0BDE8F04FFAF731BE524B142603EB66
:107AE000840306FB045693ED000AB6F80E9045F0A9
:107AF000CBFF96F81EE01EF0010F14BF52222D227C
:107B00001EF0020F14BF54232D231EF0040F07EEA6
:107B1000903A14BF56232D231EF0080F14BF4FF0C8
:107B2000430C4FF02D0C81B21EF0800F4FF03C0B38
:107B3000B1FBFBF105914FF0640114BF4FF0530E00
:107B40004FF02D0E80B201FB09F1671CCDE902E177
:107B50000093049017EE903ACDF804C03946504691
:107B6000FAF750FEB37FDB073AD55C232E4A634316
:107B7000D118D05891ED010A70B1DFED2C7AB8EE32
:107B8000400A20EE270A07EE900AF8EE677A80EEA8
:107B9000270A45F079FF00B2642290FBF2F102FB64
:107BA00011022348FAF72EFE142101FB075701FBAF
:107BB0000454F988628A0491218B0391E18A02912D
:107BC000A18B0191A18A009102F0030319214B437B
:107BD0001848218A9208FAF797FE08F1010853E73E
:107BE0001548FAF78BFDDFE7144807B0BDE8F04F02
:107BF000FAF7BCBD04000010200900104AB70608BF
:107C00005AB706083406001071B706087CAB00208E
:107C10009EB70608FAB7060850100010CC090010ED
:107C2000AAB80608F81500104006001000401C46CF
:107C300073B8060888B806087FB80608AEB8060804
:107C400056B806082DE9F84F1F4DDFF88490DFF88D
:107C500084A006460C4636274FF000082046FCF765
:107C60008FFAD5F800B048B921465846F9F76AF9B5
:107C700020B968682146F9F765F980B15846FAF7E6
:107C80003DFD696811B15046FAF7BCFDA96811B114
:107C90004846FAF7B7FDFAF751FD4FF00108013FEA
:107CA00005F11005DAD12046FCF76AFA48B9B8F1B7
:107CB000000F06D1224630460449BDE8F84FFBF7D5
:107CC000BABBBDE8F88F00BFDC320608D6B806089C
:107CD000D0B80608CAB80608F2F7C4BA10B5044608
:107CE00045F0D2FE81B22046BDE81040F2F7BABAA4
:107CF00070B50468236A1B69054643B1236AD0F84E
:107D000094001B69984701282AD002280DD0236AC5
:107D1000DA699AB9586958B399692162BDE8704027
:107D2000C3E90522F2F756BC2362236ADA691433E9
:107D3000002AF9D1236ADA69002AEBD0216A94F883
:107D400024200E7B1433F6B22362D2B996B92846AA
:107D5000F2F7C4FB28460121BDE87040F2F786BB6C
:107D6000236A143B014623622846F2F77FFBCEE7E5
:107D7000206270BDAB68002BE9D01A689B885383E2
:107D8000E5E700212846F2F771FB002384F8243050
:107D9000002EDCD0EEE700BF8069002834D00368F5
:107DA0001A6A127B1ABBD3E904125B6849686AB18C
:107DB00010B4546800220A6022609A885DF8044B6F
:107DC00022F003021204120C9A8091E71A8912061B
:107DD000FCD41A89D20708D400220A609A8822F0BB
:107DE00002021204120C9A8082E79A89F1E78268F3
:107DF000002AD8D0116892880A83D3E904125B68FC
:107E00004968002AD4D1E1E7704700BF806900B912
:107E10007047016830B4D1E904424B68646872B1BC
:107E20005568002222602A609A8822F00302120418
:107E3000120C9A800B6A1B7B9BB930BC58E71A89DD
:107E40001506FCD41A89D20713D4002222609A881E
:107E500022F002021204120C9A800B6A1B7B002B88
:107E6000EBD08368002BE8D01A689B88138330BC62
:107E70003EE79A89E6E700BF30B50446006E838985
:107E8000A16023F400531B041B0C838195B063791C
:107E9000009113F0040F21794FEA03324FEA0323D4
:107EA00003F48063ADF8083001F0010302F40052DE
:107EB00014BF4FF480550025002B4FF00003ADF8A0
:107EC0000620ADF80C3007BF002208230C23042243
:107ED000ADF804508D07694654BFADF80A20ADF8DF
:107EE0000A303DF0D3FB6279236ED00700F18A801F
:107EF00012F0080F9A8A7FD092B242F008029A825A
:107F00009A8992B242F400529A812279D10732D5ED
:107F1000E06B002800F088800023E26D0793CDE934
:107F20000B33CDE90F33CDE911334FF4807509934D
:107F30006369E1680D9505920693626C04924FF4B3
:107F400080634FF480350A9308910E953DF054F903
:107F500004A9E06B3DF0E6F9E16B236E0A6842F09C
:107F600001020A609A8A92B242F040029A824968FB
:107F7000227989B26165920737D5206C00285FD0DD
:107F80002369A26D0893A36CCDE90432002240233B
:107F90000025CDE906234FF480314FF480630A9326
:107FA0000E91CDE90B55CDE90F55CDE91155099548
:107FB0000D953DF021F9206C04A93DF0B3F9226C38
:107FC000236E506940F080005061106840F0160048
:107FD000106055609A8A92B242F0800203F10C015F
:107FE0009A820A6842F040020A609A8992B242F488
:107FF00000529A8115B030BD22F008021204120C12
:108000009A827DE71D498B4223D0A1F54C418B42DA
:108010001DD001F580618B421DD102200121F2F7B4
:10802000B3F86279236E63E74FF6DF711980D96880
:1080300041F02001D960D96841F01001D9609AE778
:10804000DA6842F0800203F10C01DA60C9E701202E
:10805000E4E70020E2E701F580618B420AD001F5F8
:1080600080618B4208D001F544418B427FF440AFE0
:108070000520D3E70320D1E70420CFE7001001401B
:1080800030B50446006E21718389A26823F4005341
:108090001B041B0C8381637995B013F0040F0092CD
:1080A00014BF4FF480520022ADF804201A031B02C3
:1080B00003F48063ADF8083001F0010302F40052CC
:1080C000002B4FF00003ADF80620ADF80C3007BFD1
:1080D000002208230C2304228D07694654BFADF803
:1080E0000A20ADF80A303DF0D1FA6279236ED0074C
:1080F00000F18A8012F0080F9A8A7FD092B242F083
:1081000008029A829A8992B242F400529A812279A4
:10811000D10732D5E06B002800F088800023E26DA3
:108120000793CDE90B33CDE90F33CDE911334FF48C
:10813000807509936369E1680D9505920693626CF9
:1081400004924FF480634FF480350A9308910E95A2
:108150003DF052F804A9E06B3DF0E4F8E16B236ECA
:108160000A6842F001020A609A8A92B242F0400222
:108170009A824968227989B26165920737D5206C65
:1081800000285FD02369A26D0893A36CCDE9043267
:10819000002240230025CDE906234FF480314FF41F
:1081A00080630A930E91CDE90B55CDE90F55CDE9CA
:1081B000115509950D953DF01FF8206C04A93DF06F
:1081C000B1F8226C236E506940F080005061106855
:1081D00040F01600106055609A8A92B242F0800218
:1081E00003F10C019A820A6842F040020A609A89FF
:1081F00092B242F400529A8115B030BD22F00802CA
:108200001204120C9A827DE71D498B4223D0A1F5FE
:108210004C418B421DD001F580618B421DD1022063
:108220000121F1F7B1FF6279236E63E74FF6DF7149
:108230001980D96841F02001D960D96841F0100156
:10824000D9609AE7DA6842F0800203F10C01DA6043
:10825000C9E70120E4E70020E2E701F580618B42F5
:108260000AD001F580618B4208D001F544418B4270
:108270007FF440AF0520D3E70320D1E70420CFE708
:1082800000100140B04B1B6893B32DE9F0475B69C8
:1082900086B0984748B3AD4DD5F8CC36002B01DDFC
:1082A000F7F720F8AA4C6378022B22D0032B1CD1BD
:1082B00095F8E83713B1A748F7F78EF895F8D43654
:1082C00013B1A548F7F788F895F8183713B1A34804
:1082D000F7F782F895F85C373BB1A14806B0BDE8E6
:1082E000F047F7F779B80323637006B0BDE8F0876D
:1082F0007047A37804F1040804F1080704F5BD569B
:10830000072BF2D801A252F823F000BFA583010881
:10831000D5840108CF830108998301082D830108C2
:108320005384010867840108E78201082378207DCF
:10833000032B0CBF4FF080094FF480794FF0010AF6
:10834000002800F0B2800128FAD1D5F840386268E0
:10835000D5F83818580202314FF0FF33B3FBF0F371
:108360009A184FF0000343EB03009142834138BF5A
:108370000A4602203946F5F7B1FF032800F284814E
:1083800001A353F820F000BFEB8201087F840108AD
:10839000EB8201087F84010895F8A037002BA4D058
:1083A00070489BE7002305A9092218460391F5F7B9
:1083B0003FFE012899D1059B93F8FE21552A00F034
:1083C000D7800222012385F8E42763708DE7664B8E
:1083D00000930322A270654962483023052243F0CE
:1083E00081FC82E723690622652BA2703BD92278A3
:1083F000032A0CBF6FF07F026FF0FF02A3F1650349
:1084000003EA020303F101030CBF80224FF48072E0
:108410009A42236127D2E268D5F8381898180231B9
:10842000884207D395F8E41711B9012185F8E417BC
:1084300001216170C4E90120C5F8C427D5F840289E
:1084400002FB03F35B02C5F8A837C5F8AC37052378
:10845000A370A26841460120F5F7DCFF012840F037
:10846000CA800623A37000213046F6F78FF8012852
:1084700040F0C180A3780133DBB2A37040E7D4E9B8
:1084800001C32269A3EB0C01914288BFC4E903C177
:108490000328A7D00133B3FBF9F209FB12320AB16A
:1084A0004B449B1A002063602075D5F8382841465C
:1084B0000232F5F713FF032800F2E68001A353F818
:1084C00020F000BFEB8201083D850108EB82010826
:1084D000E5830108D5F82C0805A900230922F5F742
:1084E000A7FD01287FF401AF0022059B2270B3F89D
:1084F0000B20B2F5007F1BD11A7C022A18D193F809
:10850000FE21552A14D193F8FF21AA2A10D1B3F8DD
:108510000EC0D5F82C686644C5F830685F7BC5F896
:1085200040787A1E7F2A03D87A4237EA02026AD05C
:108530000322012385F8E4276370D6E6636884F894
:1085400014A00133A360FBE69820002068400020BF
:1085500068300020504800203C4700208047002021
:10856000C447002008480020198E0008B4BE060841
:1085700093F8FF21AA2A7FF424AFD3F8C6210399E8
:108580004AB193F8C201A0F10B06012E2DD900F0DB
:10859000F700062829D0D3F8D6214AB193F8D201A2
:1085A000A0F10B06012E20D900F0F70006281CD000
:1085B000D3F8E6214AB193F8E201A0F10B06012EAF
:1085C00013D900F0F70006280FD0D3F8F621002ABF
:1085D0003FF4F7AE93F8F231A3F10B00012804D970
:1085E00003F0F703062B7FF4ECAE0123C5F82C282B
:1085F000A370104671E702287FF477AE012385F857
:10860000E437637071E67A02013AC5F84828D88ADF
:1086100000B9586AC5F83408B3F81120520102F2C3
:10862000FF125212C5F85028B3F8131001B9196A95
:1086300094440CEB400CA1EB0C01B1FBF7F140F6BC
:10864000F477B9424FEA4000C5F8381819D94FF607
:10865000F477B94211D903212170DB6AC5F84C388F
:10866000324495F810381044C5F83C080BB9F6F7B9
:10867000A7FFA3780133A37037E6022323700023FA
:10868000ECE70123237053E7207D59E62DE9F84FED
:10869000A04C237ADB072DED028B80466BD59E4BD9
:1086A000657A1F889D4E012D56D0022D35D0002DA4
:1086B0003ED094ED078AF37B33B1B38923B1984B55
:1086C0001B78002B40F0CB80A27AAA4238BF2A4602
:1086D000317A632906D8022D00F0DE80237D002B3D
:1086E00040F0ED808F4BDFED906A1A70D4E90B30CB
:1086F00023631B1A07FB03F307EE903AF8EEE77AC1
:10870000B0EE487AA7EEA67AB17B84ED077A00290D
:108710005FD1BDEC028BBDE8F88FE389BB42C8D2C4
:10872000824B94ED078A1B68236201256572C2E7BC
:10873000238ABB4219D37D4B216A1A68F37D03EB70
:10874000830303EB8303521AB2EB830FB1DB0125E2
:1087500094ED078A6572AEE7638ABB4280F08A8037
:10876000A389BB423CBF00256572704B94ED078A1C
:108770001B6823629FE7657ADFF89C91EB1E012B53
:1087800033D9B9F80800C0F30B0044F091F9092877
:1087900040F3AA80614EB9F80070F3889F4203D37A
:1087A0003288BA42BFF47FAFB7EB430F3FF77BAFDE
:1087B0000323DFED5F7A5A4A6372A3720023B0EE9F
:1087C000678AC4ED077A1370A381E38123826382F1
:1087D00081E0012A00F08180022A9AD1BDEC028B4F
:1087E0000720BDE8F84F0AF015BB4C4EB9F80070F1
:1087F000F3889F4202D33288BA4202D2B7EB430FCA
:1088000065DDB9F80800C0F30B0044F051F9092800
:108810007CDD337D00256572A572002B00F08E8013
:108820003F4A137099B2B288738812FB01F213FBAE
:1088300001F3717C92B28A429BB2A28186BF521A26
:1088400092B200228B42E38186BF5B1A9BB2002367
:1088500063826423637500232282A36123E712F0FD
:10886000E9FD002844D102239D422A46A37238BF65
:108870001A462DE72D4B216A1A68337E03EB8303DA
:1088800003EB8303521AB2EB830FFFF612AF0225FC
:1088900094ED078A65720EE7207D80B90123C4F844
:1088A00018802375234BC1F1640100FB01F183FBA8
:1088B0000103C917A1EBA3516431617512E7A069E7
:1088C0001D4BA8EB00009842ECDB61750AE7032D15
:1088D00079D194ED078A0325EDE6BDEC028B0820E3
:1088E000BDE8F84F0AF096BAB9F800700B4EDAE618
:1088F000337C834206D301239D422A46A37238BFAC
:108900001A46E5E60023A3722A46E1E6032DE0D0ED
:10891000CFE600BF7CAB0020B8750020FC640020CF
:10892000B7750020B6750020ACC527379C20002005
:10893000000000006BCA5F6B80969800274A284DA4
:10894000126892F96C103288B7FBF2F20132082AF1
:1089500028BF08225FFA82FC914285F800C02AD025
:1089600049B3204991F800E00EF1010101F0030143
:10897000714520D0DFF870B04FF0FF304FF0A40AFF
:108980000AE0B0F1FF3F02D1002B08BF08460131D9
:1089900001F00301714511D00AFB01B393F96C306A
:1089A0009A42EED10846C0B2F9F732FB2B78B9F8FB
:1089B0000070657A36E71D46634633E7431CF2D103
:1089C000634600252EE7B9F80800C0F30B0044F019
:1089D0006FF809283FF7DFAE6BE600BF8063002029
:1089E000B7750020605F0020C06000202DE9F843CB
:1089F000CD4CA36820469847002800F08F80B4F93A
:108A00000E30A17D06EE903AB4F9103007EE903AA0
:108A1000B4F9123007EE103AF8EEE66AF8EEE77AAB
:108A2000B8EEC77A0123092984F85430C4ED126ADC
:108A3000C4ED137A84ED147A72D004F1480027F063
:108A4000A9FFBA4DAA8DAB6A002A40F0F980B84A56
:108A50001268520700F1C180B3F9002094ED125A58
:108A600094ED136A94ED147A05EE902AB3F902207E
:108A7000B3F9043006EE902A07EE903AF8EEE55A84
:108A8000F8EEE66AF8EEE77A75EE655A76EE666A13
:108A900077EE677A2B88C4ED125AC4ED136AC4EDE1
:108AA000147ADBB395ED025A95ED056A95ED087AD7
:108AB000D5ED033A95ED064AD5ED094A75EEC55A4E
:108AC00076EEC66A77EEC77AA5EEA35AA6EE846A5A
:108AD000A4EEA77AD5ED015AD5ED046AD5ED077A53
:108AE00085ED025A35EE652A76EE662A37EE673A4C
:108AF000E3EE825AE2EE846AE4EE837AC5ED015A2F
:108B0000C4ED125A85ED056AC5ED046AC4ED136A19
:108B100085ED087AC5ED077AC4ED147ABDE8F883CF
:108B2000D4ED0B5A94ED0C6A94ED0D5AD4ED094A2C
:108B300094ED084A7F4B67EEA55A27EE866A67EEEA
:108B4000857A94ED0A5A1B78A6EEA46AE6EE845A5A
:108B5000E6EE857AD4ED0E6AD4ED0F4A94ED105A04
:108B6000E6EE875AF0EE466AE4EE876AE5EE077AAB
:108B7000C4ED125AC4ED136AC4ED147A002B7FF4CD
:108B800060AF6D4B93ED055A93ED036A93ED047A54
:108B9000D3ED014A93ED004A26EE866A26EE877AE7
:108BA00066EE856A93ED025AA5EEA47AE5EE856A33
:108BB000A5EE846AD3ED064A93ED075AD3ED085A21
:108BC000A7EEA46AA7EE857AE7EEA56A84ED126A9D
:108BD00084ED137AC4ED146A33E7584EB6F840209A
:108BE000322A63D0002A40F0CD8096F85E20002A19
:108BF0003FF432AF06F1500007C8514F4FF0000C60
:108C000087FB028E86F85EC0D217A689C2EB2E12B1
:108C1000921B9A8087FB0062C017C0EB221087FB73
:108C20000127C917C1EB271118805980454B012234
:108C3000A3F80EC0C3F80A20F9F7D2FBAB6A0BE722
:108C4000B2F5C87F00F082803C4994ED127AD1EDF4
:108C50000D6AD4ED137A94ED146AF8EEE66A0026F4
:108C600076EE876A91ED0E7AA664B8EEC77AFDEECD
:108C7000E66A37EE277AD1ED0F7AC1ED0D6AF8EE8C
:108C8000E77ABDEEC77A77EE867A0020FDEEE77AC6
:108C9000012A188081ED0E7AE6645880C1ED0F7AC2
:108CA0002665988073D0013AAA85D0E61A68726466
:108CB000B3F90420A6F84820224ADFED237AD268CF
:108CC000F26494ED127A0020002177EE877AA06496
:108CD0001980B6F84020FDEEE77A322AC6ED147A04
:108CE00000F0828096ED157AD4ED137AD4ED146AF3
:108CF000E064B8EEC77A012A37EE277AD6ED167A05
:108D00005980F8EEE77ABDEEC77A77EEA67A20654D
:108D1000FDEEE77A998086ED157AC6ED167A74D065
:108D2000013AA6F8402060E7E4140010AC110010EE
:108D3000F8640020410500202C6900207CAB002055
:108D40001F85EB514C65002000000000D4ED126A35
:108D500094ED137AD4ED147A354EFDEEE66ABDEE4D
:108D6000C77AFDEEE77A00200021A064C6ED0D6A07
:108D7000198086ED0E7AE0645980C6ED0F7A206581
:108D8000998090E7D6ED147AF8EEE77A99E717EE36
:108D9000906ADFF8A4E0B4F80C80C8368EFB0619A0
:108DA00016EE90CAF11717EE107AC1EBE9110CF12B
:108DB000C80CA1EB08019980C8378EFB0C614FEA03
:108DC000EC7CCCEBE11C8EFB071EFF17C7EBEE170C
:108DD000A3F800C05F80174BC3F80A20D881F9F7C9
:108DE000FFFAAA8DAB6A5EE794ED137AD4ED147A9C
:108DF000E064BDEEC77AFDEEE77A598086ED157A1C
:108E00002065C6ED167A99808AE70B2086F85D20EA
:108E100086F85C1009F0FEFFAB6A726C1A60B6F956
:108E200048209A80034AF16CD160B6F8402077E779
:108E30007CAB00204C6500201F85EB5138B5074CFA
:108E4000074DAC4203D3074B01221A7038BDD4E959
:108E50000210A28845F090FB1C34F2E790EC060863
:108E60006CF50608DC5F0020302821D0312826D0A0
:108E7000322828D0332828D0342828D0352828D0A4
:108E8000202828D0212828D0102828D0112828D000
:108E9000122828D0132828D0142812D0152826D01C
:108EA000162826D0172808BF0F2202D000207047AE
:108EB0000022114B03EBC20393F87C03704701229D
:108EC000F7E70C22F5E70222F3E70322F1E7042299
:108ED000EFE70522EDE70622EBE70722E9E70822A4
:108EE000E7E70922E5E70A22E3E70B22E1E70D22A3
:108EF000DFE70E22DDE700BFC43206080123302879
:108F000003FA01F129D031281ED032281CD0332891
:108F10001AD0342813D0352811D020280FD021287A
:108F20000DD0102810D011280ED012280CD01328E4
:108F30000AD0142803D0152801D0162809D111F021
:108F4000030018BF0120704711F0070018BF01206F
:108F500070471728F3D00020704711F0070018BFA2
:108F600018467047244B82B09A79019092B393F8D7
:108F70002630DFED226A224A07EE903AF8EEE77AD1
:108F8000204B127886EEA77A83ED187A02B31E4939
:108F90009FED1E6AB1F86A10DDED017A07EE101A36
:108FA000B8EE477AF8EE677A27EE067AF7EE006AAF
:108FB00027EE277A203377EE266A0021C7EE267A3D
:108FC00003EBC2021960083343ED017A9A42F9D1EA
:108FD00002B070470E4A12681201F9D593F8263094
:108FE000DFED066A07EE903AF8EEE77A054B86EE7B
:108FF000A77A83ED187AEBE79C270020555555405A
:1090000050100010F81500107CAB002027D4D23689
:10901000F864002010B5437B82680446581C6073D6
:10902000D154627B237B934206D82AB12368D4E9CA
:10903000010198470023637310BD00BF427B42B11A
:1090400010B503680446D0E9010198470023637313
:1090500010BD704730B5056895F800E0BEF1010F0E
:1090600095B004468C4608D0BEF1020F02D11946D5
:109070002B6AB3B1002015B030BD95F90450691CBE
:10908000F8D0022DF6DC0179009228466246F2F70C
:109090006BFD0028EED0284615B0BDE83040F2F751
:1090A000DBBCCDE90A210DF10F0204920122CDE9CA
:1090B0000532CDE908336CF07F018DF81C308DF856
:1090C00030208DF844200D9310931293002200233A
:1090D000CDE90E238DF80F10EFF3118C102383F3DD
:1090E000128803681B6A0BB3069B04A802461BB1D7
:1090F000D3691432002BFBD12B6A6BB1996839B953
:109100009A4209D0196829B15B6899680029F7D09B
:109110001433F3E7C3E900405FFA8CFC8CF3118849
:109120002268136A002BFCD10120A4E704AB2B6258
:109130005FFA8CFC8CF31188F1F74CFAF0E700BF72
:1091400030B40568EFF3118C102383F312880368A1
:109150001B6AEBB18B6804460A461BB1D369143213
:10916000002BFBD12B6A6BB1986838B9934209D0B8
:10917000186828B15B6898680028F7D01433F3E7C3
:10918000C3E900415FFA8CFC8CF3118830BC704756
:1091900029625FFA8CFC8CF3118830BCF1F71ABAA3
:1091A00030B5056895F800E0BEF1010F95B00446B2
:1091B0008C4608D0BEF1020F02D119462B6A7BB152
:1091C000002015B030BD95F90400411CF8D00228EC
:1091D000F6DC217900926246F2F7C6FC15B030BD8C
:1091E000CDE90A210DF10F0204920122CDE90532E9
:1091F000CDE908336CF07F018DF81C308DF83020FC
:109200008DF844200D931093129300220023CDE992
:109210000E238DF80F10EFF3118C102383F31288B7
:1092200003681B6A0BB3069B04A802461BB1D369F3
:109230001432002BFBD12B6A6BB1996839B99A4271
:1092400009D0196829B15B6899680029F7D01433EF
:10925000F3E7C3E900405FFA8CFC8CF311882268C5
:10926000136A002BFCD10120ABE704AB2B625FFA41
:109270008CFC8CF31188F1F7ADF9F0E730B593B0C1
:1092800000238DF807108DF806200DF1060101224C
:10929000CDE90332CDE90631CDE908320DF10705FC
:1092A0008DF814308DF828208DF83C200B930E9308
:1092B000109300220023CDE90C2301680295044697
:1092C000EFF3118C102383F3128803681B6A0BB32E
:1092D000049B02A802461BB1D3691432002BFBD1B8
:1092E0000B6A6BB1996839B9934209D0196829B1F1
:1092F0005B6899680029F7D01433F3E7C3E90040AD
:109300005FFA8CFC8CF311882268136A002BFCD165
:1093100013B030BD02AB0B625FFA8CFC8CF311888A
:10932000F1F758F9F0E700BF30B505682C78012C4B
:1093300083B006D0022C01D12B6ACBB1002003B040
:1093400030BD95F904408DF80720631C8E460179E5
:10935000F4D0022CF2DC0DF107037246204640F0F7
:1093600025FD0028EAD02046F2F776FB03B030BD99
:10937000FFF784FF0120E2E730B595B0002301221A
:10938000CDE90532CDE908338DF81C300D931093EB
:1093900012930DF10F030DF107050B928DF830209C
:1093A0008DF844200A93002200238DF80710CDE9A0
:1093B0000E23016804950446EFF3118C102383F308
:1093C000128803681B6A1BB3069B04A802461BB1E4
:1093D000D3691432002BFBD10B6A6BB1996839B990
:1093E000934209D0196829B15B6899680029F7D0C0
:1093F0001433F3E7C3E900405FFA8CFC8CF3118867
:109400002268136A002BFCD19DF80F0015B030BD07
:1094100004AB0B625FFA8CFC8CF31188F1F7DAF87D
:10942000EEE700BF134B1B68B0EB930F14D2B0EB09
:10943000D30F13D2B0EB131F12D2B0EB531F11D2C4
:10944000B0EB931F10D2B0EBD31F0FD2B0EB132FA2
:109450000ED24FF48070704702207047042070478E
:109460000820704710207047202070474020704728
:109470008020704794200020013902292DD81C4BF0
:1094800001EB810C10B403F16C0403EBCC0304EB8F
:10949000CC0493F86C2004604FF0010C022A80F891
:1094A00088C003F16C041AD0C9B2124A090152589B
:1094B0001A6772B1022283F86C2000F110014FF498
:1094C00080724C30A281C3E921105DF8044B6046E4
:1094D000704700205DF8044B70470020704793F8F8
:1094E00079205DF8044B6244604683F87920704728
:1094F0007CAB00204824002010B5036804469B681C
:109500009847FF230122A373627310BD036810B54F
:1095100004461B689847236801219B6820469847AA
:10952000E37B0133E37310BDF0B583B00446089FBD
:109530000193384616460D4642F08EFD2268E672CB
:109540002844A0729769019B324629462046BC46B2
:1095500003B0BDE8F040604703689B6A184700BF4E
:1095600003685B6D03B11847704700BF0368DB6C8D
:1095700003B11847704700BF002310B5C37342748E
:109580008A6C0160044603730AB119469047236848
:1095900001219B6820469847FF222368A273DB6C59
:1095A000012262731BB12046BDE81040184710BD70
:1095B000074A00235168814202F1240203F10103AA
:1095C00003D0102BF6D100207047D8B2704700BFEF
:1095D000140200202DE9F04F984A537C012B85B0EE
:1095E00021D0022B17D000230193954BDFF864B2F2
:1095F0004FF0000A99469BF80030022B15D00AF173
:10960000010ABAF1030F0BF1280B09F10509F2D198
:1096100005B0BDE8F08F93792BB19378083B18BF64
:1096200001230193E1E70193DFE799F903506A1CF5
:1096300000F0E780EDB22B465FFA8AF6721C0C212F
:1096400002921F46012D4FFA85F800F2D3800823BD
:109650007C4A11FB083C002405E00134152C02F182
:109660001C0200F0C7801378002BF6D15378B34268
:10967000F3D152F80C000028EFD0FFF799FF019BBF
:109680000C2123B1A0F10903072B40F2B8806E4AE8
:1096900000F1FF3C0CEBCC0302EB83031A7F002AA2
:1096A00040F0A8804FF014021A77029A5A770028E7
:1096B00000F0A08007461846C4EBC403614ACBF80B
:1096C000100008EB48089B0003EB88031344DB6899
:1096D000C360DCF1000303F007030CF0070C58BF74
:1096E000C3F1000C80F808C03846F1F783FB99F904
:1096F00004506B1C00F08880EDB229465FFA8AF6B0
:10970000731CCDE902370F46012D4FFA85F851D869
:109710000C2208214B4B12FB081C002404E00134EE
:10972000152C03F11C0345D01A78012AF7D15A7879
:10973000B242F4D153F80C000028F0D0FFF738FF04
:10974000019B1BB1A0F10903072B37D93E4B00F158
:10975000FF3C0CEBCC0203EB8202137F53BB4FF0B8
:10976000130111770299517720B31146C4EBC40459
:109770004246029302EB4202324B039FCBF8141095
:10978000A40004EB82021A448046D268CA60DCF16D
:10979000000202F007020CF0070C58BFC2F1000CE7
:1097A00081F808C0F1F726FB029B87BB0023CBE9B9
:1097B000043324E70135EDB2AF42A5D2039F002F59
:1097C000F4D0214A2423781E03FB00200024CBF888
:1097D0001000CBF81440F0F731FE5846F0F700FEC9
:1097E00023461A4922463846F1F71EFB01238BF81F
:1097F0000C3004E70135EDB2BD427FF623AF002700
:1098000075E70123002517E70121002576E7DBF83E
:1098100014000293F0F712FEDBF81000F0F70EFED2
:109820005846F0F7DDFD029B09491A464046F1F71C
:10983000FBFA01238BF80C30E1E600BF9C270020E7
:10984000F4680020F8EB0508140200200D7E0108E2
:10985000997D0108E8AB00204A484B494B4BDFF8A3
:1098600030C12DE9F04F4FF0010A4FF002094FF0DF
:10987000040808271026202540244FF0800E30F8D9
:10988000022B12F0010F03D01960A3F804A00833D3
:1098900012F0020F03D01960A3F80490083312F0FD
:1098A000040F03D01960A3F80480083312F0080FE6
:1098B00002D019609F80083312F0100F02D0196097
:1098C0009E80083312F0200F02D019609D8008336B
:1098D00012F0400F02D019609C80083312F0800F04
:1098E00003D01960A3F804E0083312F4807F05D098
:1098F0004FF4807B1960A3F804B0083312F4007FA2
:1099000005D04FF4007B1960A3F804B0083312F4BB
:10991000806F05D04FF4806B1960A3F804B0083352
:1099200012F4006F05D04FF4006B1960A3F804B077
:10993000083312F4805F05D04FF4805B1960A3F800
:1099400004B0083312F4005F05D04FF4005B1960D7
:10995000A3F804B0083312F4804F05D04FF4804BC5
:109960001960A3F804B00833D20B04D04FF40042BE
:1099700019609A80083301F5806161457FF47FAFFB
:10998000BDE8F08F74EE0508000002407C24002042
:109990000018024010B50409013C052C16D80D4AE8
:1099A00032F8141000F00F0341FA03F212F0010232
:1099B0000ED0012098400138084043F079F8064B5A
:1099C000064A1B5D184402EBC00010BD002010BD0C
:1099D000104610BD74EE050880EE05087C240020BA
:1099E000F8B50C4F97F834308BB10B4C0025A668B6
:1099F00030790135FFF7CEFF18B1217DF279F1F70B
:109A0000B9FC97F83430AB4204F18C04EFDC012050
:109A1000F8BD00BF840A00106419002038B505465F
:109A200000780C46FFF7B6FF611CC9B2044610B1BE
:109A300041238371C17120466978F1F70FFBAB7840
:109A400020461BB1BDE83840F0F7BEBCBDE8384049
:109A5000F0F7C0BC0D4B2DE9F0411F680C4E0546D8
:109A60000024A74201DCBDE8F08104EB440303EBD2
:109A70000608F05CFFF78EFF854204D12146404680
